:020000040800F2
:1000000000A000200513010849C4000839030108B5
:1000100047C4000845C4000843C4000800000000AD
:1000200000000000000000000000000041C40008C3
:100030003FC40008000000003DC4000837F000087D
:100040006D1301086D1301086D1301086D1301088C
:100050006D1301086D1301086D1301086D1301087C
:100060006D130108E9D500086D1301086D1301082F
:100070006D1301086D540008FBB300086D130108EF
:100080006D1301086D1301086D1301086D1301084C
:10009000A9C400086D1301086D1301086D13010850
:1000A0002DD6000859D600081DD6000869D60008CC
:1000B0004DD600083DD600086D1301086D130108E8
:1000C0006D1301086D1301086D1301086D1301080C
:1000D0006D13010825D8000819D800080DD80008AC
:1000E00045F000086D1301087DF900086D13010843
:1000F0006D1301086D1301086D1301086D130108DC
:100100000000000000000000000000006D13010866
:100110006D1301086D1301086D1301086D130108BB
:100120006D1301086D1301086D1301086D130108AB
:100130006D1301086D1301080000000000000000AD
:100140006D1301086D1301086D1301080000000014
:10015000000000000000000000000000000000009F
:1001600000000000000000006D1301086D1301087D
:100170006D130108000000000000000000000000F6
:08018000000000006D130108EE
:100188002DE9F04F2DED068B6D4E6E4B3360AFB001
:10019800002373600DF04BFB18B90DF06BFB09F0F1
:1001A80067F909F023FA684B684C1A7842F00102A3
:1001B8001A70674A4FF47001C2F888100022099239
:1001C8000A92226842F4803222600493236803F47E
:1001D80000330A93099B013309930A9B1BB9099BB6
:1001E800B3F5A04FF2D1236813F4003318BF0123ED
:1001F8000A930A9B012B7AD0554F564BFB60636AD2
:10020800B360636ADFF884B1DFF88481DFF8849132
:1002180043F080736362636943F4FC032EAD63614A
:1002280003238DF86A3041F6FF7325F8503D4FF0EF
:100238009040294605F00CFA4FF6FF7358462946B8
:10024800ADF8683005F004FA4348294605F000FA8D
:100258004248294605F0FCF94148294605F0F8F9D5
:100268002946404805F0F4F9284605F053FF1A9B43
:100278003D4AB3FBF2F33D4A13603D4B3D4A4FF014
:10028800000AC3F800A03C4B5A60F02287F82320EC
:100298000722C3F808A0394F1A60D8F808303B6025
:1002A80099E80300636985E8030043F480236361E8
:1002B8002023CBF818301BA91A9805F0C9F9642037
:1002C8000EF0A6FEC8222E48514613F0C8F8E3697E
:1002D8002C4A43F00303E361A36943F4A123A36118
:1002E800636943F4C023636102F1900C54E0264B28
:1002F80012221A606368636063686360636843F42A
:1003080080636360636823F47C136360636843F409
:10031800E8136360236843F08073236022680B4B03
:100328009201FBD55A6822F003025A605A6842F0DB
:1003380002025A60636803F00C03082BFAD15BE7EA
:10034800580800205B8D0008742A00200010024025
:1003580000ED00E00005FA0500080048000C004820
:10036800001000480014004840420F00DC2500201F
:10037800E02500203F19010010E000E0382A0020A5
:100388002826002078640108002002400004004864
:10039800401D002098440108937B506892F80FE0B4
:1003A80003F00701DB0800EB83038900186A4FF0AC
:1003B8000F0A0EFA01FE0AFA01F120EA0101196298
:1003C800196A10324EEA010162451962E4D100232C
:1003D800DFF89CA20AF10C02002199540133092B81
:1003E800F6D1FF23964A8AF815308AF816308AF82B
:1003F80017308AF818308AF81930924BDFF874B23F
:100408001360914A0393042010705846302213F069
:1004180026F8142202218BF800208BF824100122E0
:100428008A49039B8BF8182098F805B081F800B02A
:10043800A3F5EF71CAF81C1085493F68A3F58F73BF
:100448000B60844B03EBCB035B78CAF82030BB0608
:1004580048BFCAF8202000237F4A40F2DC5122F826
:1004680013100133082BF7D113A800211C2212F016
:10047800F6FFBBF10E0F03D00BF0EF03082B02D1F0
:1004880001238DF85E30022006F0D2FD18B14088B5
:10049800003018BF0120C7F340038DF85230C7F36E
:1004A80080138DF85530C7F340338DF84C30C7F3BF
:1004B800C03300F001008DF84F3017F400638DF859
:1004C800510007D098F8843103F1FF3EDEF10003B4
:1004D80043EB0E038DF85030C7F300438DF85630C8
:1004E800336AB8F844E1ADF862E0003318BF01237D
:1004F8008DF85730C7F300538DF85830B8F84631A7
:10050800ADF85C30B8F85231ADF85A30C7F38043D3
:100518008DF8533098F85431181C07F00101C7F3CF
:10052800C00218BF0120FF0448BF4C4F8DF854008B
:10053800B8F8500144BFB7F84C71ADF86270B0F527
:10054800FA7F8DF84D108DF84E20ADF8600002D975
:100558000BB9ADF8623098F8D431414886F82430A8
:10056800002386F8253043709DF85E30002B0CBFC1
:100578000023022301B902B1013309EB83094FF0CB
:10058800000AD9F808309A1E103303920593039A8B
:1005980032F8023F03924FF6FF72934200F08A81CD
:1005A8009DF851004FEA132CDAB25FFA8CF378B158
:1005B8002C4F2D4807EB02177968814208D13889FA
:1005C800B0F5806F00F07181B0F5006F00F06D81BB
:1005D8009DF8560090B11001DFF888E00EEB000797
:1005E8005EF800E02148864500F05F811E48796882
:1005F800814203D1B87B082800F057819DF852004A
:1006080050B1184F07EB02177868B0F1904F03D13B
:100618003889202800F049819DF84F0050B1114FCA
:10062800114807EB02177968814203D138890428F9
:1006380000F03B81BCF1020F1ED19DF84C1020E068
:10064800282500202E1F0020080F0020C0020020AF
:100658006C27002058660108C80E0020401D0020A5
:100668007D08002078640108000400480044014027
:10067800580800202C250020BCF1010F04D19DF85A
:100688004D10002900F011819DF8571031B19DF8E7
:100698005E1019B9911F012998BF0423CC4F9DF80A
:1006A80058104FEA02194F4431B19DF85E1019B93C
:1006B800043A032A40F2E280012B43D1FF2386F853
:1006C8006C3086F86D30C24BF76703EB09024FF0C8
:1006D8000008517B50688DF86A1002F1080B1289E6
:1006E800ADF868201AA9022286F8708006938DF862
:1006F8006B2086F82880C6F82C80C6F83080C6F8AB
:100708003480C6F8688086F86E8086F86F8004F0BA
:100718009FFF069B9BF8021053F80900424604F01D
:10072800EBFD38460DF0ACFDAA4BAB49C6F880305E
:10073800AA4BC6F88430C6F8888038460A1D0DF0E2
:1007480007F8B2E0022B46D15FFA8AF21C2101FBBE
:1007580002FC06EB0C089E4A88F871A0012188F873
:10076800701002EB09014FF0000B91F80DE048689A
:1007780088F872B001F108020989ADF8681088F8A4
:100788007AB01AA9C8F87C70CDF81CC08DF86AE058
:1007980006928DF86B3004F05BFF8D4B069A53F888
:1007A800090091785A4604F0A7FD38460DF068FD17
:1007B800DDF81CC088498A4AC8F880206144894A03
:1007C800C8F88420C8F888B038460A1D0CF0C0FF65
:1007D8000AF1010A69E0032B4ED19DF85330DFF886
:1007E8003C82DFF83C9203B39DF8543098F826C059
:1007F800DFF800B2CDF818C053B17B4BBDF86020CC
:10080800B3FBF2F23846082192B2BDF8623003E039
:10081800384608214FF6FF7204F043FFDDF818C090
:1008280049F82C00C0F80CB020E0BDF8602098F81A
:1008380026B0BDF86230B2F5FA7F0BD96A49B1FB30
:10084800F2F23846082192B204F02BFF674B49F8C0
:100858002B000AE06649B1FBF2F23846012192B258
:1008680004F01FFF634B49F82B00C36098F826304B
:10087800013388F8263018E0042B16D196F8258025
:10088800BDF85A205A4B93FBF2F23846BDF85C305B
:10089800012192B204F005FF96F8253006EB88088E
:1008A8000133C8F8500186F82530039B059A934216
:1008B8007FF46DAE96F8252086F870214E4A4F4B8E
:1008C80092F800E0AEF117020027022A1F709C463A
:1008D8001AD8F3693B44D3ED007AF5EE407AF1EE8D
:1008E80010FA02D1336A73BB26E0454A07EB0208C7
:1008F8000FCB88E80F009CF8003010370133C02F69
:100908008CF80030E5D1EDE73E4B13F83E908CF8BB
:10091800009003EBCE03D3F804A0BAF1000FE1D0A6
:100928004F45DFDA364A3B0103EB020853440FCB4D
:10093800013788E80F00F3E7334B1A6812F4805F39
:10094800984624D11DE0314B314A13F83E0010700F
:1009580003EBCE035E68002EEED000238342EBDA71
:10096800C3EBC3017218DFF8BC80D2F8009041F8DD
:10097800089001EB08079188B9809279BA71013320
:10098800ECE70EF0EF03082B224B4DD14FE09CF81B
:100998000020012AF5D9204B03EB02121032103344
:1009A8009342EED053ED047AB6EE007A67EE877A7A
:1009B80043ED047A53ED057A67EE877A43ED057ABD
:1009C80053ED037A67EE877A43ED037AE7E700BFD2
:1009D80078640108B9500008D80800209951000827
:1009E800FD5300089150000800127A00B951000820
:1009F80040420F00A9510008C00200202426002010
:100A0800FC01002058660108382A0020404E0108E1
:100A1800F8260020A81A0020040200205808002008
:100A2800F4250020F9260020BEF10E0F09D11A780E
:100A380042F010021A70BEF1180F09D10EF056FDDF
:100A480006E01A7822F010021A70BEF1190FF4E7C6
:100A58000EF030FDD8F80030B84E5F035EBFB84BDB
:100A680001221A70049B049A1B7843F00403137044
:100A780063694FF0010B4FF0020943F40033294634
:100A8800ADF868B08DF86AB08DF86B904FF0904073
:100A9800636104F0DDFDAB4BAB4A1A6000200EF039
:100AA800D5FAE36943F48043E361236943F480435F
:100AB8002361636943F480236361736A23F47003D9
:100AC8007362736A43F4A0037362736A23F07063FA
:100AD8007362736A43F0A0637362736A23F07043AE
:100AE8007362736A43F0A0437362736A23F47023DA
:100AF8007362736A43F4A023002773624FF0030AFA
:100B08004FF46043304629461A938DF86C908DF85F
:100B18006DA08DF86E708DF86F7005F069FC4FF45C
:100B28008052304629461A9203928DF86CB08DF89F
:100B38006DA08DF86E708DF86F7005F059FC236903
:100B48008249039A43F480432361236923F4804351
:100B580023618B8823F480531B041B0C8B808B88A8
:100B68009BB243F480538B800B8803F4415343F4C6
:100B7800457343EA0A030B808B8823F470631B04D4
:100B88001B0C43F4E0638B808B8B23F400631B0402
:100B98001B0C8B8307230B820B889BB243F040030B
:100BA8000B806B4BB2616B4E1E60636943F400337C
:100BB8006361E36943F48003E361236B23F020035B
:100BC8002363236B43F0805343F0200323634FF0E8
:100BD800904318465A6A22F0F0025A625A6A42F062
:100BE80040025A625A6A22F470625A625A6A42F49D
:100BF80080625A6229464FF400721A9203938DF864
:100C08006E708DF86F708DF86C908DF86DA005F092
:100C1800EFFB039B04934FF48062184629461A920F
:100C280005F0E6FB326822F00102326031684A4A78
:100C38000A403260494A3261326842EA0B02326045
:100C4800B760F760B760B26842F40042B2603268D9
:100C58003260726822F0784222F400427260326890
:100C680042EA0B023260D8F800503D4E05F40043CA
:100C7800102230463946039312F0F1FB4FF6FF720B
:100C880015EA09050E928DF83D908DF83E708DF8A5
:100C98003F708DF83CA0049B0ED02EA92022184648
:100CA80041F8802D05F0A4FB072386F800907770A3
:100CB800F37086F802B05D46039B7BB12EA904232E
:100CC80041F8803D1D4805F093FB0C233371072341
:100CD800F371012375711D44B371EDB2E36A2148C4
:100CE80023F4F873E362E36A43F4D873E362636955
:100CF80043F0805343F00203636105F040F91AA8FA
:100D080005F012F9184B1A93184B1B93022D4FF04C
:100D1800000314BF1A4680221F924FF48072114CB0
:100D280020924FF4806221922022204622921AA912
:100D38004FF400521C931E931AE000BF00040048B1
:100D480028070020802A002095EE0008003800407F
:100D58008C0E002000580040FFE0CF00300E5000FD
:100D680034110020080402404001005044110020C2
:100D780023922493ADF8745005F0E3F8236843F008
:100D880001032360C24CA36823F04053A360A36807
:100D980043F08053A3600A200EF03AF9A36823F0C9
:100DA8008043A360A368A360A36843F00043A360E3
:100DB800A368B74A002BFBDB9368B64923F040537E
:100DC8009360936843F0005393608868B24B034084
:100DD80043F468338B60D168B04B0B4043F4005345
:100DE800D360136B013D23F00F0C45EA0C05156326
:100DF800002401233219917800296BD05D1C042B43
:100E0800375DD078DFF888E2EDB20ED803EB430304
:100E18005A00DEF830101F23934021EA030107FA35
:100E280002F30B43CEF8303031E0092B0ED8053BE6
:100E380006225A43DEF834101F23934021EA0301A7
:100E480007FA02F30B43CEF8343020E00E2B4FF0B4
:100E580006010ED8A3F10A024A43DEF838C01F2360
:100E680093402CEA030107FA02F30B43CEF838301B
:100E78000DE00F3B01FB03F2DEF83CC01F2393405B
:100E88002CEA030107FA02F30B43CEF83C30092F92
:100E98007F4A0FD99369A7F10A0303EB43039769C4
:100EA8000721994027EA0101916191699840084317
:100EB80090610EE053697B1E03EB430357693821A9
:100EC800994027EA01015161516903339840084369
:100ED80050612B460434102C8CD16D4B9A6842F02B
:100EE80001029A601A461168694BCE07FBD5DA6889
:100EF8006B4E22F00202DA60DA6842F00202DA602F
:100F0800DA6842F00102DA609A6842F004029A60F4
:100F1800B6F85831002B40F05886B6F95A21002A05
:100F280040F05386B6F95C21002A40F04E86D8F886
:100F380000305C4C13F4003F1FD0C8200EF068F856
:100F4800AE200CF0D7FA08B10CF010F9564D84F821
:100F58007101C8200EF05CF8544BC4F874310021BC
:100F68000C22284612F07BFA0223EB7007F0FFF9F7
:100F78000EF032F84E4B0344AB604E4BDFF8249131
:100F88001B684D48B3F8627096F85F5100210C2237
:100F980012F065FA4FF0000A00211422474812F0B7
:100FA8005EFA51460C2284F878A109F5BE7089F8DA
:100FB80079A112F054FA424BC4F8883123200EF07C
:100FC80027F8752001210BAA0CF0CCF9002800F0B5
:100FD80082803C4BC9F880313B4BC9F8843150467C
:100FE800432301210CAA89F87C310CF0BBF99DF848
:100FF800303003F07E038DF8303040B1682B06D1D5
:10100800012389F878311D2389F87C3163E09DF844
:101018002C3003F07E03682B8DF82C3056D1022338
:10102800062084F878310146D4F880311AAA984706
:101038009DF86D1001F001029DF86B1001F001019F
:101048004B0043EA82019DF8692002F001030B433B
:101058000AD05BB2012B01D1002302E0022B0FD191
:10106800012384F8793136E00E4B0C20D3F8803117
:1010780001210EAA98479DF8383013F00F0303D1C9
:1010880003200EF037F826E0042BE9D1E4E700BF8F
:101098000001005000030050E010FCFF07C0FFFDF6
:1010A800401D002058080020FC0D0020C81E00200C
:1010B800404B4C00D80E0020A8250020B019002075
:1010C800B04401086DD3000861D30008702B04BF39
:1010D800042384F87831454B00221A7094F878215B
:1010E800022A994616D1424B42491960424843495F
:1010F80059604349D96002704249434A1961032142
:1011080089F80010116841F0010EC2F800E09B4612
:10111800924603E001200DF0EDFF88E00A2D2B46F2
:101128004FF0010228BF00239A4040F2B235154023
:10113800B5B912F04D0F13D0344B354A1A60354A01
:101148005A6094F87921002A0CBF6F226E221A7215
:101158000323314A437019431370CAF8001005E09D
:10116800012B4FF00005D9D82B4B1D70DAF8003051
:101178009D0702D5254B1B689847284B4FF47A7278
:1011880000251A6084F88C51DBF80030BC209847A1
:10119800234B96F855211D700AB189F8002096F85E
:1011A80056210AB11C490A7096F8572102B11A70E3
:1011B800DAF80030180737D53FB2642297FBF2F30C
:1011C80002FB137212B207EE902AB8EEE77A07EE26
:1011D800903ADFED146AF8EEE77AE7EE267AB2EE97
:1011E800047A67EE877AC4ED647A20E0C419002097
:1011F800B019002089CD000804010020D1D20008D0
:10120800B5D2000890C1793D940E0020A825002091
:1012180029CE000819D30008962A0020000F0020C4
:10122800932A00208988883C0023C4F89031B94B60
:101238001A7842F002021A70B74A202191610A25F1
:101248000393B54FBB8A9BB283F02003BB8219205E
:101258000DF0DEFE01200DF0F9FE19200DF0D8FE8C
:10126800013D00200DF0F2FE15F0FF05E9D1202325
:10127800BB61AA4B9FEDAA8A1F68DFEDAA8A3B7B58
:1012880000EE103AB8EEC00A20EE080A08F08EF810
:10129800A54B83ED000AA54B1B8807EE903AF8EEA4
:1012A800E77AB7EE007AC7EE277AA14BB0EE680A64
:1012B800C3ED007A9F4BD3ED047A9F4B67EE887A93
:1012C800C3ED007A3B789D4F07EE903AF8EEE77A47
:1012D8009B4BC7EE277AC3ED007A77EE677A994B76
:1012E800C3ED007A984B83ED027AC3ED008AC3ED13
:1012F800018A964B83ED027AC3ED008AC3ED018A19
:1013080008F054F8B0EE408AB0EE680A07F0EEFF35
:1013180020EE006A68EE086A66EE007A8C4BE6EE0C
:10132800887AFF211B2220EE087AC3ED007A67EE47
:10133800007A3846F0EE675AD7EE085AE7EE087A90
:1013480028EE468AC3ED015AA6EE808AC3ED027ADA
:1013580083ED038A7F4B1D7012F081F87E4A7F4B24
:1013680012683D70012112F0020F19701FBF7970C9
:1013780003211970022118BFB970510741BF1978AC
:101388004D1C1D70032548BF7D5412F00A0F3846C6
:101398000CD01A780421B954511CC9B205257D54C2
:1013A800D11C0232D2B219700621B954D8F80010F3
:1013B8008A0641BF1A78551C1D70072548BF8554F9
:1013C8007579082D01D00E2D04D11A78571C1F707D
:1013D8000B2787541A7811F4803F4FF00C0E00F851
:1013E80002E002F101071CBFDFF870E10232FFB230
:1013F8001F701FBF8EF80020504A4FF00E0E02F8E3
:1014080007E04A0741BF1A78571C1F70102748BFCA
:1014180087541A78571CFFB24FF0120E11F4806FE0
:101428001F7000F802E00ED096F810E2BEF1000F2F
:1014380009D0DFF828E102328EF800203F4A4FF049
:10144800130E02F807E08F0541BF1A78571C1F706A
:10145800152748BF8754182D0DD11A781627875499
:10146800571CFFB24FF0170E00F807E0D71C0232E6
:10147800D2B21F7085540D0341BF1A78551C1D70D8
:10148800192548BF8554CA0541BF1A78511C1970DF
:101498001A2148BF81541A78511C19701423835497
:1014A800002198222E4811F0DAFF0CF0D7FF2D4BBF
:1014B8002D4A1A602D4BB6F84E1119802C4900237D
:1014C8000B808B702B490A602B4AB6F89611137063
:1014D80088B22A4A22F813000133122BF9D1284D79
:1014E8002B6813F4805F08BFB6F89C01D0801B07F7
:1014F800A84640F1238196F89031062B00F2188116
:10150800DFE803F00440477692B1B10045F2F052AB
:101518003AE000BF742A002000040048AC1A0020FA
:1015280035FA8E3C00000000A41A002008000020B4
:101538005C1A0020B0190020601A0020A10E0020BB
:10154800C01A0020B01A0020C41A0020B41A0020C3
:10155800941A00201A1A0020940E0020A00E0020D1
:10156800A81C0020EC0D0020C81E0020F00D002053
:10157800482A0020342A00206F0D0020821C0020F9
:10158800382A002042F6F822454B1A800DF004F85C
:10159800CDE007EE901ADFED436A414BB8EEE77AEB
:1015A800DFED417AE7EE267A42F6F8221A80002328
:1015B800FCEEE77A3D4A17EE901A42F82310013301
:1015C800122BF7D13A4A3B4911603B4A402013702D
:1015D80005F00AFE002800F0AB8001234FF0070950
:1015E80090F90000354A8DE808024021344B99E013
:1015F8002B4B42F6F8221A802D4B324A1A602E4B9A
:10160800102240201A7005F0EFFD002800F09080AD
:1016180001234FF0000C90F900002B4A8DE80810C8
:1016280040214FF4E1337DE01D4B42F6F8221A8049
:101638001F4B264A1A60204B082240201A7005F0DA
:10164800D3FD002874D001234FF0000E90F900005C
:101658001F4A8DE8084040214FF4E13305F0E8FBCC
:10166800C4F8940160E00E4ADFF87CE0194F1A4D87
:101678001A4842F6F82111800F490C22062B0A70ED
:1016880034D000232B708EF800303B701B2303707E
:10169800134B1A70134B05221A704FF4E13531E0E1
:1016A800BA010020CDCCCC3F0000B0C46029002096
:1016B800A4000020E900010820250020FD01010800
:1016C800A0860100495B000851010108315B000850
:1016D8007D5C0008C1100020C0100020C21000204E
:1016E80043100020C310002044100020002129705E
:1016F8008EF80010397021210170C349C34D0A705A
:10170800C34A1370C34BC44A1A60402005F06CFDED
:1017180070B101230027C14A90F9000040218DE8EB
:1017280088002B4605F084FB003018BF012028B93B
:10173800082007F063FEB74BB94A1A60D8F80020B2
:10174800B84B12F4804F1FBF12211970B149B64827
:1017580018BF086042F20101114002F0010002F4D2
:10176800005579B1B14944F620670F8025B10821A9
:101778001970A849AE4D0D6020B10C211970A5490A
:10178800AC4808601978AC4F04395970AB49AC4B78
:101798000B60AC4980330B600025D1033D7040F1EC
:1017A800AE8007F0E9F8DFF8D0C2DFF8D0A2CDF8B4
:1017B80018C040F22A334FF001091A4660462946FC
:1017C800059387F8009011F04AFEDAF814209E4835
:1017D8009E4F42F48022CAF81420426A22F00F0277
:1017E8004262426A032142EA090242624FF4807B64
:1017F80002228DF835100CA98DF8342004928DF84A
:101808003650CDF830B08DF8379004F0F1FDDAF8A5
:101818001810049A41F40031CAF81810398821F4D4
:1018280040710904090C39801D21F96238463A854E
:101838000EA93D866022C7F814900E92ADF83E506E
:101848001095ADF84450ADF84650ADF84850ADF895
:101858004A50ADF83C9004F01FFCBA6942F0080207
:10186800BA617A6C42F400427A64DAF8142042EAE7
:101878000902CAF81420AAF57D6A504604F07FFBD5
:101888001AA804F051FB059B714AADF87430802307
:101898001A92DDF818C01F9310224FF400535046D7
:1018A8001AA92393CDF86CC01C921E95CDF880B070
:1018B80021952295249504F044FBFB6843F40073BA
:1018C800FB60DAF8003043F00203CAF800300BA8D6
:1018D8000D238DF82C308DF82D908DF82E508DF825
:1018E8002F900CF0AFFC5B4B1A685B4B43F825203C
:1018F8000135202DF7D103F0CDFD03F0CBFDD8F84D
:1019080000305A0542D5554BD4F8C4741F600420E2
:1019180005F06AFC0421C4F8C80405F03FFC504BEC
:1019280084F8CC0408201F6005F05EFC4D4B4E4D3A
:101938001860082105F032FC2C22002184F8CD041F
:10194800284611F08CFD7C232B708E236B70E023CE
:10195800EB7010207D2385F82B30C4F8D07405F087
:1019680043FC1021C4F8D40405F018FC84F8D8040A
:101978002020C4F8DC7405F037FC2021C4F8E0040A
:1019880005F00CFC84F8E40406F0C8FB374A2E4F37
:10199800138823F040031B041B0C1380138823F0C7
:1019A80038031B041B0C138013889BB243F04003BD
:1019B800138000259F2332208DF838308DF8395058
:1019C8008DF83A508DF83B504FF480590DF020FBBC
:1019D8008DF869501AAD0422A7F8289028460EA958
:1019E8000CF0FAFBC7F818909DF86A309DF869204A
:1019F8001B0243EA02429DF86B3013431C4A934290
:101A08001C4A54D045D83BE04310002090D0030036
:101A1800C3100020A40000204D5A00085D5B000898
:101A28004D010108202500201D010108BA010020F0
:101A38003D0101082D010108B30700208412002090
:101A4800601F00208012002000040048004401406C
:101A580034440140C8440108B4070020340700207A
:101A6800700700208C070020400700200038004045
:101A780018BA20000C000020F009002000100240D5
:101A880089498B420CD001F51A4102318B4209D0A9
:101A98001BE086498B4205D001318B4207D014E008
:101AA800202300E0802313804FF4807302E04FF47A
:101AB800807313805380938811881B0293604B4373
:101AC800D360012384F8E53404E0002313805380B5
:101AD8009360D360D7681FB3FF0AB9464FF0000B75
:101AE800BB450BDA0BEB070A4FEA6A0A4FEACA2032
:101AF800294610220BF014FB0F2806DC07F090F89B
:101B08004FEAC923C4F8E8340AE0002355F8232033
:101B1800013256D10133042BF8D1D1465746DFE7BD
:101B2800D8F80030624A13F4002318BF0123137059
:101B38000DF052FA5F4B18607379052B02BF5E4BAC
:101B48004FF4C8721A805D4B4FF47A721A805C4A5F
:101B5800137843F0080313705A4A137823F00203EA
:101B68001370D8F8002040F6020313406BB1564BAF
:101B780056491960564B03211970564B01211970AB
:101B8800554900230B8055490B80930341BF544BA3
:101B980003221A71DA7844BF42F00102DA70514B1D
:101BA8009B68C8F80030504B01221A70039B039AB7
:101BB8001B7863F07F0313702FB0BDEC068BBDE874
:101BC800F08F0AF1010BBA46A8E71BB208EE103AEB
:101BD800B6F95A31DFED457A454A09EE103AB6F9B9
:101BE8005C31B8EEC88A08EE903A28EE278AB8EE3B
:101BF800C99AF8EEE88A0021B0EE480A29EE279A39
:101C080068EEA78A117007F0D1FBF0EE409AB0EEAB
:101C1800480A07F06BFBB0EE408AB0EE490A07F0BD
:101C2800C5FBB0EE40AAB0EE490A07F05FFBF0EE44
:101C380040AAB0EE680A07F0B9FBB0EE409AB0EEE1
:101C4800680A07F053FB60EE296A68EE097AF0EE3D
:101C5800665AE7EEAA5A274B29EE296A28EE007A37
:101C6800C3ED035AF0EE465A2AEE400AE7EE6A5AE6
:101C7800E6EEAA7AA6EE6A7A29EE0A9A83ED010AB6
:101C880028EE4A8A2AEE290A83ED009AC3ED02AAB1
:101C9800C3ED045A83ED058A83ED067AC3ED077A0E
:101CA80083ED080AFFF743B9152020001740EF001D
:101CB800BE2700208C0100202E1A0020902A002028
:101CC800A81A0020942A00202C110020BA1E0020F7
:101CD800A425002008010020600E0020620E0020CC
:101CE800FC0D0020401D00202807002035FA8E3CFE
:101CF8004C000020081100202DE9F04F9849994C1C
:101D08000A68DFF8989202F59C432DED028B203388
:101D18002360954B1E7887B08A46C6B193490968F7
:101D28008A4240F2EF80013E1E70EBE0D9F80030A5
:101D38008F48072D98BF595D8E4B88BF29461B6871
:101D48009847032D0AD904EB45050136A880884B2E
:101D58001A78F5B2AA421A46E8D820E0D9F8002045
:101D680005F10E0302EB83039988DA880028EAD08C
:101D78004FF47A73401A5843531A90FBF3F040F625
:101D8800C90300F57A70984205DC40F2EE239842C8
:101D9800B8BF184601E040F6CA0080B2D3E7764BD8
:101DA8001B6842F2010B03EA0B0BBBFA8BFB4FEAF1
:101DB8005B1BBBF1000F06D194F8293084F828305A
:101DC8006E4B5978197094F828701FB16B4B1F78B7
:101DD80087F0010792F8008094F82B20D9F80010BA
:101DE8000F230326B2FBF6F606EB460684F82A30E4
:101DF800961B634BF6B2002545454BDA1FB1614887
:101E080030F8150000E03846B1F814E0864503D8EC
:101E1800B1F816E0864513D2E8B28DE80E000EF050
:101E280011FA032DDCBF4FF0010E94F82AC09DE88B
:101E38000E00DEBF0EFA05FE2CEA0E0E84F82AE02C
:101E4800BBF1000F1FD194F874E023F81600BEF11F
:101E5800000F06D1022A16D942484FF0010E80F829
:101E680074E0B3F800E058887044B3F804E07044B4
:101E7800DFF82CE180B22EF8150000B24FF0030E07
:101E880090FBFEF080B2DFF80CE106332EF8150067
:101E98000135B1E794F82A203B493C4BA2F10F07E2
:101EA8007A427A4184F88E206AB1394A126856011A
:101EB80009D40A68D9689A60521AC82A1DD9012219
:101EC80083F8212019E02D4A0120507010700A680B
:101ED8009968DA605B68521A9A4282BF2B4B0022DB
:101EE80083F821200025454507DAE8B20EF0AAF963
:101EF800284B23F815000135F5E794F82B3001330A
:101F080084F82B301C4B1A6812F4805F984605D071
:101F18001F4B1B68DD0701D40DF0B2FED9F8007025
:101F2800DAF80010BB7A002B3CD0013B19483A7B09
:101F380030F813301AB1C3F53B6308339BB21BB2B8
:101F4800A3F57A73B3F57A7FA8BF4FF47A7323EABF
:101F5800E37307EE903A9FED107AF8EEE77A5AE0CD
:101F6800782A0020440D0020402A00203C2A002026
:101F780020250020A4000020382A0020030000208B
:101F8800700D0020480D0020442A0020482A002017
:101F98009C0E0020821C002000007A44342A002075
:101FA800BA0D0020D8F80020100440D5D4F89000CD
:101FB800914E081A00283ADB904A01F59C402030DF
:101FC800C6F8900050798E4A32F81050A8B2FD7ABF
:101FD80090FBF5F596F89400013000F00F0286F8B2
:101FE8009420324482F895501A468648185C01338A
:101FF8000244102B92B2F8D112B292FBF3F31BB247
:10200800642BA8BF642323EAE37307EE903A9FED9D
:102018007E7AF8EEE77AC7EE877A7C4A9FED7C7A7B
:1020280067EE877AFCEEE77A17EE903A1380D8F8D5
:102038000030784F13F4807F00F00581764BDFF88D
:10204800E891994205D999F8022012B9012289F834
:10205800022099F80220002A00F0F5806F4A94F8CF
:10206800285011683E78002DC1F38063C6F38006BE
:102078000093924614BF4FF0000B4FF0030B99F8F2
:102088002020052A00F2D980DFE802F0034D5275BE
:1020980084A1002E3AD0D4F8A800B4F8AC100CF003
:1020A80056FF012809D15E495E4A09681268C98845
:1020B800642000FB0122C9F81020009B6BB1584A2C
:1020C800126812794AB10DF0EDFF032289F8202039
:1020D8004FF47A72C9F81C20D1E7002D40F0AD808A
:1020E800504AD9F8101010684F4A88420AD901920C
:1020F8000DF0D8FF019A032182F8201040F6B8317C
:10210800D161BCE7012182F82010B8E7009B4FF4A9
:10211800806013B107F062F901E007F04FF900227F
:10212800C9F8102089E0002D46D10DF0BBFFA6E7C5
:1021380025B1052289F82020012000E0284666B153
:10214800D4F8A820D189394A118051809180344926
:1021580009684988D1804FF0020B324A1168D9F8D2
:102168001420914201D8002E64D147F23052C9F8A8
:102178001C20032221E03A7842F002023A700DF066
:102188007FFD284AD9F81C1012680A44C9F818209B
:10219800042212E0234A9DB11168D9F8182091420F
:1021A8004BD9234A92781AB9DAF80020D10744D4D7
:1021B8003A7822F002023A70052289F820205EE778
:1021C8001268D9F81C100A44C9F8182035E01449D7
:1021D800144A09681268C988642000FB0122C9F8FA
:1021E80010204FF48060002289F8202089F803200D
:1021F80007F0E4F843E700BF440D00203411002045
:1022080044110020D90D00200000C842FA0E002019
:1022180000C07F44942A0020404B4C009C0E0020B4
:102228005C290020442A0020482A0020821C002023
:102238000300002000287FF422AFBBF1000F02D07A
:1022480058460CF01DFF8D4D05F5C470B5F84E11BC
:102258000CF07DFE834668B90DF016FF884BC3F875
:1022680000B0C3F804B0C3F808B0864B00221A6067
:102278005A609A603B785A0736D5D8F80030DB06A2
:1022880032D5814B1B78DE062ED4804B9B7893B1D8
:1022980095F8E031BBF1000F15D17BB17C4B1A6882
:1022A800D4F8B0309B1A002B08DA0DF0E9FC794B12
:1022B80083F8B4B018E0BBF1000F0DD110200CF07A
:1022C800DFFE01230EE03BB1714A12684FF47A71C8
:1022D80001FB0323C4F8B03094F8B43023B10CF0F8
:1022E800BBFE002384F8B430002295F8DEA195F8EF
:1022F800DF11B5F898E1B5F89AC113466648009021
:1023080030F912609B087645C4BF63F07F03DBB2E7
:1023180001326645B8BF43F04003042AEED194F871
:10232800B5205C489A4205D190F8B620F92A04D81D
:10233800013200E0002280F8B62084F8B530534B13
:10234800564E9A789946E2B93368D80708D5BBF152
:10235800000F16D13B78DA0713D50DF013FB10E008
:102368003B785B070DD54B4B93F828304BB14C4B62
:10237800DB7833B911B10DF083FC02E0BBF1000F3B
:10238800F9D094F8B630434ADFF82CB1142B40F05A
:10239800A58099F802301AF1000A18BF4FF0010A17
:1023A8006BB392F8B5305F2B11D13B7803F004037F
:1023B80003F0FF0113B10DF063FC08E00B2002915C
:1023C80001920CF05DFE019A029982F8B610BAF1FA
:1023D800000F14D094F8B5307D2B10D13B7803F062
:1023E800040303F0FF0213B10DF04AFC07E00B20D1
:1023F80001920CF045FE274B019A83F8B6203B78F2
:1024080003F0040303F0FF01002B67D194F8B53003
:10241800204A572B0BD1234B4FF47A721A80224B48
:102428001B6813F0080359D1204A138056E0D8F8E6
:102438000000400716D55A2B14D11D4B187820B12F
:1024480019701C4B01221A7048E092F8B73083F0DB
:10245800010382F8B7300BB10C2000E00D200CF01E
:102468000FFE3BE05D2B00F034845B2B00F03384DF
:102478005E2B23D1032000F02FBC00BF401D00209D
:1024880054190020EC120020A81A00200300002094
:10249800442A0020440D0020821C00209C0E0020AD
:1024A800482A0020902A0020940E0020F80E0020D0
:1024B800591A00205A1A0020D80E0020562B01D194
:1024C80007F026FA99F80230002B00F01A8494F8E5
:1024D800B5306F2B40F00F840DF054FAD8F8003067
:1024E8005A0732D594F8B730A3B13B785B0711D5BA
:1024F800009BB3F90620B5F898319A420ADD336893
:1025080013F0010301BFAC4A32211180AB4A08BF66
:1025180082F8B7303368D8030AD5A94B1A782AB994
:10252800A84A127812B9A44A3221118001220BE07C
:10253800A44A13784BB13B7803F0040303F0FF017E
:102548001BB9A14B117001221A70DBF800A00023FF
:1025580033600AF187090AF1D70B99F8002099F836
:10256800013019F8010C9A420BD249460CF0B8FC1C
:1025780038B119F8022C012303FA02F23368134325
:10258800336009F10409D945E7D1904B1B782BB189
:102598008F4E3368990700F13D8334E30AF1D6067C
:1025A8000AF58F793278737816F8010C9A4225D299
:1025B80031460CF095FC08B3B37896F804C0854A08
:1025C80096F803A07D480C21013B01FB0C4103EB6D
:1025D80043031344D1F8C8209A420FD0C1F8C83039
:1025E800002390F8F420C1F8CC30012303FA0CF34F
:1025F80022EA030381F8C4A080F8F43006364E4579
:10260800D0D1754B1E68754B1B68029394F828301F
:102618000393734B009300230193009B1A68002ACD
:1026280000F0E68292F800A0BAF1000F00F0E08214
:102638005B680299CB1A002B0CDB01F5FA73009941
:102648004B60019901238B4094F8F41021EA0303AD
:1026580084F8F430039B002B00F0CA82009B517869
:1026680013F8043C0433DBB2002940F080825D4952
:1026780031F91310B5F8963103F1C800814202DD33
:1026880092F802B015E0C83B994203DA9178C1F19B
:10269800000B0EE0019A0123934094F8F42022EAFB
:1026A800030384F8F430029B009A03F5FA7353602D
:1026B8009EE2019A94F8F4301341DA0700F1988207
:1026C800BBF1000FCCBF022001200CF0FBFC0AF18B
:1026D800FF33DFF8E890132B00F28282DFE813F073
:1026E8001400250037004B0064008A00ED005001FB
:1026F800B701E501150280024B005A008A00ED007F
:102708005001BF002201870196F80090D944B9F121
:10271800FA0FA8BF4FF0FA0929EAE979304686F896
:1027280000900CF0C3FB01200FE096F80190D9440B
:10273800B9F1640FA8BF4FF0640929EAE979304676
:1027480086F801900CF0B2FB02204946DAE196F8CF
:1027580003A0DA44BAF1640FA8BF4FF0640A2AEA6A
:10276800EA7A86F803A03046D9F8F81004F044FD58
:1027780003205146C6E1717959446429A8BF6421F0
:1027880021EAE17171710D200CF012FCBAF10D0F04
:1027980000F02682317959446429A8BF642121EACE
:1027A800E17131710E20ADE1B179594481F308012D
:1027B800B1710520A6E100BF401A0020440D002099
:1027C800581A0020591A00205A1A0020952A002069
:1027D8009C0E0020F8440108040F0020442A002021
:1027E8000C0E0020821C002000007A440000C84221
:1027F80000000000D9F8FC301A78022A20D107EE30
:1028080090BAB8EEE70A5FED077A93ED097A80EEA1
:10281800270A30EE070AB5EEC00AF1EE10FA07D41F
:10282800B4EE670AF1EE10FAC8BFB0EE670A01E02D
:102838001FED110A83ED090A0F200CF0A3FB0AE033
:1028480099785944C829A8BFC82121EAE17199702B
:102858000F200CF0ADFBBAF10F0F00F0C181D9F8D1
:10286800FC301A78022A1ED107EE90BAB8EEE78A31
:102878005FED227A93ED080A88EE278A38EE000A7F
:10288800B5EEC00AF1EE10FA07D4B4EE670AF1EE1D
:1028980010FAC8BFB0EE670A01E01FED2B0A83EDFE
:1028A800080A122056E159785944C829A8BFC821F6
:1028B80021EAE1715970122024E1D9F8FC301A7824
:1028C800022A20D107EE90BAB8EEE70A5FED397A0E
:1028D80093ED0C7A80EE270A30EE070AB5EEC00AAF
:1028E800F1EE10FA07D4B4EE670AF1EE10FAC8BF99
:1028F800B0EE670A01E01FED420A83ED0C0A1020D2
:102908000CF040FB0AE0197B5944C829A8BFC8212C
:1029180021EAE171197310200CF04AFBBAF1100F8B
:1029280000F05E81D9F8FC301A78022A1ED107EE31
:1029380090BAB8EEE78A5FED537A93ED0B0A88EE0A
:10294800278A38EE000AB5EEC00AF1EE10FA07D46D
:10295800B4EE670AF1EE10FAC8BFB0EE670A01E0FC
:102968001FED5D0A83ED0B0A1320F3E0D97A594471
:10297800C829A8BFC82121EAE171D9721320C1E092
:10298800D9F8FC301A78022A22D107EE90BA1FED46
:102998006A0AF8EEE77A87EE800AD3ED0F7A30EE0E
:1029A800270AB5EEC00AF1EE10FA09D45FED717A84
:1029B800B4EE670AF1EE10FAC8BFB0EE670A01E09C
:1029C8001FED750A83ED0F0A11200CF0DBFA0AE0FF
:1029D800997D5944C829A8BFC82121EAE171997590
:1029E80011200CF0E5FABAF1110F00F0F980D9F8CE
:1029F800FC301A78022A20D107EE90BA1FED860A19
:102A0800B8EEE78A88EE008A93ED0E0A38EE000ADF
:102A1800B5EEC00AF1EE10FA09D45FED8C7AB4EE87
:102A2800670AF1EE10FAC8BFB0EE670A01E01FEDC1
:102A3800900A83ED0E0A14208CE0597D5944C82968
:102A4800A8BFC82121EAE171597514205AE0D9F8C4
:102A5800FC301A78022A1ED107EE90BAB8EEE78A3F
:102A68005FED9E7A93ED0A0A88EE278A38EE000A0F
:102A7800B5EEC00AF1EE10FA07D4B4EE670AF1EE2B
:102A880010FAC8BFB0EE670A01E01FEDA70A83ED90
:102A98000A0A09205EE0D9785944C829A8BFC82184
:102AA80021EAE171D97009202CE0D9F8FC301A78B4
:102AB800022A1ED107EE90BAB8EEE78A5FEDB57A22
:102AC80093ED0D0A88EE278A38EE000AB5EEC00AA3
:102AD800F1EE10FA07D4B4EE670AF1EE10FAC8BFA7
:102AE800B0EE670A01E01FEDBE0A83ED0D0A0A2069
:102AF80030E0597B5944C829A8BFC82121EAE171AF
:102B080059730A200CF054FA6AE0D9F8FC301A78A4
:102B1800022A22D107EE90BA1FEDCD0AB8EEE78A55
:102B280088EE008A93ED100A38EE000AB5EEC00A66
:102B3800F1EE10FA09D45FEDD37AB4EE670AF1EE3C
:102B480010FAC8BFB0EE670A01E01FEDD70A83ED9F
:102B5800100A0B200CF016FA42E0D97D5944C82916
:102B6800A8BFC82121EAE171D9750B20CAE701295C
:102B780036D190788F4A32F91390B9F5617F05DB29
:102B880040F633039945A8BF994601E04FF46179AF
:102B9800BAF10C0F24D1884A4FF4966393FBF0F0F6
:102BA8001378A9F5617999FBF0F95FFA89F94B4532
:102BB80016D0B9F1040F34BF4B46022313707F4A75
:102BC8000AFB035303F2AA73136006F0EBFC5046AA
:102BD80049460CF0EDF909F10100C0B20CF072FAA7
:102BE800019A0123934094F8F420134384F8F430B5
:102BF800019B01330193009B0C330093019B042B31
:102C08007FF40BADC4E4D8F80030DB0511D56C4B6C
:102C1800DB7873B16B4B1B689C070AD56A4B1B8822
:102C280013F001040AD10DF02FFA012006F0D6FBAB
:102C380004E0012006F0C2FB012300E00023326813
:102C480050070DD563B1012006F0B8FB5E4B1B8819
:102C5800990708D40DF018FA022006F0BFFB02E02D
:102C6800022006F0ABFB33681A054FF4807002D5DA
:102C780006F0B4FB01E006F0A1FB6B79082B01D04C
:102C88000E2B02D1402006F099FBD8F800305B05E6
:102C980040F18B8095F810321BB93B7813F0040F84
:102CA80002E0336813F4002F0AD0484B00221A7050
:102CB8003C200BF0B7FC002877D00BF005FEF7E7B7
:102CC80005F02CFA07B0BDEC028BBDE8F04F0BF015
:102CD800C5BB012000E002205FFA80F909F1FF334B
:102CE80085F8A83706F0C4FB06F080FC48460CF0CF
:102CF800E9F9FFF7F3BBBAF1000F02D07E2B3FF4DE
:102D0800EBAB94F8B530324A972B05D1314B4FF4E1
:102D1800C8721A80FFF7E2BBA72B06D12E4A137898
:102D280043F004031370FFF7D9BB0021BB2B0591B7
:102D380001D1022303E0B72B04D14FF6FE73ADF89F
:102D4800163009E0BE2B01D1022303E0BD2B1AD1B6
:102D58004FF6FE73ADF81430DBF80030BDF81410F0
:102D6800B3F864200A44A3F86420BDF81610B3F839
:102D780066200A44A3F8662006F0CAFD002384F8FA
:102D8800B630FFF7ABBB792B04D192F8BB3023F0F8
:102D9800010306E07A2B7FF4A1AB92F8BB3043F035
:102DA800010382F8BB30FFF799BB07B0BDEC028B7B
:102DB800BDE8F08F821C00207C250020040F002035
:102DC800482A0020940E0020980E00202525002077
:102DD800440D00202E1A0020A81A00202DE9F04FDB
:102DE800BB4BB3F90610BB4B2DED028B1F687A89DC
:102DF80091B0914201930EDBB1F5FA6FFC79BDBF3A
:102E08008B1A6343A2F5FA64C4F16404BCBF93FB54
:102E1800F4F4643400E06424AF4AB04BB2F896A1ED
:102E280092F95E211868049092B205920546002234
:102E38000293A74B33F912300393CAEB030303F24F
:102E4800F31640F2E63086424FEA420B03D8002BD5
:102E5800B8BF5B4201E04FF4FA73022A00934FF0C7
:102E68006400049B9E4E31D093F81DE1BEF1000F23
:102E780006D0009B7345CCBFCEEB03030023009321
:102E8800009BDFF8A0E293FBF0FC6FF063093EF8CB
:102E98001C8009FB0C390CF1010C3EF91CE00FFAFF
:102EA80088FCCCEB0E0E0EFB09FE9EFBF0FEC64422
:102EB80026F80BE0BE18367973438A4E93FBF6F377
:102EC80064339BB2634393FBF0F031E093F81EE167
:102ED800BEF1000F06D0009B7345CCBFCEEB0303B9
:102EE80000230093009BDFF8288293FBF0F06FF03B
:102EF800630C38F910E00CFB00390130BDF81430D0
:102F080038F91000CEEB000000FB09F999FBFCF939
:102F1800CEEB090919FB03F9009BA6F80490B879D0
:102F2800002BB8BF5B4243436E4893FBF0F064301C
:102F38006B786D4E4FF0640E434393FBFEF3B3542E
:102F48006A4EEB7A434393FBFEF3B3546B7D644EB6
:102F58005843674B90FBFEF0022A9854654B0FD1FB
:102F680083F802E0039B53450EDB5B4CB4F89821D1
:102F7800914215DBB1F5FA6FA8BF4FF4FA6110E082
:102F88009C54039B534504DA36F80B305B4226F811
:102F98000B300132032A05F101057FF44AAFE4E75B
:102FA8001146891A4FF47A73DFF87CE14C4D594386
:102FB8006FF06303C2F5FA626427B1FBF2F191FB8B
:102FC800F7F23EF8120003FB0211013203B23EF998
:102FD8001220D21A514391FBF7F30344F380464B76
:102FE8001B885B0635D5454B454A1B881288DFEDA3
:102FF800457A9B1A1BB208EE103AB8EEC88A28EE3A
:10300800278AB0EE480A06F0D1F9F0EE408AB0EE11
:10301800480A06F06BF9B5F9023006EE903AB5F9B0
:103028000030F8EEE66A07EE903A20EE667AF8EE9F
:10303800E77AA7EEA87A67EE807ABDEEC77AE6EE61
:10304800A87A17EE103AFDEEE77A2B8017EE903A41
:103058006B802D4D2B689F0740F1A1802B4B2C4F87
:103068001A687B6945F20721D31A8B4240F397808F
:103078007A6103F0D1FA274BDFF8B0901A78032A67
:103088009846B9F8003053D10A2B5BD90023282081
:1030980088F800300BF0BCFF03F0BEFA1E4B18880E
:1030A80003F0A4FA1D4B1A68D37890FBF3F00130B3
:1030B80008281B4BA8BF08201870537980B213FB4F
:1030C80000F33B83137913FB00F078833AE000BFE9
:1030D800821C0020040F0020401D0020D80E002074
:1030E8003C1900200CFEFFFF00130020560E0020A4
:1030F8001413002044190020980E0020F80E002018
:10310800BC27002035FA8E3C382A0020782A002077
:10311800480E0020A42500204C1100202C1100206E
:1031280008010020CC25002032120020D8110020F0
:103138000A2B07D80323A04A88F80030002313700D
:103148003B837B8398F800309C4A012B0CD002D338
:10315800022B1BD023E03A8BB9F800309A421EDDCF
:10316800012388F800300FE0B9F800107B8B8B4200
:1031780002DD022313700FE0914B1B8B0133994240
:1031880002DD002313700AE0082006E07B8BB9F803
:10319800002001339A42E3DC07200BF071FFD5F8D9
:1031A80000B0884D1BF4006F78D0874B844F1B68A4
:1031B800FA69C2EB030845F2072290456EDDFB6110
:1031C800824BB6F906C0D3F80090B4F84E1199F8BE
:1031D8000A307F4E012BACF57A7C03D045D3022B05
:1031E80020D044E07B4B396A5A7B7B4B33F8122062
:1031F800082092B291FBF0F3C91A8B18BA843B628B
:1032080040F6E44293FBF0F39BB25343B9F808202D
:10321800C2EB13334FF47A725343B9F9062093FB88
:10322800F2F323E02B78B9F808A0C6F800A05807F5
:103238001DD56A48CDF800C00BF089FEDDF800C046
:1032480020B91BF0100F18BF4FF0000C32220CFBF6
:103258000CF393FBF2F3B9F9062063445A434FF495
:103268007A7392FBF3F3534400E000233360D7E909
:103278000A01336803FB08F84FF47A7398FBF3F8F4
:1032880010EB080241EBE873C7E90A231046194618
:10329800534A00230DF06EFA524B1860524F0097B4
:1032A8003B6813F4805F02D00A200BF0E9FE4F4E12
:1032B8003268002A57D04E494E4B08681F6887422B
:1032C800894698464FD84C4BDFF838A11878516892
:1032D80008BB01201870BAF80030CB5C5BB31378D8
:1032E800013B00FA03F2D4F8D4371A4201D10BF0AB
:1032F800ADFE424B01221A700CF0F4FFBAF8003010
:10330800CBB933681B78053B012B14D80BF064FE4E
:103318003B4B18600FE04FF0000B83F800B0BAF891
:103328000030CB5C3BB158460BF090FE334B83F832
:1033380000B00CF0D7FF3268BAF800305268314854
:10334800D25CFE2A01D100230CE0FF2A02D10BF047
:1033580083FE08E0D9F800600A2111FB0262C8F870
:103368000020013303802B78590703D5264B2022F0
:103378001A8561E0009A1268D2075EBF114A43F0CD
:1033880001031370214B1B781F075EBF2B7823F0B6
:1033980001032B701E4B1A88184B1AB11D4A12686C
:1033A800960702D41C4A1288C2B302221A702B78DC
:1033B80023F001032B7036E008010020A42500202B
:1033C800480E0020942A0020782A00202C11002082
:1033D800FC0E00203411002044110020C81E0020DB
:1033E800407E0500301100209C0E0020F0250020B2
:1033F800442A0020E8250020E42500206C2A00202B
:1034080040290020EC25002000040048A81A0020CC
:103418002E1A0020940E0020902A00202978C80730
:1034280058BF02221A700BF0D7FDB44B1B68C01AA4
:10343800002801DB0CF056FFB14F04F06FFE3E7818
:10344800002E00F0AC80AF4B1A689846002A00F0B6
:10345800BD86D8F800000BF09BFE002800F0B68669
:10346800A84BA94C18680BF090FE092801D03F28FA
:1034780052D14FF0000A2668DFF8C892554636B197
:10348800A248D9F80010324610F036F810B9CA46EA
:1034980005B94D469E4B09F110099945EFD3EDB199
:1034A800D5F800C0DAF8009023681CF803E019F892
:1034B8000300704512D15A1C944958B92D2B09D8CC
:1034C800DFF844E2CEF800204FF0200E01F803E0C8
:1034D800885403E001F803E02260E5E723680BB1B4
:1034E800554510D08B480BF0E7FA554507D855F8E5
:1034F800100B0BF0E1FA09200BF0D6FAF5E7864835
:103508000BF0DAFA002623689E42A2D27F4B985D20
:103518000BF0CAFA0136F6E72368002B40F03C8628
:10352800042840F05E86794803F0F4FF00F04EBEB0
:10353800D9F80000DFF8ECA10BF02AFE28B3DAF87E
:1035480000000BF022FEDBF8003093F8481002462A
:10355800A9BB24286CD1012283F84820DBF800306D
:10356800DFF8E4A193F84820062AE1D193F849004E
:1035780000F0C2FE8346002800F083800BF0F0F9CB
:10358800D8F80030002283F84820644B93F837308D
:10359800002B40F0EF854C36982E00F01786604BD4
:1035A800F21892F84A100129F5D1DFF89C81F358F6
:1035B800C8F800205B4AC34613609146B8E7012962
:1035C80004D14D2814BF00220222C5E7022904D1E4
:1035D8003C2814BF00220322BEE703290CD140284F
:1035E8004FF0000102D983F84810B7E758711971F4
:1035F800D97198710422AFE7042906D1997983F823
:1036080049004A409A710522A6E70529A6D15879AA
:1036180019798842987906D950409871481C1871D0
:103628000B441A729AE790420CBF0622002293E7D5
:103638002B783D495B0791D42328DAF8003013D161
:103648000090012038702F480391036033480363CA
:1036580036480BF031FA30480BF02EFA0399009AED
:103668000B7843F002030B70314B1B681B789342B5
:1036780001BF304B304A1A60304B04BF304ADA6021
:103688006CE7DAF8002092F849304A2B00F06D8593
:1036980000F28580332B00F0718421D8292B00F0AB
:1036A800F68309D8252B00F0CE83272B00F0D18391
:1036B800232B40F0928569E22D2B00F0F98307D87F
:1036C8002B2B40F08A850BF01FF9607100F04DBD7F
:1036D8002F2B00F0BF84312B00F0D18400F07DBD8A
:1036E8003E2B00F03D8146D8372B00F07A842DD848
:1036F800352B00F0868200F070BD00BF702A0020D4
:10370800952A0020A02500207C1200204C120020C1
:10371800804D0108086501080D650108480E002064
:10372800A81C00209C250020942A00203D65010843
:1037380028250020FC9F0020EFBEADDE00ED00E054
:103748000400FA05B04B010898250020392B00F039
:103758008D833C2B40F04185DFF81894D9F800A000
:103768000BF0D2F88AF80000D9F80030187808F081
:103778001DFE00F0FABC432B00F0118405D8412B44
:1037880040F02B854FF00009FDE3442B00F0AC849A
:10379800482B40F0228509F09BFC00F0E6BCD02BBA
:1037A80000F02F835FD8CA2B00F0E38016D84E2B89
:1037B80000F0B683C82B00F0A2804C2B40F00D859A
:1037C8000BF0A2F884F8D6010BF09EF884F8D70124
:1037D8000BF0A4F8A4F8D80100F0C7BCCD2B00F07A
:1037E8001B8304D8CC2B00F0348200F0F6BCCE2B1F
:1037F80000F01B83CF2B40F0F0840BF08FF86FF4B0
:10380800AF6E00EB0E039BB2C62B98BFA4F89601CF
:103818000BF084F8A4F840010BF080F8A4F84201FA
:103828000BF07CF8A4F844010BF078F8A4F8D80160
:103838000BF06AF80BF068F80BF066F80BF064F818
:1038480084F885010BF060F884F892010BF05CF8BD
:10385800C84BD3F800900BF061F800EB80004000F3
:10386800A9F8620002E3D82B00F015810FD8D32BFA
:103878003FD003D8D22B29D000F0AFBCD42B00F016
:103888004782D62B40F0A9844FF0000935E2F22B8D
:1038980000F08C8212D8EF2B40F09F84DFF8D4928E
:1038A800D9F800A00BF03AF8AAF86600D9F8009009
:1038B8000BF034F8A9F8640000F057BCF32B00F0C3
:1038C8001884FA2B00F0BB8200F087BC2B7803F039
:1038D800040303F0FF09002B40F047840BF014F8B1
:1038E800022884F8A80740F29282A34B83F8A8978D
:1038F8008DE20BF013F8A14B988600F036BC92F8D5
:1039080005904FEA5909B9F1120F03D90AF086FE5A
:1039180000F02BBC4FF0000ACA4507D20AF0FEFFA0
:1039280007AB23F81A000AF1010AF5E74A46002313
:103938004B4507DA07A931F81300914921F813001C
:103948000133F5E7122A05D08D4B002123F8121018
:103958000132F7E7894B012283F8362000F005BCD5
:103968000AF0D2FF84F8E0010AF0CEFF84F8DF0104
:10397800FBE3804B1A681278022A824699466FD177
:10398800D9F800B00AF0C0FF07EE900AF8EE677A9F
:10399800B2EE048AC7EE887A0BEB8A0BCBED087A75
:1039A800D9F800B00AF0B0FF07EE900A9FED757ADB
:1039B800F8EE677A0BEB8A0BC7EE877ACBED0B7ABA
:1039C800D9F800B00AF0A0FF07EE900A9FED6E7AD2
:1039D800F8EE677A0BEB8A0BC7EE877A0AF1010AD1
:1039E800BAF1030FCBED0E7ACAD1BAF1070FD9F8A5
:1039F80000B01CD10AF088FF07EE900AF8EE677A4B
:103A0800C7EE887ACBED117AD9F800B00AF07CFFBE
:103A180007EE900AF8EE677AC7EE887ACBED127A4D
:103A2800D9F800B00AF070FF8BF84C0012E00AF0E9
:103A38006BFFD3448BF80100D9F800B00AF064FF9B
:103A4800D3448BF80B00D9F800B00AF05DFFD344DB
:103A58008BF815000AF1010ABAF10A0FC5D184E3FF
:103A6800D9F800B00AF050FFD3448BF80100D9F818
:103A780000B00AF049FFD3448BF80B00D9F800B026
:103A88000AF042FFD3440AF1010ABAF10A0F8BF88F
:103A98001500E5D169E38246DFF8D8909FED3A8AB0
:103AA800D9F800B00AF03AFF07EE900AF8EE677A04
:103AB8000BEB8A0BC7EE887ACBED087AD9F800B001
:103AC8000AF02CFF07EE900AF8EE677A0BEB8A0BE8
:103AD800C7EE887ACBED0B7AD9F800B00AF01EFF52
:103AE80007EE900AF8EE677A0BEB8A0BC7EE887A36
:103AF8000AF1010ABAF1030FCBED0E7ACCD1BAF173
:103B0800070FD9F800B01CD10AF008FF07EE900A99
:103B1800F8EE677AC7EE887ACBED117AD9F800B05B
:103B28000AF0FCFE07EE900AF8EE677AC7EE887A8C
:103B3800CBED127AD9F800B00AF0F0FE8BF84C0001
:103B480012E00AF0EBFED3448BF80100D9F800B07C
:103B58000AF0E4FED3448BF80B00D9F800B00AF061
:103B6800DDFED3448BF815000AF1010ABAF10A0FF9
:103B7800C5D1FAE2D80E0020401D0020480E0020D2
:103B8800A82900200000C84200007A440AF0BCFEC0
:103B9800132883463FF6BAAEDFF870A3DAF8009030
:103BA8000AF0B2FE0023D44A0C2101FB0322117A49
:103BB800814222D10FFA8BFB09EB8B09137889F824
:103BC80085300AF0A1FE89F886000AF09DFE89F882
:103BD80087000AF099FEC94BC94A1A6089F888001B
:103BE800C84BDAF800001860002185300BF09EF908
:103BF800C54B80F001001870B7E201331C2BD2D1FD
:103C080084E60AF081FE0B2882463FF67FAEBF4B62
:103C1800D3F800900AF078FE03283FF677AE062323
:103C280003FB0A9989F8DA000AF06EFE89F8D500D4
:103C38000AF06AFE89F8D6000AF066FE89F8D7000D
:103C48000AF062FE89F8D8000AF05EFE89F8D90009
:103C58008BE25379092B7FF659AE019BD3F800907C
:103C68000AF052FE019B89F80000D3F800900AF090
:103C78004BFE89F801000AF047FE019B64281B6887
:103C8800A8BF642018710AF03FFE019B64281B68D6
:103C9800A8BF642058710AF037FE019BFF281B68F3
:103CA800A8BFFF2098710AF02FFE019B6428D3F863
:103CB800009028BF642089F807000AF025FE019BC0
:103CC80089F80200D3F800900AF01EFE019B89F8DB
:103CD8000300D3F800900AF021FED8F80030A9F8C4
:103CE8000A005B790A2B40F24082894BD3F8009096
:103CF8000AF00AFE89F8080037E20AF00FFE854B41
:103D080023F8190009F10109B9F1080FF5D12CE2DE
:103D180053790F2B7FF4FAAD0AF0F6FD0728814698
:103D28003FF6F4AD029BD3F800A00AF0F7FD0E238E
:103D380003FB09F9CA44029BAAF82501D3F800A09D
:103D48000AF0ECFDCA44029BAAF82701D3F800A0A8
:103D58000AF0E4FDCA44029BAAF82901D3F800A09E
:103D68000AF0D2FDCA44029B8AF82B01D3F800A0BE
:103D78000AF0CAFDCA44029B8AF82C01D3F800A0B5
:103D88000AF0C2FDCA44029B8AF82D01D3F800A0AC
:103D98000AF0BAFDCA44029B8AF82E01D3F800A0A3
:103DA8000AF0C6FDD144C9F82F01DEE10AF0ACFDE6
:103DB8000F2881463FF6AAADC9EBC9090AF0A4FD50
:103DC80004EB090303F1D00983F8D0000AF09CFD45
:103DD80089F801000AF098FD89F802000AF094FDBC
:103DE80089F803000AF090FD89F804000AF08CFDB8
:103DF80089F805000AF088FD89F806000BF076FBC3
:103E0800B3E12B78580700F1B08109F033FD05F0D4
:103E18002FFB05F0EBFBA8E12B78590700F1A581F2
:103E28003D4B4FF4C8721A809FE12B785A0700F176
:103E38009C813A4A137843F00403137095E12B7878
:103E48005B07E4D5C9E1A0600AF072FD05F0DEFA6F
:103E58008BE10AF063FDA4F858010AF05FFDA4F8AD
:103E68005A010AF05BFDA4F85C017EE10AF04CFD02
:103E780084F87A010AF048FD84F87E010AF044FDCE
:103E880084F87D010AF040FD84F87F016DE10AF0B5
:103E980045FDA4F880010AF041FDA4F882010AF06A
:103EA80033FD84F884010AF039FDA4F886015CE149
:103EB8000AF02AFD84F890010AF030FDA4F89A016E
:103EC8000AF02CFDA4F896010AF028FDA4F8980140
:103ED8000AF01AFDDAF8003084F891015B79082BB2
:103EE80040F243810AF01AFDA4F89C010AF016FD7D
:103EF800A4F89E0139E100BF644501083C0E00208A
:103F0800801E0020400E002005000020D80E002052
:103F1800040F00207E2500202E1A0020A81A002059
:103F280092F805900323B9FBF3F9B9F1120F3FF6A4
:103F3800EDACDFF8C0A34FF0000BCB4580F0158146
:103F48000AF0E2FC8AF8A0010AF0E8FC40F2ED234E
:103F5800984205DD40F6CA039842A8BF184601E01A
:103F680040F2EE20A0F2EE2019230BF1010B90FB9A
:103F7800F3F00AF1020A8AF89F01DEE70AF0C4FCAE
:103F880084F89201F1E00AF0BFFC04EB090309F19F
:103F98000109B9F1080F83F88801F4D1E5E00AF0C6
:103FA800B3FCC4F808B060710AF0C2FC05F02EFA40
:103FB8000AF0AAFC84F890010AF0B0FCA4F85801B1
:103FC8000AF0ACFCA4F85A010AF0A8FCA4F85C01B9
:103FD8000AF0A4FCA4F880010AF0A0FCA4F882016D
:103FE800C3E053794FF0070AB3FBFAF2C2EBC202FF
:103FF8009A1A12F0FF0F7FF489ACB3FBFAFA0AF1B0
:10400800FF3A5FFA8AFABAF1FF0F00F0AE800AF0C1
:104018007BFC5FFA80FB4FFA8BF003F009F88146CE
:1040280000283FF473AC80F800B00AF077FCA9F8D8
:1040380002000AF069FC89F804000AF065FC89F8B6
:1040480005000AF061FC89F807000AF05DFC89F8B0
:104058000600D4E7DFF89C9209F1400A0AF05EFCFA
:10406800A9F8A0020AF050FC89F8A2020AF04CFC58
:1040780009F1040989F89F02D145EFD175E00AF0EA
:1040880043FC1F2881463FF641ACD8F800305B79E5
:10409800082B7FF43BAC0AF041FC09F1880904EBDA
:1040A800890A00F03F00AAF802000AF037FCBAF8C3
:1040B8000230800100F4FE501843AAF802000AF00A
:1040C80023FC000104F829000AF01EFC14F829302A
:1040D80000F00F00184304F829000AF015FC8AF8CC
:1040E800010004F049FC40E0724B012283F83720BC
:1040F8003BE00AF009FCFF28824622D100238DF814
:104108001B309DF81B30072B14D89DF81B006A4AFA
:104118009DF81B3052F8300002EBC30301215B68A5
:10412800994089B2042202F0FDFD9DF81B3001334D
:10413800DBB2E4E74FF090400121002202F0F2FDEB
:1041480013E007283FF6E2AB00200AF02DFC0AF046
:1041580007FCD9F800000BF015F818B932200AF05E
:1041680057FFF6E7504602F0EBFD00200AF01CFC72
:10417800FFF704BA514B98590BF004F818B93220DC
:104188000AF046FFF6E70BF071F905F047F94C4BDA
:104198004C4ADA60FFF7FFB90C2824D00A2826D148
:1041A800494D4A480AF088FC284623210FF08DF92A
:1041B80008B1401B20602368E3B94348236000210D
:1041C80030220FF04CF93B78002B46D1404B9B68CE
:1041D800002B69D03F48984766E00AF01FFAFFF7BE
:1041E800CDB90C2847D13C480AF066FC35E00D28CB
:1041F80035D1D5E75A1EA95C202901D11346DBE742
:10420800314A23600021D154344B354DD3F800A0F6
:10421800D5F800B0DFF8B09058460FF064F90646BC
:104228003246484659460FF067F92E4A28B919F818
:10423800063053445B78590703D010359542E7D3CD
:1042480006E0954204D2701CEB684844984702E0A7
:1042580025480AF031FC0023AFE7244807E07F280F
:104268000DD1013B184A224823600021D1540AF09D
:1042780023FCFFF7EEB87F2804D1FFF7EAB82F2B0D
:104288003FF6E7A8A0F12002D2B25E2A3FF6E1A8E5
:1042980013B920283FF4DDA85A1C22600A4AD054DA
:1042A8000AF002FCFFF7D5B811B0BDEC028BBDE8EF
:1042B800F08F00BF480E002030680108A81C0020BD
:1042C80000ED00E00400FA054C120020FC73010820
:1042D800B0190020800E0020126501080C01002092
:1042E800B04B0108804D01081D6501080D650108E6
:1042F80039650108401D00202DE9F0472DED028B9E
:104308004728A0B0044600F0528600F2CE802E283E
:1043180000F0018667D8222800F0AC8423D803284F
:1043280000F03A8214D8012800F02B82022840F0CD
:104338008A8604200AF038FB43200AF002FB4C204E
:104348000AF0FFFA46200AF0FCFA4C2000F0B5BD4E
:10435800042800F02B82052840F075861A200AF000
:1043680023FB002432E2282800F06E8515D8242883
:1043780000F05585262840F06686C34C06200AF0D2
:1043880013FBB4F858010AF012FBB4F85A010AF00A
:104398000EFBB4F85C0100F0A1BD2A2800F0678587
:1043A8002C2840F05086B84C0C200AF0FDFA94F8FE
:1043B80090010AF0C6FAB4F89A010AF0F8FAB4F8CB
:1043C80096010AF0F4FAB4F898010AF0F0FA94F8B1
:1043D80091010AF0B6FAB4F89C010AF0E8FAB4F8C8
:1043E8009E0100F07BBD3A2800F0DB821DD83428FE
:1043F80000F070840DD8302800F0A385322840F0F2
:10440800228601200AF0D0FA9F4B93F8920100F01F
:1044180054BD362800F06585382840F014860420FD
:104428000AF0C2FA984C00F000BD402800F0488518
:1044380011D83B2800F017843D2840F00486924CA0
:1044480002200AF0B1FA94F8E0010AF07AFA94F836
:10445800DF0100F032BD452800F0E28500F29685C4
:10446800422840F0F085884C10200AF09DFA6079C7
:104478000AF067FAA0680AF0A3FA94F890010AF023
:1044880060FAB4F858010AF092FAB4F85A010AF03E
:104498008EFAB4F85C010AF08AFAB4F880010AF0DE
:1044A80086FAB4F8820100F019BD6F2800F0CA82BC
:1044B80000F2F280662800F0C58100F2BE804D2827
:1044C80000F0DB8415D8492800F0B5824B2840F06D
:1044D800BA856D4C04200AF067FA94F8D6010AF000
:1044E80030FA94F8D7010AF02CFAB4F8D80100F0A1
:1044F800F5BC642800F08381652840F0A485634CEE
:104508000B200AF051FA20880AF051FA6268604BD1
:104518009A420CBF2089608980B20AF048FAE368A1
:10452800C3F3C000C3F38002800040EA4200C3F333
:1045380040021043C3F3401240EAC20003F01003E4
:1045480018430AF034FA228A6369247E02F00801CB
:1045580003F4475949EA010903F4804149EA01098A
:1045680003F4004149EA010903F4803149EA0109E9
:1045780003F4003149EA010903F4802149EA0109F9
:1045880003F4002149EA010903F4801149EA010909
:1045980003F0007349EA0303DFF8F89099F80090F4
:1045A80012F0010FC9F3800914BF4FF002084FF051
:1045B800000843EA090312F0020F43EA080314BF94
:1045C8004FF0040C4FF0000C12F0040F43EA0C0CEF
:1045D80014BF4FF0100E4FF0000E12F0400F14BF32
:1045E800202700274CEA0E0E12F0100F14BF4FF4CC
:1045F800007600264EEA070712F0200F14BF4FF48A
:10460800806500253E4312F4807F14BF4FF400609C
:104618000020354312F4007F14BF4FF4001100212D
:10462800284312F4806F41EA000114BF4FF0806301
:104638000023002019430346F1E0692800F0978120
:104648000AD8672800F01E81682840F0FC841020F2
:104658000AF0AAF9002482E16D2800F09B8100F29B
:10466800BD816C2840F0EF84084C06200AF09CF9C4
:10467800B4F86C000AF09BF9B4F86E000AF097F9E8
:10468800B4F8700000F02ABC401D0020880E0020FD
:1046980000540040942A0020772800F079834BD8F2
:1046A800732800F095833CD8702800F0F5817228B3
:1046B80040F0C984BD4C16200AF076F9B4F896018A
:1046C8000AF075F9B4F840010AF071F9B4F842013A
:1046D8000AF06DF9B4F844010AF069F9B4F8D801A0
:1046E8000AF065F900200AF02CF900200AF029F9EF
:1046F80000200AF026F994F885010AF022F994F8C6
:1047080092010AF01EF900200AF01BF9A84B1B6D54
:104718000A20B3F9623093FBF0F080B20AF047F94F
:1047280083E3742800F0FB82752840F08C842F20E6
:104738000AF03AF99F4C8EE2A02800F062830AD86A
:10474800782800F0AB807B2840F07D843C200AF07C
:104758002BF9002429E2F12800F0DB80FE2800F084
:104768004283F02840F06F84914C04200AF01CF931
:10477800236DB3F866000AF01AF9236DB3F86400E4
:10478800ACE303200AF010F900200AF0DAF820461A
:104798000AF0D7F80D2090E30AF006F901200AF094
:1047A800D0F80B200AF0CDF8002086E306200AF0A6
:1047B800FBF84D200AF0C5F84F200AF0C2F8542043
:1047C8000AF0BFF84F200AF0BCF818E37A4B185DDE
:1047D80001340AF0B6F80B2CF8D10024774B185D99
:1047E80001340AF0AEF8082CF8D10024744B185D97
:1047F80001340AF0A6F8072CF8D100F022BC0720F3
:104808000AF0D2F8E7200AF09CF8684B58790AF0C9
:1048180098F800200AF095F8042000F010BCA34294
:104828000AD2684A9D5C012202FA05F50D421CBFB6
:104838009A4010430133F2E70AF0C2F85B4B93F851
:10484800A8073AE312200AF0AFF85F4B1B88B3F5CC
:10485800806F8CBF082601260025554C04F13403CF
:1048680033F9150090FBF6F0013580B20AF09FF895
:10487800032DF2D1608F0AF09AF8A08F0AF097F80A
:10488800E08FB4E210200AF08FF800244F4B185D37
:1048980001340AF056F8102CF8D1D2E370200AF04F
:1048A80083F80026424D0E242B6D744323440136B1
:1048B800B3F825010AF07BF82B6D2344B3F82701E0
:1048C8000AF075F82B6D2344B3F829010AF06FF844
:1048D8002B6D234493F82B010AF033F82B6D2344F6
:1048E80093F82C010AF02DF82B6D234493F82D0131
:1048F8000AF027F82B6D234493F82E010AF021F8CB
:104908002B6D1C44D4F82F010AF05AF8082EC9D18F
:1049180097E37020254C0AF047F804F1700594F8E5
:10492800D0000AF00EF894F8D1000AF00AF894F8CA
:10493800D2000AF006F894F8D3000AF002F894F8C6
:10494800D40009F0FEFF94F8D50009F0FAFF073407
:1049580094F8CF0009F0F5FFAC42E0D171E31C4BAD
:10496800185D013409F0EDFF102CF8D169E3194DF9
:104978002878400000F0FE000AF016F800242B7892
:104988009C4280F05E83144B33F814000AF00FF851
:104998000134F4E706200AF007F800200AF010F8BE
:1049A8002DE204200AF000F848E300BF401D002073
:1049B800880E002033450108006301080C630108D4
:1049C800E1620108A10E002008000020C80E0020A6
:1049D800DC0E002020250020821C0020072009F082
:1049E800E3FFB54BB54C1888FF28A8BFFF20C0B21D
:1049F80009F0A7FFB24B18684FF6FF75A842A8BF89
:104A0800284620EAE07080B209F0D1FFB4F87200BD
:104A180009F0CDFFAB4B606F93F885313BB10A23AA
:104A28005843A842A8BF284620EAE07001E000F3F6
:104A38000F0080B252E2022009F0B6FF9F4BB3F894
:104A480078004BE29D4C0B2009F0AEFFE36F18781D
:104A580009F077FFE36F587809F073FF00262546C1
:104A6800EB6F964C33440136187909F06AFF032E30
:104A7800F6D1E36FD87909F064FFE36F987809F00D
:104A880060FFE36FD87809F05CFFE36F588909F09D
:104A98008EFFE36F187A10E2884C1E2009F084FF1D
:104AA800236D1B78022B4FF000056BD1236D03EBB0
:104AB800850393ED080AB2EE048A20EE080A0EF088
:104AC800DDFE80F30800C0B209F03BFF236DDFED87
:104AD8007E7A03EB850393ED0B0A20EE270A0EF08E
:104AE800CDFE80F30800C0B209F02BFF236DDFED87
:104AF800777A03EB850393ED0E0A20EE270A0EF072
:104B0800BDFE80F30800C0B2013509F01AFF032D7D
:104B1800CCD1072D236D23D193ED110A20EE080A7D
:104B28000EF0ACFE80F30800C0B209F00AFF236D56
:104B380093ED120A20EE080A0EF0A0FE80F308009A
:104B4800C0B209F0FEFE236D93F84C3000EE103A27
:104B5800B8EE400A0EF092FE80F30800C0B20BE0F7
:104B68002B44587809F0EDFE236D2B44D87A09F0D0
:104B7800E8FE236D2B44587D013509F0E2FE0A2D2D
:104B8800C7D15EE2236D2B44587809F0DAFE236D15
:104B98002B44D87A09F0D5FE236D2B440135587D76
:104BA80009F0CFFE0A2DEDD14BE2444D9FED478A27
:104BB8002B6D03EB840393ED080A20EE080A0EF030
:104BC8005DFE80B209F0F3FE2B6D03EB840393EDD9
:104BD8000B0A20EE080A0EF051FE80B209F0E7FE3B
:104BE8002B6D03EB840393ED0E0A20EE080A0EF0FA
:104BF80045FE013480B209F0DAFE032CD5D1072C2A
:104C08002B6D16D193ED110A20EE080A0EF036FE30
:104C180080B209F0CCFE2B6D93ED120A20EE080A43
:104C28000EF02CFE80B209F0C2FE2B6D93F84C00FA
:104C38000BE02344587809F0BAFE2B6D2344D87A48
:104C480009F0B5FE2B6D2344587D013409F0AFFE01
:104C58000A2CD4D1F5E114F8010F002800F0F181F5
:104C680009F06FFEF7E7012009F09EFE134B1B6D5C
:104C7800187822E1502009F097FE00250F4B1C6D93
:104C8800134B04EB85040C2194F8852001FB0233B7
:104C9800013593F8380009F054FE94F8860009F0BD
:104CA80050FE94F8870009F04CFE94F8880009F04B
:104CB80048FE142DE2D1C4E1D8110020880E00204E
:104CC80030110020401D00200000C84200007A4436
:104CD80034450108482009F067FE0025C54B1C6DC6
:104CE800062303FB0544013594F8DA0009F029FE90
:104CF80094F8D50009F025FE94F8D60009F021FEB5
:104D080094F8D70009F01DFE94F8D80009F019FEB0
:104D180094F8D90009F015FE0C2DDFD191E14FF080
:104D2800000801260027B34B1A7E974227DA193369
:104D38000024FA5CB04D0C2305F130016343595C43
:104D4800914207D12B44586B0EF0CDFB82462EB909
:104D5800B14605E001341C2CECD10EE080440CE097
:104D6800D1450ADA0C2303FB04535B6B13F80900E3
:104D780009F0E7FD09F10109F2E70137D3E7002E51
:104D880000F05F815FFA88F009F00EFE0026C9E79F
:104D9800984D287E09F008FE00242B7E9C4280F066
:104DA8005081964BE65C002193480C2200F13007B5
:104DB80002FB01F3DA5DB24205D1034493F83800EF
:104DC80009F0BFFD02E001311C29EDD10134E4E70F
:104DD800082009F0E9FD0124E0B2013409F0B1FD31
:104DE800092CF9D12DE1082009F0DEFD002009F099
:104DF800DEFD002009F0DBFD002009F0D8FD0020D1
:104E08006CE00C2009F0D0FD7D4B186809F0D8FD46
:104E18007C4B186809F0D4FD7B4B18680FE104201F
:104E280009F0C2FD794B986809E194F87A0109F014
:104E380088FD94F87E0109F084FD94F87D0109F05D
:104E480080FD94F87F0138E0704C072009F0ACFD34
:104E5800B4F8800109F0ABFDB4F8820109F0A7FDB0
:104E680094F8840109F06DFDB4F8860136E001205C
:104E780009F09AFD654B58791FE0654C654D20781F
:104E880000EB4000C0B209F08FFD002623789E4257
:104E980005F1020580F0D58015F8020C09F051FDE6
:104EA80015F8010C00EB800000EB800000F2EE200A
:104EB80080B209F07CFD0136E8E709F042FDC0E068
:104EC800082009F071FD0024504B2344013493F865
:104ED800880109F036FD082CF6D1B2E009F067FD2B
:104EE800AFE0444B494C93F88000C0EBC000C0B21F
:104EF80009F05AFD04F1200594F8F0010023464A10
:104F0800D25C904200F0A1800C33302BF7D10834EA
:104F1800AC42F1D195E040203C4C09F045FD04F14C
:104F28004005B4F8A00209F042FD94F8A20209F085
:104F380008FD043494F89F0209F003FDAC42F0D157
:104F48007FE0E020314C09F02FFD04F18005B4F832
:104F5800220200F03F0009F02AFDB4F82202C0F353
:104F6800861009F024FD94F82002000909F0E9FCF4
:104F780094F8200200F00F0009F0E3FC043494F8E0
:104F88001D0209F0DEFCAC42E1D15AE0234C0D20B1
:104F980009F00AFD07F09EFF09F0D3FCA08809F08C
:104FA8000FFD206909F00CFD07F084FF47E009F0C8
:104FB800BFFC0546842009F0F7FC284609F000FDEF
:104FC800164B1C6905F18003A3428CBF641B802427
:104FD80003F026FE28462246694608F0A1F8002478
:104FE8000546AC422DDA1DF8040009F0AAFC01348C
:104FF800F7E700BF880E002034450108A10E002005
:10500800ACF7FF1FB0F7FF1FB4F7FF1F401D0020CC
:1050180020250020E01E00202C250020080000206C
:10502800132009F0C1FC0024164B185D013409F067
:1050380088FC0B2CF8D1002009F0C2FC002009F0F4
:10504800BFFC012018E0002016E009F07AFCB4F853
:10505800F20109F0ACFC94F8F40109F072FC94F840
:10506800F50109F06EFC94F8F70109F06AFC94F870
:10507800F60109F066FC4AE720B0BDEC028BBDE8FA
:10508800F08700BF0063010810F80A3C0133DBB267
:105098000A2B84BF10F8131C044A00F80A3C82BF8C
:1050A800002322F8113000F80A3C7047CC29002070
:1050B800334A136C90681944081A40F68C239842B6
:1050C80070B513469160D06051603BD9127893F95E
:1050D80045108A4210460BD1111F082908D893F8A9
:1050E8004610182901D8013103E083F8442002E072
:1050F800002183F8461093F944402149A24219D16E
:1051080091F84740B4B10C310024944206DA1D4DA1
:1051180051F8046F25F814600134F6E70C2805D01F
:105128001849002421F810400130F7E716480178A3
:105138000131017083F84520002201211A7083F89B
:10514800471070BD92F84710C9B1A0F2EF2440F2A1
:10515800DA518C4208D811780B2905D80B1D01317A
:10516800117042F8230070BD002283F84720074BD6
:1051780003F13002002143F8041F9342FAD170BDB5
:1051880080080020CC2900207D0100208C08002008
:10519800024A136C013319441164704780080020D7
:1051A800024B53F820301B6819607047F425002023
:1051B800064B53F820301A681B89A1F57A715943B8
:1051C8004FF47A7391FBF3F111607047F4250020D6
:1051D800F0B5046D8668236823F0010323608379A2
:1051E800054613F0020F40790CBF4FF0000E4FF444
:1051F800005E13F0040F14BF4FF48067002710F00F
:10520800010F14BF042100218307206820F001004A
:105218002060626822F440524EEA0202626022680C
:1052280022F4B05323F00C0348BF41F008013B437C
:105238000B432360A36895B023F44073A3606846CA
:1052480000F068FF284B9C4201D10C9B0EE0274BD5
:105258009C4201D10D9B09E0254B9C4201D10E9B3C
:1052680004E0244B9C420CBF0F9B109B2268A8793A
:10527800170448BF5B00B3FBF6F206FB1233B3EB2F
:10528800560F236828BF01321E0441BF4FF6F07342
:10529800C2F34201134041EA03026B7992B213F060
:1052A800020FA28100F0010114BF4FF40032002266
:1052B800DC0748BF42F480322B6D11B159680A43AC
:1052C80002E0596821EA02025A609A6801074CBF55
:1052D80042F0080222F008029A601A6842F00102BD
:1052E8001A6015B0F0BD00BF00380140004400400E
:1052F80000480040004C00403D4B1B78012B30B566
:1053080014BF00240324B1B9036A23F00103036224
:105318008169036A21F0F30123F00A0341F00101D6
:1053280042F001021A4341EA041181610262836971
:1053380023F00C031BE004291DD1016A4FF6EF731B
:105348000B4003628169056A120121F473414FF62B
:105358005F7342F0100241F480712B4092B2134304
:1053680041EA043181610362836923F44063836104
:105378008369836130BD0829016A1AD14FF6FF633A
:105388000B400362C169036A9BB289B223F42063AC
:1053980043F4807321F0F30143EA022241F0010152
:1053A80092B241EA0411C1610262C2694FF6F37315
:1053B80019E04EF6FF730B400362C369056A40F6B5
:1053C800FF41194045F6FF732B4043F4805343EAED
:1053D800023241F4807192B241EA0431C161026241
:1053E800C2694FF2FF331340C361C369C36130BD63
:1053F8007C08002038B510F80E2C50F8043C044600
:1054080052B9012200F80E2C20F80C1C997A186861
:105418000222BDE838406FE730F80C2C20F80A1C4F
:10542800891A89B220F8081C074A10F80F0C0025C1
:1054380022F8101004F80E5C1868997A2A46FFF7CB
:105448005BFF04F8065C38BDCC290020044B53F8F8
:1054580020301BB107289CBF1B681960704700BF2C
:10546800A8090020084A13689B050BD5074B0021A3
:105478001970074908684FF6FE7303400B604FF434
:1054880000735360704700BF00000240922A00205A
:10549800300002402DE9F047664D2B6866490A78CE
:1054A800581C02F0FF068E460AB10346F6E72B6049
:1054B800687BAB6895F80C80AA7B374639B22029FF
:1054C80000F09B80DFF880C10CEB81033CF82110D1
:1054D800DC789B78C3F1FF039BB2002B65D0C3F146
:1054E800FF0363434FF03C0C1B12B1FBFCF9B9F10D
:1054F800050F5DD8DFE809F0030B1A293A4AE01ACC
:10550800DAB24143B1FBFCF01044C0B251E0B1FB48
:10551800FCF00CFB101189B2DAB2C1F13C01E31ABC
:105528004B432046B3FBFCFC94442CE0B1FBFCF05D
:105538000CFB10115FFA83F8E21A89B24A43B2FBF6
:10554800FCF24244D2B2204632E0B1FBFCF90CFB3B
:10555800191189B25FFA83F8E01AC1F13C01484396
:10556800B0FBFCF04044C0B2224621E0B1FBFCF89D
:105578000CFB1811D8B289B2E31A01FB03F2B2FB93
:10558800FCFC224684445FFA8CF412E0B1FBFCF880
:105598000CFB181189B2D8B2C1F13C01E31A4B4394
:1055A800B3FBFCF20244D2B203E02246204600E0FC
:1055B80044464FEA042C4CEA004C4CEA020C1723F0
:1055C80006F117014FF0010808FA03F8C91A18EA9A
:1055D8000C0F89B2DFF8748014BF4FF011094FF037
:1055E800090913F1FF3308F80190E9D21836013799
:1055F800B6B2BFB2114BA04660E7AA73AB60104ABF
:10560800E98001238EF800300E4985F80C8040F2BD
:105618002A336873AE80536000234B620B889BB2B9
:1056280043F001030B80136843F001031360BDE8E6
:10563800F08700BF0C0F0020922A0020180F0020CE
:105648003000024000440140B4070020F009002067
:1056580073B506460D46002401232A88A340134249
:105668001AD0AA78009302F003038DF80430EB787F
:10567800022B03D0032B0CBF032301238DF8053025
:105688003046C2F301136946C2F381028DF8063031
:105698008DF8072000F0ACFE0134102CDCD102B0EC
:1056A80070BD2DE9F04F734EF57B07460C4687B069
:1056B80011469A4600686B1C914622464FF0020B31
:1056C800F37307F0D5FF3B897868ADF8043001A97A
:1056D8008DF806B08DF807B0FFF7BAFF0023ADF8D4
:1056E8000A30ADF81230ADF8163070230193BA7A4B
:1056F8003C68CDF80CA0012306F110082D01ADF887
:1057080008304FF48073A844ADF810B0ADF81430E9
:105718000C2A7ED8DFE802F0077D7D7D0F7D7D7D38
:10572800387D7D7D5E00204601A900F0B5FCA369A7
:1057380043F0080326E0236A4F4823F0100323624E
:10574800236A6168A26922F0807222F4E6428442E8
:1057580042F4E04206D000F50060844202D043F0F3
:10576800300307E023F0E00321F4406143F0300305
:1057780041F480616160A261C4F838A02362A36922
:1057880043F40063A36144E0236A3B4823F4807335
:105798002362226A6168E369844223F0730343F059
:1057A800700306D000F50060844202D042F44072D3
:1057B80007E022F4606221F4405142F4407241F45F
:1057C80080516160E361C4F83CA02262E36943F060
:1057D80008031DE0236A284823F480532362226AC1
:1057E8006168E369844223F4E64343F4E04342F406
:1057F800405203D000F50060844201D141F4804159
:105808006160E361C4F840A02262E36943F4006385
:10581800E3613A7B3B681AB15A6C42F400425A641D
:105828001A8892B242F001021A80BA7A0C2A18D861
:10583800DFE802F0071717170B1717170F171717B7
:105848001300721903F134010AE0721903F13801E7
:1058580006E0721903F13C0102E0721903F14001FC
:10586800116135444046A5F818906B6107B0BDE852
:10587800F08F00BF0C0F0020002C0140054B984210
:105888000CBF054A054A138801339BB213800020D8
:10589800704700BF00540040900E0020920E002078
:1058A800400070B5C5B22D482D4B00684FF4204418
:1058B8001C608669360404D52646013C002EF8D1C2
:1058C80012E04668274C344044F0807444F4903425
:1058D8002C4344604FF420441C608669B60726D4E4
:1058E8002646013C002EF8D11C601AE02146013CF6
:1058F8000029F9D081690E06F8D544681949214074
:1059080041F0007141F48031294341604FF4204156
:1059180019608469A4070FD40C460139002CF8D10A
:105928001960FFF7ABFF003018BF012070BD4FF4BE
:10593800204481621C60DDE782624FF420421A60D5
:105948008169890605D41146013A0029F8D11A60FF
:10595800E7E71A602023C361012070BD8C0E002088
:10596800F41A0020009800FC10B5214A18B91368F1
:1059780002221A8210BD1F48146800230380217870
:1059880011F07F0102460DD1637A990644BF0221C6
:10599800017013F0400F037814BF43F0010323F0A4
:1059A800010315E0012921D002291ED1637913F0E2
:1059B800800F03F00F034FEA830303F1804303F5DD
:1059C800B8431B6806D003F03003102B07D101231E
:1059D800137004E003F44053B3F5805FF6E7064B19
:1059E8001B681B699847034810BD184610BD00BFC7
:1059F8007C1C002008100020DC1A002010B5064C82
:105A080018B9236801221A8210BD044B1B689B68D1
:105A1800984720680C3010BD7C1C0020DC1A002040
:105A280010B5064C18B9236801221A8210BD044B20
:105A38001B681B68984720680A3010BD7C1C002032
:105A4800DC1A002003788B4283BF034B03EB410130
:105A580048880020704700BF0810002070B5002259
:105A68001346244914180C44A47E83EA042308240A
:105A780013F4004F4FEA430318BF83F4815304F132
:105A8800FF3418BF83F0010314F0FF049BB2EFD179
:105A98000132192AE5D100F1190200F11A050A4468
:105AA8000D44967EAA7E02EB062292B29A421FD13C
:105AB800104B93F83B50E2B2AA4216D2431C03EBB8
:105AC8004203DBB2CA1801330B44927E9B7E03EB80
:105AD80002239BB24FF4AF6253431B13064A03F5EC
:105AE800487322F814300134E5E7012381F83C308B
:105AF80070BD00BF081000200A10002003788B42F8
:105B08000BD9074B1A78074B89001944086C02B166
:105B1800400800F5777080B270470020704700BFDA
:105B2800242500200810002007299DBF034B03EB04
:105B38008101B1F870000020704700BF08100020F4
:105B4800034B03EB4101B1F89000C008704700BF58
:105B58000810002070B5334C054609F03DFAD4F81A
:105B6800B030C4F8B000C31AB3F5FA5FC4F8B43063
:105B780082BF002384F8B83084F8B93094F8B8307C
:105B88002BB9A12D02BF274A012182F8B91094F838
:105B9800B910244A29B1D118EDB201338D7682F8B3
:105BA800B83094F8B85094F8BA30AB4239D11D4B9C
:105BB80093F8BB30052B02D0062B03D02CE0002035
:105BC800FFF74CFFE37E1E2B26D100200246C1B210
:105BD8006B1E994219DA21448B7E0821DBB283EAD5
:105BE8000206F60744BF83F01803C3F3460301F126
:105BF800FF3154BF5B0843F0800311F0FF01C2F38B
:105C08004702ECD101301A46E1E723449B7E9A42D1
:105C180002D10320FFF722FF002384F8B93084F86B
:105C2800B83070BD0810002010B5044609F0D4F94A
:105C38000F4BD3F8BC20C3F8BC00821A41F288315C
:105C48008A42C3F8C02084BF002283F8C42093F896
:105C5800C420074913440F2AE4B218BF013283F85D
:105C6800C54012BF81F8C420012381F8D53010BD8A
:105C78000810002010B5044609F0AEF90F4BD3F810
:105C8800D820C3F8D800821A41F288318A42C3F872
:105C9800DC2084BF002283F8E02093F8E020074945
:105CA8001344142A18BF013283F8E14012BF81F867
:105CB800E020012381F8F63010BD00BF0810002055
:105CC8002DE9F843324F3D682A8A2E7AB2B9042E5C
:105CD80014D1304C30482378012B0BD12F4B196845
:105CE8002F4B89B20B445B0019681A60302303807C
:105CF800227048E010230380072644E0AC8AAB6991
:105D0800A24294BF04260226944228BF14461FFAD2
:105D180084F840469847214A13689BB203F1005320
:105D280003F540535B0004F1010E1B689BB203F1BD
:105D3800005303F540534FEA6E0E5B000021714596
:105D480000F1020009D010F8019C10F802CC4CEACE
:105D5800092C23F821C00131F1E71268104B92B2E7
:105D680013445B001A681C602B8AC8EB03032B8260
:105D78006B8A9844084BA5F8128030221A80094B88
:105D88004FF440521A803B681E72BDE8F88300BF8A
:105D98007C1C0020972A0020D61A0020505C004066
:105DA80002300020D41A00200E4B0F4A1B689BB209
:105DB80003EBC00002443E294FEA420209D94B09CD
:105DC800C80604BF03F1FF339BB29B0243F40043B0
:105DD80004E04B08C90748BF01339B0211681360F0
:105DE800704700BF505C00400630002010B5454B9E
:105DF8001A68107810F07F0004D1537A23F020033A
:105E0800537210BD02287AD15388002B78D11379A8
:105E1800002B75D1537923F08000840004F1804170
:105E280001F5B84113F0800F096814BF01F0300183
:105E380001F44051032862D8002960D0927A002AE0
:105E48005DD004F1804404F5B8441906226825D5CC
:105E580002F03002102A4CD103F07F039B0003F1BB
:105E6800804303F5B8431A68510641BF196840F6E4
:105E78000F720A4042F4004244BF42F0C0021A6066
:105E88001A6822F4E04222F0400292B282F0300214
:105E980042F4004242F080021A602AE002F44052C2
:105EA800B2F5805F25D128B9174B93F82C10FFF76E
:105EB8007BFF11E09B0003F1804303F5B8431A68A8
:105EC800520441BF196840F60F720A4042F440423A
:105ED80044BF42F080021A60236823F4804323F011
:105EE80070039BB283F4405343F4004343F08003B0
:105EF8002360064B1B685B699847002010BD022091
:105F080010BD00BF7C1C0020D0000020DC1A00203F
:105F180020F01F01012300F01F00024A83408B502C
:105F2800704700BF1404014000230360436083608E
:105F38008381036143618361C36103624362836256
:105F480070478A68036810B50C6A14430A691443D9
:105F58004A6914438A691443CA6914434A6A144350
:105F68008A6A23F4FF4323F0700322431343036038
:105F78008B8943600B6883604B68C36010BD0268FF
:105F88004FF6FE7313400360002303604360836091
:105F9800C360294B984201D1284A27E0284B9842F0
:105FA80001D1264A2AE0274B984201D1234A2DE005
:105FB800254B984201D1214A30E0244B984201D127
:105FC8001E4A33E0224B984204D11C4A536843F4DA
:105FD80070032EE01F4B984204D1184A536843F0CF
:105FE800706326E01C4B984204D11C4A536843F066
:105FF8000F031EE01A4B984204D1184A536843F025
:10600800F00316E0174B984204D1144A536843F43E
:1060180070630EE0144B984204D1104A536843F45D
:10602800704306E0114B984204D10C4A536843F47C
:1060380070235360704700BF080002400000024010
:106048001C00024030000240440002405800024058
:106058006C00024080000240080402400004024034
:106068001C04024030040240440402405804024028
:10607800084BDA68D10709D4DA68D20608D4DB6895
:1060880013F0040F14BF0320042070470120704749
:106098000220704700200240036A23F001030362D4
:1060A800036A70B5446882690D6822F4803222F070
:1060B800730215438A8923F0020313438A88134322
:1060C800134A90420FD002F5006290420BD002F5BD
:1060D8004062904207D002F58062904203D002F5F8
:1060E800806290420DD1CA89CE8823F008031343F9
:1060F8000A8A24F4407414434A8A23F0040333437D
:1061080014438A68446085614263036270BD00BFBE
:10611800002C0140994A536803F00C03042B2DE925
:10612800F04105D0082B06D095490160B3B916E0B7
:10613800934B036012E053685468C3F38343991C7C
:10614800E30349BFD36A8F4B8D4C03F00F0344BF61
:106158000133B4FBF3F34B43036000E000235168C1
:10616800894FC1F303117D5C0168EDB221FA05F492
:1061780044605668C6F30226BE5D24FA06FEC0F8DF
:1061880008E05668C6F3C226BE5DF6B2F440C460A5
:10619800D2F82C80C8F3041808F00F0C07EB4C0C4D
:1061A80018F0100FBCF810C01FFA8CFC07D0BCF117
:1061B800000F04D0B3FBFCFCC0F810C000E0016184
:1061C800D2F82CC0CCF3442C0CF00F0807EB48078E
:1061D8001CF0100F3F8ABFB204D01FB1B3FBF7F712
:1061E800476100E04161176BFF065ABF644F876142
:1061F8008161176BBF065ABF614FC761C161176BD9
:106208007F065ABF5E4F07620162176BFF0506D50E
:10621800994204D1AE4202D14F00476200E0446285
:10622800176BFF0406D5994204D1AE4202D14F0044
:10623800876200E08462176BBF0506D5994204D1D6
:10624800AE4202D14F00C76200E0C462176B7F05FF
:1062580006D5994204D1AE4202D14F00476400E00E
:106268004464176B3F0506D5994204D1AE4202D16A
:106278004F00876400E08464176BBF0406D5994219
:1062880004D1AE4202D14B00C36400E08464156BB4
:106298003A4BAD0701D1046315E01C6B04F003040D
:1062A800012C01D101630EE01C6B04F00304022CE5
:1062B80002D14FF4004305E01B6B03F00303032BEB
:1062C80001D12F4B0363146B2C4B14F4403F02D1C4
:1062D800C0F834E018E01C6B04F44034B4F5803F97
:1062E80001D1416310E01C6B04F44034B4F5003F65
:1062F80002D14FF4004306E01B6B03F44033B3F5BF
:10630800403F01D11E4B4363146B1C4B14F4402FC8
:1063180002D1C0F838E018E01C6B04F44024B4F54E
:10632800802F01D1816310E01C6B04F44024B4F584
:10633800002F02D14FF4004306E01B6B03F4402307
:10634800B3F5402F01D10E4B8363146B0B4B14F440
:10635800401F02D1C0F83CE020E01C6B04F440145C
:10636800B4F5801F01D1C16318E01C6B04F440141C
:10637800B4F5001F0AD14FF400430EE000100240AC
:1063880000127A0000093D001C0000201B6B03F47A
:106398004013B3F5401F01D1134BC363126B134B6A
:1063A80012F4400F03D1C0F840E0BDE8F0811A6B49
:1063B80002F44002B2F5800F02D10164BDE8F08119
:1063C8001A6B02F44002B2F5000F02D14FF40043F9
:1063D80006E01B6B03F44003B3F5400F01D1024BF9
:1063E8000364BDE8F08100BF00127A00001002408B
:1063F800F0B500230E681C460125A54005EA060EE7
:10640800AE452BD10F797A1E012A15D8856803224B
:106418009A4025EA020282604D7982689D401543C0
:106428008560828892B222EA0E0282808A79858803
:10643800A2402A4392B28280032205689A40D2433E
:106448001540056005689F402F430760C7681740DF
:10645800CA7902FA03F547EA0502C2600134102C32
:1064680003F10203C8D1F0BD38B52DED048B4A4CB9
:106478000368C4F8F8308388A4F8FC30013A0D4664
:10648800072A42D8DFE802F0040A101822292F351B
:10649800B4F8F8300B80B4F8FA3013E0B4F8FA30F6
:1064A8000B80B4F8F83005E0B4F8F8305B420B80A4
:1064B800B4F8FA305B4205E0B4F8FA305B420B807E
:1064C800B4F8F8306B80B4F8FC301DE0B4F8F8305C
:1064D8005B420B80B4F8FA3012E0B4F8FA300B8063
:1064E800B4F8F8300CE0B4F8F8300B80B4F8FA30AF
:1064F80005E0B4F8FA305B420B80B4F8F8305B4240
:106508006B80B4F8FC305B42AB80244B93F830309E
:10651800002B3ED1B5F9003094ED430AD4ED407A12
:1065280009EE103AB5F9023008EE103AB8EEC88A0A
:10653800B5F90430B8EEC99A28EE000A08EE903A88
:10654800A7EE890AF8EEE88AD4ED467AA7EEA80AFB
:106558000DF094F994ED440AD4ED417A288028EEA0
:10656800000AA7EE890AD4ED477AA7EEA80A0DF02B
:1065780085F994ED450AD4ED427A688028EE000A40
:10658800A7EE890AD4ED487AA7EEA80A0DF076F9A5
:10659800A880BDEC048B38BD081000201C0000202A
:1065A800104BDFED117AD3F82421D3F828319289E2
:1065B80083F31003D31A07EE103AB8EEC77A27EE22
:1065C800277A07EE902AF8EEE77AC7EE277AFDEEEB
:1065D800E77A17EE900A6428A8BF642020EAE070E2
:1065E800C0B27047081000200000C842094BD3F819
:1065F8002421137844F6FB7103EB431300FB0313C8
:106608005078C0EB0030B3FBF0F39078B3FBF0F0B8
:1066180080B270470810002010B50A4C94F82D314C
:1066280004EB43030A22B3F83C1104F5A47089B2C1
:10663800A4F8441108F0B2FD80B2FFF7D7FFA4F820
:10664800D00110BD08100020F8B504460E461746C4
:106658000025204620210CF038FF0446D0B1013433
:1066680020460CF097FFB0F5617F05DB40F6340358
:106678009842A8BF184601E04FF46170A0F5617018
:10668800192390FBF3F00DB9307000E070703B787F
:1066980001333B700DB90125DBE72046F8BD30B565
:1066A80005460C461346294622460248BDE83040B6
:1066B80002F08ABD286701087FB504780646E4B968
:1066C800354B1B6803EB8403192193F8870093F873
:1066D800886093F8852093F886304FF4617511FB34
:1066E800005011FB0651009001912C4821460134BD
:1066F80002F06AFD142CE3D14BE00CF04BFF132899
:10670800054641DC244B701C1C68202100238DF8B1
:106718000F300CF0DAFE2035064670B101363046EF
:106728000CF038FF1A289FBF04EB850358719DF8B9
:106738000F30013398BF8DF80F30304620210CF010
:10674800C4FE064670B1013630460CF023FF0D2812
:106758009FBF04EB850398719DF80F30013398BFF4
:106768008DF80F3004EB85043046E11D0DF10F0262
:10677800FFF76AFF9DF80F30042B0AD0601D002137
:1067880004220CF06CFE04E0054800211322FFF7F8
:1067980086FF04B070BD00BFD80E0020476701080F
:1067A8005C670108014808F087B900BF6267010803
:1067B800F8B50478064674B9304DB5F8C421B5F873
:1067C800C6312F482146013402F0FEFC042C05F1A5
:1067D8000405F2D1F8BD2B490CF04AFEA8B9274BA5
:1067E8004FF47A714FF4FA62A3F8C411A3F8C621E2
:1067F800A3F8C811A3F8CA21A3F8CC11A3F8CE2195
:10680800A3F8D011A3F8D221F8BD30460CF0C2FE8F
:10681800032805462BD8304620210CF056FE0446A6
:1068280030B1013420460CF0B5FE0126074600E0E1
:106838000646204620210CF048FE10B9BDE8F84075
:10684800B0E701300CF0A6FE012EF7D1A7F2EE2238
:1068580040F2DC539A42F1D8A0F2EE229A42EDD8E7
:10686800064B703503EB85039F80D880F8BD06483A
:1068780000210322BDE8F84011E700BF401D0020B9
:1068880070670108836701081C7501082DE9FF413D
:1068980004780546002C39D17348744D08F00CF97A
:1068A800D5ED047AF5EE407AF1EE10FA00F0D880D2
:1068B80021466F4802F088FC95ED040A684602F00C
:1068C80003FB01466B4802F07FFC95ED050A68461C
:1068D80002F0FAFA0146674802F076FC95ED060ADE
:1068E800684602F0F1FA0146624802F06DFC95ED47
:1068F800070A684602F0E8FA013401465E4802F0E9
:1069080063FC0C2C05F11005CAD1A9E05B490522EE
:106918000CF0F2FD40B9554B03F1C002002143F8D9
:10692800101F9342FAD19BE02846554904220CF0E7
:10693800E3FD04462846002C40D120210CF0C5FD7B
:10694800002800F08D80451C28460CF0CCFD074639
:106958004C4B53F824601EB94B4808F0ADF87FE063
:1069680028463146FAB20CF0C7FD01340028EFD1B1
:106978003E4B03F1C0029E46002143F8101F93428C
:10698800FAD1424B03EBC4029846D2F804C0BCF1DA
:10699800000F04D131463E4802F016FC57E00027AC
:1069A80018F834309F42F5DA3B010EEB03056344D7
:1069B8000FCB103585E80F000137F1E70CF0EAFD41
:1069C8000B28064647DC284620210CF07EFD0546AC
:1069D80050B10135284602F0EDF9244B03EB0613BC
:1069E80083ED040A012400E00446284620210CF027
:1069F8006CFD054648B10135284602F0DBF91B4B12
:106A080003EB061383ED050A0134284620210CF018
:106A18005CFD054648B10135284602F0CBF9134B19
:106A280003EB061383ED060A0134284620210CF0F7
:106A38004CFD10B9FFF7B6FE12E0013002F0BAF9CA
:106A48000A4B032C03EB061686ED070AF2D1114810
:106A5800FFF71CFF04E0104801210C22FFF71FFE7E
:106A680004B0BDE8F08100BF89670108401D00201F
:106A7800A4670108AA670108A072010883670108D2
:106A8800AE670108804D0108B36701085866010820
:106A9800C26701083C6501085C670108F0B5047825
:106AA80087B006461CBB514B1968062303FB04112B
:106AB800192091F8D65091F8D77091F8DA2091F80A
:106AC800D5304FF4617610FB056510FB0760009523
:106AD800019091F8D8000290D0314548497A039145
:106AE8002146013402F070FB0C2CDCD17CE00CF068
:106AF80051FD0B28044672DC3C4B701C1D6820219C
:106B080000238DF817300CF0E0FC064680B1013602
:106B180030460CF03FFD03289FBF062303FB0453B8
:106B280083F8DA009DF817309CBF01338DF81730D1
:106B3800304620210CF0C9FC074680B101373846A1
:106B48000CF028FD0D289FBF062303FB045383F890
:106B5800D5009DF817309CBF01338DF817300626F5
:106B68006643A9193846D6310DF11702FFF76CFDB7
:106B780020210CF0AAFC074670B1013738460CF00A
:106B880009FD14289FBF9DF817307619013386F840
:106B9800D80098BF8DF81730384620210CF095FCA6
:106BA80078B101300CF0F6FC0D289FBF062303FBDB
:106BB800045383F8D9009DF817309CBF01338DF832
:106BC80017309DF81730062B0ED0062202FB045012
:106BD8000021D5300CF043FCFFF7E4FD04E0054844
:106BE80000210B22FFF75BFD07B0F0BDD80E002097
:106BF800CE6701085C6701082DE9F347047807466A
:106C08004CB9204601A907F0FBFB0134FFF7F4FF5C
:106C1800122CF6D179E00CF0BDFCC5B2112D6FD85D
:106C2800781C20210CF051FC394C3A4F05F1D00664
:106C3800034614F8168030B9A8F10202D2F1000810
:106C480048EB020843E000F1010A597838460CF095
:106C58003CFC60B1032D8CBF03230023C01B3B44C5
:106C680053FA80F090F80490B9F1030F02D1FFF7BE
:106C780099FD4AE0A9F10203D3F1000850464FF00C
:106C8800200148EB03080CF020FCD8B1B8F1000F44
:106C9800EDD001300CF07EFC40F2ED2380B298423A
:106CA80005DD40F6CA039842A8BF184601E040F245
:106CB800EE2004EB4603A0F2EE20192290FBF2F03E
:106CC800587002E0B8F1000FD1D104F8169014F80A
:106CD8001630FA5CB8F1000F0DD00D4B0E4803EBDF
:106CE80046062946737840F2EE24192505FB03432E
:106CF80002F06AFA09E02946084802F065FA04E059
:106D0800074800211122FFF7CAFC02B0BDE8F0874E
:106D1800401D0020C4460108EE670108006801080C
:106D28001C75010807B50123ADF8041001A98DF8F9
:106D380006208DF80730FEF78BFC03B05DF804FBE6
:106D48002DE9F041064672B62D4D80214027298550
:106D5800284604222F85FFF7E5FF284639460122F9
:106D6800FFF7E0FF274850F8364000EBC6002368DD
:106D780042680126510006FA01F848EA03039640E2
:106D88002360A661AF612B8A1F06FCD4236848EAFA
:106D9800030323601A4B4022B1B221851A852022B1
:106DA8009A6140F60557164D2B8A180603D4002F12
:106DB800F9D0013FF7E7A66120460422FFF7B2FFAA
:106DC80087B10F4B1A8A1206E0D5228A92B2164270
:106DD8004FF040014FF0200215BF996119859A6163
:106DE8001A85EEE740212023A9612846AB610222DB
:106DF800FFF798FF62B60A20BDE8F04108F008B92D
:106E08000004004830680108002208490C2303FBED
:106E180002135968814204D10022C2621A725A6070
:106E280070470132042AF0D1704700BF2C2500209A
:106E38002DE9F04F87B0074602919DF8444011466E
:106E48001A469DF8403000250C20674E684300EB39
:106E5800060E8057B842B14605D19EF808A0BAF18F
:106E6800000F04D0BBE00135042DEDD1B7E0012FB0
:106E780000F0A48005DC002F40F0B18000945B484E
:106E8800A1E0022F00F09D80142F40F0A880584EFA
:106E9800B36943F00103B36173694FF0904443F45D
:106EA8000033736103224FF0010B4FF4805804A99B
:106EB8004FF090408DF815200392CDF810808DF892
:106EC80014B08DF816B08DF817A0FFF791FAA4F852
:106ED8002880C82008F09CF8C4F818807369039AC1
:106EE80043F40033736120464FF4C0538DF81520E6
:106EF80004A902228DF81420039204938DF816A099
:106F08008DF817A0FFF774FA636A23F4704363627D
:106F1800636A43F460436362636A23F470236362C1
:106F2800636A43F460236362324B334C4FF480212D
:106F380019601223A36404F14800082384F84D3033
:106F480084F84EB007F0C8F92C4B2D49C3F800A0BF
:106F5800F369039A43F40003F3612A4B04A8D96048
:106F68008DF810708DF811208DF812A08DF813B0DF
:106F780007F068F92A238DF810309DF813308DF842
:106F880011B08DF812A01BB104A807F05BF904E05A
:106F98001D4B4FF48062C3F884201C4A1C4B1360BD
:106FA80002221A721B4A1C4B13601C4A1C491B689C
:106FB800116098471B4B23600F4807E000941A485C
:106FC80001E01A48009404F035FA40B10C2303FBA1
:106FD80005959DF8083007712B72686000E0002065
:106FE80007B0BDE8F08F00BF2C2500200038014015
:106FF8000010024014040140E0110020D800424271
:107008000005FA0500ED00E000E100E07C1C00202E
:107018005C250020E01A0020D0000020DC1A0020A7
:1070280050000020D04601080044004000480040BD
:1070380010B5084B1968002201EBC20393F902400E
:10704800844201D1981C10BD0132042AF4D10020D9
:1070580010BD00BF28250020F0B5027887B08AB996
:107068004A4C04F1200694F8F02100234849595667
:1070780050B281426ED00C33302BF7D10834B44271
:10708800F1D181E0002204920592451C0CF082FAAD
:10709800C4B260B2FFF7CCFF074618B18DF81040B4
:1070A800012400E00446284620210CF00EFA05468B
:1070B80038B1013528460CF06DFA0134ADF81200EC
:1070C800E4B20026284620210CF0FFF9B0B3451C95
:1070D80028460CF05FFA00222E4951F822308342EC
:1070E8005FFA82FE04D00132082AF5D1002300E0BD
:1070F800734651F82320824220D1022E0FD0032E4E
:1071080012D05A1E012ED2B204D0042A13D88DF8F8
:1071180014300EE0042A0ED88DF8153009E0052B3E
:1071280009D88DF8173004E09A1E052A03D88DF87F
:1071380016300134E4B20136042EC3D1052C04D82C
:1071480007B0BDE8F040FFF72DBB04AB03CB3860B8
:10715800796019E094F8F5010E4B94F8F45153F85E
:107168002000B4F8F221009094F8F70153F82000B9
:10717800019094F8F60153F82000029053F8253056
:10718800054802F021F879E707B0F0BD401D00205E
:107198002C250020FC5301080F68010838B14388EA
:1071A80011EA030003D08B420CBF01200220704774
:1071B80030B50B4B0B491C6891F85020032A0BD8AB
:1071C800134604EBC303551CEAB29D882842F5D048
:1071D80081F85020981C30BD81F85020002030BD27
:1071E80028250020E0110020024B002283F85020BF
:1071F800DEE700BFE01100202DE9F047877890F81E
:1072080003C0214DBBB2C7F1640E03EB83065C4299
:10721800C3F178005FFA8EFE7600CCF16408A4B260
:1072280080B2A3B20FFA83F9B9F1000F05DC002B85
:1072380014BFBA464FF0010A00E0F24613FB03F30D
:1072480003FB0CF21AFB0AF392FBF3F3434403FB30
:1072580009F30A2293FBF2F333449BB225F8023F69
:10726800B1F800904A880A34C9EB020AA4B21AB2EB
:1072780002FB0AF24FF47A73844292FBF3F34B4415
:107288002B80CED1BDE8F0873012002038B500241D
:107298000B4D6059254407F00FFC696811B1094886
:1072A80001F092FFA96811B1074801F08DFF074866
:1072B800103407F001FCB4F5E87FE9D138BD00BF10
:1072C800B04B01087068010876680108FC73010872
:1072D80070B5054628460CF006F9064658B91A4B0B
:1072E8001A485A791A4B03EB8203BDE87040D3F869
:1072F800CC1101F069BF2846164932460CF0FCF85B
:1073080060B91548154C07F0D7FB54F8041F19B19C
:10731800134801F059FFF8E7124805E00024124B22
:1073280053F8241021B91148BDE8704007F0C4BBD8
:10733800284632460CF0E0F801340028EFD1024B21
:107348000B4D5C71C6E700BF401D00207C6801083A
:10735800B04B0108886801088D6801087C4D010858
:10736800A0680108FC730108804D0108B367010893
:107378003C650108F0B585B004460CF0B4F808285F
:1073880026D1621EE01D1F4912F8013F0968194401
:10739800497801F00301022908BF203B824213709B
:1073A800F1D1254604F1080715F8016B1648314656
:1073B8000CF08BF820B1284631460CF086F810B155
:1073C800FFF7F0F91CE0BD42EED1204607F0C6F801
:1073D8000E4807F071FB00230D4A1A4404A992F8DD
:1073E80088210A440849595C02F80C1C0133082B0F
:1073F800F2D1002307488DF80C3001A901F0E4FE12
:1074080005B0F0BD0C01002016720108A46801083F
:10741800401D0020A07201082DE9F04105460CF03E
:1074280062F82F4B04469E6888B92E4807F044FB43
:107438002D4B53F8241041B10123A340334202D00D
:107448002A4801F0C1FE0134F2E7294821E0284624
:10745800284922460CF050F858B92748274C07F01D
:107468002BFB54F8041F0029EFD0204801F0ACFE94
:10747800F7E72B782D2B03BF013504F1FF344FF0CC
:1074880001084FF000080026174B53F8267027B95B
:107498001B48BDE8F04107F00FBB28463946224695
:1074A8000CF02AF8C8B90120B040020601D51548E9
:1074B800EFE78305FBD4B8F1000F03D001F09EFF7E
:1074C800114802E001F0A2FF104807F0F5FA39462A
:1074D8000F48BDE8F04101F077BE0136D4E700BFA0
:1074E800401D0020AA680108E84D0108A0680108AD
:1074F800FC73010888680108B4680108E44D0108B4
:10750800B3670108C0680108CE680108D768010898
:107518009F72010810B5084807F0CEFA074B0024FF
:107528001C701C63064B1C7007F0C4FF07F076FC48
:10753800044B1C6010BD00BFDF6801084C1200201E
:10754800952A0020A025002070B5064600240B4B84
:10755800E518AA8816420AD0E158094801F034FE15
:107568002846002107F035FA064807F0A5FA143432
:1075780040F6CC339C42EAD170BD00BF5C5601088E
:107588000B690108FC73010808B5084801F01CFEE6
:1075980005F09EFD05F09EFC18B9642007F038FD43
:1075A800F8E70348BDE8084001F00EBE1569010878
:1075B800226901082DE9FF410A4806888568448840
:1075C800B0F80480C76805F075FCCDF8008002901B
:1075D800019731462A462346034801F0F5FD04B0D9
:1075E800BDE8F0810C0000202A690108F0B5047894
:1075F8008BB005460CB1002436E04B4B19680E23BE
:1076080003FB041101F59070B1F92951B1F9252155
:10761800B1F92731009591F82C51019591F82D5128
:10762800029590F90B00039001F594713F4891F988
:10763800061004912146013401F0C6FD082CDCD166
:1076480070E02D2B14D1072C1BDC28460BF0A2FF71
:107658000AAB661C03EB440424F8100C15F8013F30
:10766800303B092BFAD934462B78002BE9D104E0BA
:10767800A3F13002092A09D8E5E7082CBDF818203B
:1076880009D00BB0BDE8F040FFF78CB8202BF8D13B
:1076980001352646E7E7072AF3D8BDF81A00224B3A
:1076A800A0F2EE2189B240F2DC55A9421B68E8D865
:1076B800BDF81C10A1F2EE24A4B2AC42E1D8BDF88A
:1076C8001E6004B237B2A742DBDB0DB2AF42D8DC92
:1076D800A542D6DBBDF8247007F16404A4B2C82C17
:1076E800CFD8BDF826E00FFA8EF4112CC9DCBDF80E
:1076F8002050B42DC5D8BDF82240B42CC1D812B240
:107708004FF00E0C0CFB0233A3F82501A3F8271148
:10771800A3F8296183F82C5183F82D4183F82B7144
:1077280083F82EE10BB0F0BDD80E00208769010860
:10773800F0B504468FB020460BF0D5FEC5B225BB88
:10774800AF48B04C07F0B8F994F8D21009B9AE4870
:1077580054E049B294F8D02094F8D130009194F8CC
:10776800D310019194F9D410029194F9D510039192
:1077780094F8D6100491A5482946013501F024FD56
:10778800102D04F10704DFD1E1E72046A0490522C6
:107798000BF0B2FE0546B8B929469E4870220BF098
:1077A8005EFE9D4B196828460E2303FB001301302B
:1077B8000022082883F82F2183F8302183F831210B
:1077C80083F83221F0D119E12046944904220BF0C4
:1077D80093FE05462046002D4AD120210BF075FE68
:1077E800002800F00B81461C30460BF07CFE2C462E
:1077F80007468B4B53F824502DB98A480FB0BDE883
:10780800F04001F0E1BC30462946FAB20BF074FEB4
:1078180001340028EDD17B4A02F17001164600239D
:1078280082F8D63082F8D23082F8D13082F8D0305F
:1078380007328A42F3D17C4901EBC40191F89022C6
:10784800934210DAD1F89472C3EBC302B0183A44E9
:1078580000F1D0011768C0F8D070908888809279BC
:107868008A710133E7E72946704801F0ADFC96E0DC
:107878006F4907220BF040FE05462046002D4AD1ED
:1078880020210BF022FE06460BF02DFEC4B274BB7D
:10789800684801F099FC21466748013401F094FCDE
:1078A8000E2CF8D1584801F08FFC0024634821467B
:1078B80001F08AFC0025584A614811680E2202FB33
:1078C80004120123D2F82F215E49AB4013425E4BCC
:1078D80005F1010508BF194601F076FC0E2DEAD125
:1078E8004948013401F070FC082CDFD186E03046AD
:1078F80056490BF053FE2C46002852D0022C55D086
:107908000BF048FE06AB514943F8240000200BF069
:1079180045FE0134F0E74D490BF040FE002460B10C
:10792800082C3ED00BF036FE06AB484943F824003D
:1079380000200BF033FE0134F1E7082C31D1069B0F
:107948000F2B2ED8DDF81CE0BEF1070F29D8089FB1
:107958000D2F26D8099E06F16402C82A21D80A9D4F
:10796800FF2D1ED80B9864281BD80C99642918D8A9
:10797800884216DA0D9C032C13D8224AC3EBC303A2
:10798800134483F8D0E083F8D17083F8D26083F889
:10799800D35083F8D40083F8D51083F8D6402C4C04
:1079A800C9E60FB0BDE8F040FEF7FCBE069B072B0A
:1079B80020D807990D291DD80278722A0DD06E2A71
:1079C80018D1154A12680E2000FB032301228A40B1
:1079D800D3F82F1121EA020209E00F4A12680E209B
:1079E80000FB032301228A40D3F82F110A43C3F86E
:1079F8002F2101E0FEF7D6FE0D4C9CE60FB0F0BD3E
:107A0800AF690108401D0020FC730108DA6901080C
:107A180083670108101E0020D80E0020AE670108F9
:107A2800804D0108B3670108B04B0108C26701081F
:107A3800A76901087A680108F66901085D710108FB
:107A4800FB6901086476010804770108FF690108E9
:107A58003C6501082DE9F743047805468CB9324D99
:107A680095F8A312B5F8A02295F8A2322F480091F4
:107A78002146013401F0A8FB102C05F10405EFD1D3
:107A88004EE00BF087FD0F28044636DC28462021FF
:107A98000BF01BFD264EE4B2D6F83480451CA4003A
:107AA800002728460BF076FD5FFA87F9B9F1010F38
:107AB80083B208D0B9F1020F0BD0B3F5B47F24D24A
:107AC800726B13530AE0FF2B1FD8736B2344987013
:107AD80004E0FF2B19D8736B2344D87028462C2157
:107AE8000BF0F3FC054608B1013502E0B9F1020FCD
:107AF8000BD10137032FD4D112E00E4800210F22F9
:107B080003B0BDE8F043FEF7CABD08EB040000214E
:107B180004220BF0A4FC03B0BDE8F043FEF742BE1C
:107B280003B0BDE8F08300BF401D0020016A0108D2
:107B38004C1200205C6701082DE9F04304788FB0EF
:107B48000546002C59D17C4B0021142209A807AE08
:107B5800D3F838800BF083FC0722304600210BF065
:107B68007EFC05A80023A700059308EB0705838082
:107B78001A467249B5F802E031F813C01CEA0E0F34
:107B88000AD00DF1380C0E3102F1010E6244595C35
:107B980002F81C1C5FFA8EF20133072BE9D1002191
:107BA8000B46674AB5F802E011F802C01CEA0E0F4E
:107BB8000AD00DF1380C063203F1010E63448A5CD9
:107BC80003F8242C5FFA8EF301310629E9D118F85D
:107BD80007305C498DE841006A78029209A81A09C1
:107BE80003F00F0301F0DBFA2146574809AA0134D4
:107BF80001F0EAFA202CA6D19BE00BF0CBFC1F2861
:107C0800044600F3898028462021E4B20BF05DFC8D
:107C18001F2C02D9FEF7C6FD8BE0474B9B6B03EB8D
:107C28008404451C0021204604220BF018FC002780
:107C3800464B09AE304600210A2217F803905FFA36
:107C480087F80BF00CFC002315F8012B32B10A2B36
:107C580004D04A4502D0F2540133F5E74A4561D1D0
:107C680008F1FF33032B09D8DFE803F010050242BF
:107C78000DF1230037E00DF123011FE030460BF032
:107C880089FC2378C0B243EA001006E030460BF0C6
:107C980081FC237800F00F001843207034E0013392
:107CA800062B0BD02A4800F27B369E5D9642F6D111
:107CB800034493F8752363881343638011F8012FF5
:107CC80012B30023EEE70133072B0CD0204A02F24F
:107CD8006E369E5D8E42F6D102EB4303B3F8602305
:107CE80063881343638010F8011F69B10023EDE72F
:107CF80030460BF04FFC0F2804DC30460BF04AFCF2
:107D0800607001E0002363700137052F90D10124D2
:107D180000F032FE6CB97DE70E4800211F22FEF705
:107D2800BEFC06E02046002104220BF098FB00244C
:107D3800EEE70FB0BDE8F0834C120020104F0108A9
:107D4800254F0108156A0108246A0108314F010806
:107D5800B04B01085C6701082DE9F0412DED048B5B
:107D6800B1498AB004460BF083FBB049002820468D
:107D78000CBF012607260BF07BFBAD4900282046E7
:107D880008BF02260BF074FB002808BF0426F10781
:107D980040F1F080A748A84C06F08EFE002006F0BF
:107DA80093FCA64806F088FEA54806F085FE627991
:107DB800A44BA54803EB82032546D3F8CC1101F068
:107DC80003FAA24801F000FA4FF00008274695EDA3
:107DD800048AB5EE408AF1EE10FA04D19C4801F00D
:107DE800F3F9002570E09B48D5ED059A95ED069AC4
:107DF800D5ED078A414601F0E7F9B5EEC08AF1EE04
:107E080010FA02D5202006F04FFEB0EE480A06A868
:107E180001F05AF80146904801F0D6F9F5EEC09AFB
:107E2800F1EE10FA02D5202006F03EFEB0EE690A07
:107E380006A801F049F80146874801F0C5F9B5EEF2
:107E4800C09AF1EE10FA02D5202006F02DFEB0EE11
:107E5800490A06A801F038F801467F4801F0B4F94C
:107E6800F5EEC08AF1EE10FA02D5202006F01CFECD
:107E7800B0EE680A06A801F027F808F101080146E3
:107E8800764801F0A1F9B8F10C0F05F110059ED163
:107E9800A4E749B294F8D02094F8D130009194F82E
:107EA800D310019194F9D410029194F9D51003914B
:107EB80094F8D61004916A482946013501F084F9EE
:107EC800102D04F1070403D094F8D2100029E0D152
:107ED8006448654C06F0F0FDD7F8088054F8041F94
:107EE80019B1624801F070F9F8E70D46604B53F894
:107EF800254054B10123AB4013EA080F03D05D4875
:107F0800214601F061F90135F0E75B4806F0D4FD40
:107F180021467B180AAA93F888311344574A8A5C89
:107F280003F8102C01310829F3D1002306A954487D
:107F38008DF8203001F048F9524806F0BDFD52484E
:107F4800FFF78AF8514806F0B7FD4F48FFF7F4FDF0
:107F58004F4806F0B1FD4C48FFF77CFD4D4801F055
:107F680033F94020FFF7F0FA4B4806F0A5FD4648E4
:107F7800FEF742FEB20739D5484806F09DFD48484D
:107F880006F09AFD404806F0DFFB464806F094FDEF
:107F98003D48FEF791FB444806F08EFD3A48FEF74F
:107FA8007DFD424801F010F93748FEF701FC4048D2
:107FB80006F082FD3448FFF719FB00270E257D43A4
:107FC80000243C4AD26B2A440123D2F80A20A34059
:107FD80013421ED101340E2CF3D10137082FEDD1F5
:107FE8002C4801F0F1F88020FFF7AEFA730716D598
:107FF800314806F061FD314806F05EFD224806F082
:108008007DFB244801F0E0F84FF48070FFF79CFAFC
:1080180005E0394622462A4801F0D6F8DAE70AB0E0
:10802800BDEC048BBDE8F081306A01087F6E010861
:10803800376A01083D6A0108401D00204B6A0108A3
:108048005D6A0108B04B0108696A0108746A010891
:10805800816A01088E6A010879680108A07201081E
:10806800A66A0108966A0108E44D0108C56A010874
:10807800E84D0108D36A0108E06A01081672010890
:10808800EC6A0108F56A01083C650108046B0108FF
:10809800106B0108FC7301081E6B01082B6B0108AB
:1080A8003E6B01084C6B0108566B0108656B0108B3
:1080B800736B01084C1200207F6B0108906B01085C
:1080C800A26B0108022803D0431E5842584170474A
:1080D800064B1B681B7823B1054B1868C0F3C040DA
:1080E8007047044B1878C0F3800070471C0D0020BF
:1080F8009C0E0020942A002008B507480BF0F3F9DD
:10810800C0B21428044B04D8421C20211954D0B200
:10811800F7E700221A5408BD8C120020674B73B58C
:108128001878674DFFF7CEFF2B788342044620D09E
:10813800C8B1644B1B68E3B193F9000002230093B4
:10814800614B1B685B78003318BF0123019304213E
:108158004FF416530022FEF76BFE5C4B186040B1DB
:1081680001232B7005E0594E3068FEF74DFE346050
:108178002C70574B574D1878FFF7A4FF2B78834284
:10818800044618D088B1544B1B68A3B100220124BF
:1081980093F9000000944FF4964301920821FEF7EA
:1081A80047FE4E4B186028B905E04C4E3068FEF784
:1081B8002BFE34602C704A4B4A4D1878FFF782FF2B
:1081C8002B78834204462E4642D0002837D0464BAF
:1081D8001A68002A3CD0D37992F90000434C002B4E
:1081E80008BF022302220092002254F82330019291
:1081F8001021FEF71DFE3E4B0546186040B33D4C6E
:1082080094F84A30022B0BD094F89620022A01D118
:108218004C3405E023B1002A04F14C0418BF0024B3
:10822800354B1C6044B1204600214C220BF017F955
:108238000223256084F84A300123337008E02C4E6D
:10824800306806F041FB3068FEF7DEFD34602C70C4
:108258002A4B2B4D1878FFF735FF2B7883420446BD
:1082680029D000B3274B1B682BB3274A93F900008A
:1082780012685278002A0CBF0822092203230093AF
:1082880001924FF4614320210022FEF7D1FD1F4BDC
:10829800186080B11E4A012313702B701D4B1A6899
:1082A8001D4B1A6007E0194E3068FEF7ADFD184BFC
:1082B80034601C702C7002B070BD00BF240D00200B
:1082C80029070020200D002034070020301300204B
:1082D800250D0020380700208C0700207C0700208F
:1082E800300D0020920700202C0D0020FC530108BF
:1082F80094070020A81C0020980700203C0D0020AF
:10830800A0070020380D0020340D0020A40700200D
:10831800A8070020442A0020AC070020642928BFB1
:108328006421F8B510FB01F56424064695FBF4F4C6
:108338000027E4B2FBB2A34204D29F2004F085FFD9
:108348000137F7E7B4420BD2C4EB84101421C4EB15
:10835800800095FBF1F5663D2844C0B204F075FF36
:108368000134E4B2B44201D29A20F7E7F8BD2DE90E
:10837800F743B74C06F030FEA369C31A002BC0F2CE
:108388006B8200F5433303F5A073A361B14B1E78EC
:10839800237FC6F38006F31A18BF012326774EB150
:1083A800002B00F05982AC4B5A789A7001225A700F
:1083B8001A7025E0A84A2BB1D37843F00203D37092
:1083C80093785370D57805F0020101F0FF0339B9AD
:1083D800A1498968411A002903DB05F0010300E07F
:1083E800012303F001079C4917704BB1ED0707D52E
:1083F8000B799A4A013303F003030B71D35C4B707A
:10840800954DDFF8B8822B787BB3EB7823F0020325
:10841800EB70934B0344AE20AB6005F06BF808B1EA
:1084280004F0A4FE88F80000002800F01582B020AF
:1084380005F060F8402005F05DF8002005F05AF8D6
:10844800102005F057F84FF48067013F0020BFB2B5
:1084580005F04BF8002FF8D1384604F01AFF6A7877
:10846800804B53F8220004F00BFF98F80030002BE3
:1084780000F0F2816B78052B00F2AD81DFE813F094
:108488000600AB011700770050016B017649774A67
:10849800774B6F4800F083FE012004F0FAFE6C4829
:1084A80004F0EEFE022004F0F4FE724891E1724FEF
:1084B8003B68990735D5DFF80882DFF80892B8F8E5
:1084C800001063480A23B1FBF3F203FB121399F877
:1084D8000010009192B269499BB200F060FEFFF76C
:1084E8000BFE012004F0D5FE594804F0C9FE644B88
:1084F80099F800201868B8F80030057905FB1231A2
:1085080064234B43C1784D1B55430220B3FBF5F55B
:10851800EDB204F0BEFE29461520FFF7FFFE032545
:1085280000E001253B681A0540F15581554B564935
:108538001F68096800916423544997FBF3F2444883
:1085480003FB127300F02BFEFFF7D6FD284604F05C
:10855800A0FE3F4804F094FEFEF722F80746681C88
:1085680004F097FE15203946FFF7D8FE33E10120C5
:1085780004F08FFE464804F083FE464B1A6812F05A
:10858800020F1F4617D0444A3148B2F90210B2F917
:1085980000300091B2F9042040490192404A00F0AD
:1085A800FEFDFFF7A9FD022004F073FE284804F041
:1085B80067FE032500E002253B68DB0718D5394A2A
:1085C8002348B2F90210B2F900300091B2F9042040
:1085D80032490192344A00F0E2FDFFF78DFD28464A
:1085E80004F057FE1A486F1C04F04AFEFFB23D46DD
:1085F8002E4A2A49B2F90030B2F9022000922C4AD8
:108608001348B2F9002001922A4A2B4F00F0C7FD07
:10861800FFF772FD284604F03CFE0D4804F030FEDA
:1086280097ED000A0A4800F04FFC09480AF05BFF82
:1086380005F101085FFA88F8C0B2092844D8431C3C
:10864800DBB220222254E218002151701846F4E7C8
:108658008C120020942A0020FC0D0020B87001081C
:10866800404B4C00F44F0108BC700108C57001086C
:10867800E1620108CC700108382A0020D470010892
:108688002C110020FC0E002030110020EC70010895
:1086980001710108940E0020BC0E0020177101081A
:1086A80026710108C20E00202A710108F40E00206C
:1086B800F80E00202E7101084C080020C90900207E
:1086C800D81100200801002097ED010A204400F08D
:1086D800FBFBFFF711FD404604F0DBFD604804F0AA
:1086E800CFFD97ED020A5E4800F0EEFB5C480AF009
:1086F800FAFE0235EDB2C0B2092808D8431CDBB235
:1087080020222254E218002151701846F4E79FED08
:10871800550A204400F0D8FBFFF7EEFC284655E048
:108728000025514F3B78AB4255D90E2D53D06808E0
:10873800013004F0AEFD284605F03CFE3B78AB4224
:1087480006D9202004F081FD681CC0B205F032FE75
:108758000235EDB2E5E7454D454995F8A82740486B
:1087680000F01DFD012004F094FD3D4804F088FD53
:10877800404B41491F783A483A4600F010FD022024
:1087880004F087FD364804F07BFD0C2303FB0755F6
:108798003A4995F8AB2795F8AA37314800F0FFFC1D
:1087A800FFF7AAFC032004F074FD2D4804F068FDCF
:1087B80095F8B01795F8AE2795F8AF372848009187
:1087C8002F4900F0ECFCFFF797FC042004F061FD52
:1087D800234804F055FD002E3ED12A4B93F8203053
:1087E800052B9CBF284A9B184FF0B00094BF1D7EF4
:1087F8003F2504F07FFE0C2004F07CFE162004F0D8
:1088080079FE284604F021FDB02004F073FE022012
:1088180004F070FE172004F06DFE1C4B1B78002B33
:108828001B4B1B7814BF72202120002B18BF52202D
:1088380004F00BFDB02004F05DFE082004F05AFEA1
:10884800172004F057FE657F124B585D013505F07F
:10885800030504F0FAFC657703B0BDE8F08300BFB8
:108868008C1200200000000020250020401D002060
:10887800327101087C2500203E7101084F71010802
:1088880060710108482A0020F44F01086C0D00208F
:10889800D20D00207271010810B54B88DC0641BF6B
:1088A8002F4B14791B6853F8244044BF2D4B43F8D1
:1088B80020404B889B0641BF294B54791B6853F8CD
:1088C800244044BF274B43F820404B881C070ED553
:1088D800254B0C781B78B3EB141FA1BF204BD47821
:1088E8001B6853F82440A4BF1E4B43F820404B8814
:1088F8009B070ED51D4B0C781B78B3EB141FDFBFFD
:10890800174B54781B6853F82440DCBF154B43F8C9
:1089180020404B88DC070FD5154C0B78247803F0E2
:108928000F03A342DFBF0E4B14781B6853F8244093
:10893800DCBF0C4B43F820404B885B070FD50B7806
:108948000C49097803F00F038B42A1BF044B9278BE
:108958001B6853F82220A4BF024B43F8202010BD07
:1089680080120020B40700204B080020490800208E
:10897800480800204A080020254A2648264900239E
:10898800F0B5156803708B771C461A462E19768841
:108998004EB92F5D3FB9037000238A77CB770778EC
:1089A8001C461A460CE0360548BF013204F104049F
:1089B80003F1010348BFD2B2802CDBB2E6D1EAE76B
:1089C800E0B2B8420CD215F8240006099E4200F025
:1089D8000F00A8BF731C9042A8BF421C0134EFE7E8
:1089E80081F82020CB77C2F3470102F001020A4444
:1089F8004C1E0A490A480A70C3F3470203F00103F0
:108A0800134404700749501E074A08701370F0BDDC
:108A180084120020400800208C1200204A08002000
:108A2800480800204B080020490800202DE9FF478E
:108A3800704B714933F9103004462BB902280CD019
:108A48006E4B1B88980708D06D4B002223F8142022
:108A58006C4B1B8821F81430C8E031F814301BB96E
:108A6800694A02EB8402536201339BB221F8143045
:108A78001BB2002B18DD022C634A644809D1D66A60
:108A8800B0F90450202095FBF0F505FB0060D0629A
:108A98000AE002EB840230F91450566A802095FBF4
:108AA800F0F505FB00605062594F386890F85E2079
:108AB800934240F09B80544ADFF8448102EB8402E1
:108AC80000EB040E022C556A95FBF3F39EF8575001
:108AD800536208BF5E424FF0000221F8142007BF1E
:108AE800B6B214219EB20A21002D7DD0002E7BD073
:108AF80038F81420002A77D00FFA86F90FFA82FC8A
:108B0800E14571D089EAE9728CEAEC7AA2EBE97264
:108B1800AAEBEC7ACAEB0202B9F1000F12B209B261
:108B2800DFF8F89003DDBCF1000F03DC20E0BCF1B6
:108B3800000F1DDA8A420BDD022C90F85A2002D170
:108B480002F580720EE039F8141040320A4419E038
:108B580049428A4218DA022C11D190F85A20C2F5FB
:108B68007F42C032B9F804100A44A9F804200BE087
:108B7800002AB8BF52428A4206DD022C04D039F8D6
:108B88001420203A29F8142039F914209EF854901A
:108B980092114A4503DBAA42A8BF2A4691461D4ABC
:108BA800126812031FFA89F508D5142001A98DF857
:108BB80004400293ADF80C5001F0F2FF164B1B78FD
:108BC80073B12AB207EE902AF8EEE77AB2EE047A89
:108BD800C7EE877A3B6803EB8403C3ED087A03E0AA
:108BE8003B68234483F8019028F8146004B0BDE87A
:108BF800F08700BF3C190020EC010020980E0020EF
:108C0800E6010020DE0100208C120020C20E0020A8
:108C1800D8010020382A0020DC010020E0010020D3
:108C280030B50B4C0B4D22782B789A4285B00CD07E
:108C3800684602A904F022F90123684602A9022223
:108C480004F07CF900232B70237005B030BD00BF01
:108C5800F91B0020F81B0020F0B50124B0FBF4F547
:108C68008D4201D34C43F9E70026D4B1B0FBF4F5AB
:108C780004FB1500B4FBF1F41EB9002D01DC002C37
:108C8800F3D1092D03F1010EEFB204DD002A14BF60
:108C98003725572500E030253D441D7001367346C1
:108CA800E3E71C70F0BDF0B50124B0FBF4F58D428C
:108CB80001D34C43F9E70026D4B1B0FBF4F504FB2B
:108CC8001500B4FBF1F41EB9002D01DC002CF3D122
:108CD800092D03F1010EEFB204DD002A14BF372578
:108CE800572500E030253D441D7001367346E3E703
:108CF8001C70F0BD03685A1C0260197070472DE99A
:108D0800F843089E002B07468846144614BF4FF0C8
:108D180030094FF02009334613F8012B0AB92546CC
:108D280003E0002CFBDD013CF6E7002D04DD3846AE
:108D38004946C047013DF8E724EAE4743546A01BDC
:108D4800284415F8011B11B13846C047F7E7BDE8BC
:108D5800F883024B186806F01EBA00BF780E002090
:108D680090ED017A07EE901AB5EE407AF1EE10FA1E
:108D780001BFF8EEE77A9FED0E7A67EE877AB7EED5
:108D8800007A04BFC7EE277AC0ED017A90ED017A28
:108D9800D0ED007A30EE877A30EE670AC0EE870AA7
:108DA800E0EE807AB0EE670AC0ED007A704700BF47
:108DB800DB0FC94010B50278202A034600F10100F4
:108DC800F9D0092AF7D02D2A03D10346BFEE000AAD
:108DD80004E02B2A08BF0346B7EE000ADFED387A15
:108DE8001A46134612F8010BA0F13001CCB2092C37
:108DF8000AD807EE101AB8EEC77AF2EE046AA7EEA0
:108E0800A67AF0EE477AECE72E2816D1F2EE046A3D
:108E18001146B0EE666A0B4611F8012B303AD0B213
:108E280009280AD807EE102AB8EEC77A87EE267AFC
:108E380066EE866A77EE877AEDE71A7802F0DF0247
:108E4800452A35D15A782D2A02D10233012004E06F
:108E58002B2A14BF013302330020013B002213F8F0
:108E6800011F3039CCB2092C03D80A2404FB0212A2
:108E7800F5E7B2F59A7F28BF4FF49A721346B7EE1A
:108E8800007A072B05D9DFED0F6A083B27EE267A13
:108E9800F7E702F007032BB1F2EE046A27EE267A11
:108EA800013BF8E7F0EE476A20B1C7EE877A03E0A6
:108EB800F7EE006A67EEA67A20EE270A10BD00BF1B
:108EC8000000000020BCBE4C30B52DED028B87B0F1
:108ED800B0EE408A0C220021054603A80AF0BFFA2A
:108EE800B5EEC08ADFED2A7AF1EE10FACCBF38EE83
:108EF800278A38EE678ADFED277A28EE278A6946BF
:108F0800FDEEC87A17EE904A84EAE470A0EBE470AC
:108F180005F076FA002CACBF20232D2368468DF887
:108F28000C300AF0E0FA012807D130238DF80D3013
:108F38008DF80E308DF80F300CE0022805D1302363
:108F48008DF80D308DF80E3004E0032804BF30236F
:108F58008DF80D30694603A80AF0A8FA03A80AF0AC
:108F6800C2FA0338C4B2224603A928460AF0E8FA2E
:108F780000232B55284608490AF098FA03AB2846DF
:108F880019190AF093FA284607B0BDEC028B30BDD8
:108F98006F12033A00007A44A471010870B50646BE
:108FA80015460846B6FBF2F414B12046FFF7F6FF63
:108FB80005FB1464024B1B5D00F8013B70BD00BF4C
:108FC800A67101082DE9F04F814689B08A461646F8
:108FD8001C4600253178002900F0DD80252902D0C3
:108FE8000136484675E07278302A08BFB278A2F197
:108FF800300319BFB71C4FF0000BF71C4FF0010BE3
:10900800092B4FF0000819D8A2F13003D9B2092969
:1090180005D80A2202FB083817F8012BF4E7A2F159
:109028006103052B02D8A2F1570305E0A2F1410321
:10903800052B03D8A2F137030A2BEADD6C2A31D1BC
:109048003A78642A07F1010600F083800BD8252AB4
:109058003DD003D8002A00F09E80BBE7582A0CD0E8
:10906800632A19D0B6E7732A22D002D86E2A37D0DD
:10907800B0E7752A5CD0782AACD1271D2068A2F108
:10908800580462424FF01001624155E02CD9582A29
:1090980032D0632A2AD13E4648462178271DD04738
:1090A80001350FE0642A64D00ED9732A14D13E46E4
:1090B800236800934846514642460023FFF71FFEA7
:1090C800271D05443C4685E7252ADFD13E4648460C
:1090D8002521D04701357DE70AD86E2A06D13E46BC
:1090E800236804341D6075E7002A54D03E4671E7B2
:1090F800752A26D0782AF9D1A2F1580304F1040C74
:109108005A422068CDF80CC04FF010015A4105AB07
:10911800FFF7A2FDDDF80CC03E46644605AB0093A0
:109128004846514642465B46FFF7E9FD054451E78C
:109138002068271D0A21002205ABFFF7B4FD3C4635
:10914800ECE704F1040CCDF80CC020680A210022D9
:10915800DDE72068002804F1040708DA2D238DF8DC
:10916800143040420DF115030A210022E5E705AB52
:10917800FAE72068002804F1040C0ADA2D238DF898
:10918800143040420DF11503CDF80CC00A2100221D
:10919800BEE705ABF8E7284609B0BDE8F08F0EB486
:1091A8000FB505AB019053F8042B0649039301A8AA
:1091B800FFF708FF019B00221A7004B05DF804EB6A
:1091C80003B07047FD8C00080FB413B50B4904AB0E
:1091D80008680B4953F8042B09680193FFF7F2FE5E
:1091E8000446084B186805F0CDFF0028F9D0204642
:1091F80002B0BDE8104004B0704700BF5C08002012
:1092080058080020780E0020B0EEE06AF0EEC05A50
:10921800B4EEE56AF1EE10FAD4BFF0EE656AF0EE4E
:10922800466AF5EE406AF1EE10FA0BD0B4EEE56A44
:10923800F1EE10FA54BFF0EE657AF0EE467AC7EE1A
:10924800A66A01E0DFED1F6ADFED1F7A9FED1F7A46
:109258009FED1F5AA6EEA77ADFED1E7AE7EE267A73
:109268009FED1D7AA7EEA67ADFED1C7AE7EE267A47
:10927800F4EEC65AB1EE677ADFED197AA6EEA75A70
:10928800F7EE007AE5EE267AF1EE10FAC7EE277AC5
:10929800C8BF9FED147AF5EEC00AC8BF77EE677AAB
:1092A800F1EE10FA48BF9FED107AB5EEC00A48BF3C
:1092B80077EE677AF1EE10FA48BFF1EE677AB0EE12
:1092C800670A70470000000039094E3DE3B59EBEAD
:1092D80069A2163E88FA16BE45FE7FBFA7DFA8B46E
:1092E80099FB243FDB0FC93FDB0F4940FDEEC07AF5
:1092F80017EE903A2033402B43D8DFED237AB4EEB3
:10930800E70AF1EE10FA04DDDFED207A30EE670AA5
:10931800F3E7DFED1F7AB4EEE70AF1EE10FA04D5B1
:10932800DFED1A7A30EE270AF3E7DFED1A7AB4EEAA
:10933800E70AF1EE10FA04DD30EE670A37EEC00AEC
:109348000AE09FED157AB4EEC70AF1EE10FA44BFB1
:1093580030EE270A37EE400A60EE007ADFED0F6A3A
:109368009FED0F7AA7EEA67ADFED0E6AE7EE876A21
:109378009FED0D7AA7EEA67A20EE276AA6EE070AD9
:1093880070479FED060A7047DB0F4940DB0FC94065
:10939800DB0F49C0DB0FC93FDB0FC9BF000000006E
:1093A80092E741B99730083C15A82ABEDFED027A4A
:1093B80030EE270A9AE700BFDB0FC93F064B1A8831
:1093C80022EA0000904210B518801C4602D0012005
:1093D80005F078FE208810BD980E0020064B1A88EC
:1093E8001043904210B518801C4602D0012005F0A9
:1093F80069FE208810BD00BF980E0020024A9368BD
:1094080023EA000090607047401D0020024A9368DC
:1094180018439060704700BF401D002008B5104BEE
:109428001A780023D9B2914207D20E4951F8231075
:109438000968002008600133F4E7322005F0E8FDF0
:10944800094B1B685A0309D5084B9B685B0305D475
:1094580040F2DC50BDE8084005F0DABD08BD00BFA9
:1094680024260020F4250020382A0020401D002052
:109478002DE9F34106F020FF454A6F23137040F2AF
:10948800DC735380BE231371EF2382F8D83700238F
:1094980082F8D93719461646F25C0133514040F23A
:1094A800DC729342F8D13A4B83F8D917394B1A69D1
:1094B800120604D5384A5A6002F188325A600427E5
:1094C8000020013F17F0FF0750D0324B3422DA60FA
:1094D800002444B1002356F80480019305F02CF8C9
:1094E8000428EED117E005F027F80428E9D1294D22
:1094F8002B6943F002032B61284B6B612B6943F006
:1095080040032B6105F018F82B69042823F00203A7
:109518002B61DFD0D5E71F4D2B6943F001032B6189
:1095280004F1006303F57C331FFA88F21A8005F012
:1095380003F8042810D11A4B23440193019B4FEAE6
:109548001848A3F8008004F0F7FF2B69042823F0DB
:1095580001032B6105D0B4E72B6923F001032B61CC
:10956800AFE7043440F2DC739C42B2D1094A136974
:10957800042843F08003136102D104F058F910B9AC
:10958800052005F0B7FD06F083FE02B0BDE8F081C6
:10959800401D0020002002402301674500F0030819
:1095A80002F0030810B50E4C206805F07FFC206817
:1095B800047A002202FB02F3193B634303F6C41347
:1095C8005343192193FBF1F3064921F81230013274
:1095D800072AEFD10449BDE81040FDF70DBE00BFD2
:1095E800040F0020480E0020801E00202DE9F041C5
:1095F80004F01DF910B9042005F07CFDA74CA84D16
:1096080006F05AFEA74940F2DC72204609F01CFF1A
:1096180094F8A837022B84BF002384F8A83794F85D
:10962800A8274FF4CC7101FB02F303F538702344EB
:109638002044286093F84003022801FB024284BFBB
:10964800002083F8400392F84033974A13700C22A5
:1096580002FB0343954A03F2AA731360A26846F219
:10966800090313401BB94FF40050FFF7CFFEA3685E
:10967800D80703D54FF40050FFF7C0FEA36859047C
:1096880009D50820FFF7BAFE4FF40050FFF7B6FEE1
:109698000120FFF7B3FEA3681A0706D54FF4005060
:1096A800FFF7ACFE0120FFF7A9FEA3689B0402D5D3
:1096B8004020FFF7A3FE012284F8112294F8DE214E
:1096C800764B2AB193F8E22112B1002283F8E22105
:1096D800774B784E1E604FF0000C674604EB0C0386
:1096E800B3F8F2E14FEA5E0101F077314FEA9E03E9
:1096F80003F03333C1EB0E00C11A4FEADE0303F067
:109708001133CB1A03EB23131EF0010803F00F32B9
:109718004FF0FF0392FBF3F3C3EB032318BF0137AA
:10972800A2EB030318BFFFB2012B0ADD022B40F0A6
:10973800B280B8F1000F00F0AE801EF0BC0F00F050
:10974800AA800CF1080CBCF1200FC7D1013F012FF2
:1097580000F2A180FFF726FF302200215648574F1C
:1097680009F07DFE564BD5F800801F60554B00214F
:1097780008F18500C3F8008005F0D8FB524B80F053
:1097880001001870514B07F128021A60504B07F17D
:10979800D0021A6098F8000002F008FE4D4B94F8C9
:1097A800D601DFED4D6A07F196021A6064214B4B32
:1097B800C82211FB00225A6000229A60DA601A61FE
:1097C8005A619A61DA6183F8202083F82120444B9A
:1097D80007F12E021A602A68424B92ED1B7A02F2B8
:1097E80025111960404B02F2951119603F4B07F1A2
:1097F800080119603E4B1F603E4B07F1A20119603A
:1098080067EE266A3C4B07F1AC01B6EE007A1960A8
:1098180087EE267A39490E60B4F86411181D07EEF0
:10982800901AB4F86611F8EE677AC3ED027A07EE7B
:10983800901A92F86810197192F88410597194F876
:10984800E1111974F8EE677AB2F82211C3ED037AC0
:1098580007EE901A2A49F8EEE77A08605A6183ED14
:10986800077A9FED287A1A62C7EE277A02F170010B
:1098780099612549DF62BDE8F0419FED247A67EEE2
:10988800877AC1ED007A02F1740102F21D12596261
:109898009A6206F0FDBC04F021FE5BE7401D002043
:1098A800D80E002000F003087C250020040F0020BB
:1098B800342A0020C81E0020080E0020801E002028
:1098C8003C0E0020400E002005000020C819002092
:1098D8001C0D00205C290020DB0F4940482A00208D
:1098E800301A002088120020E4020020F026002010
:1098F800F4260020F8010020BC120020BC02002041
:10990800AC1A002000006144F40100204C3D0F44D3
:1099180008B5FFF7ADFDFFF769FE0120BDE8084077
:1099280005F0D0BB2DE9F04F2DED0A8B87B08346AB
:10993800039390F85030029101925BB1322BA8BF8B
:10994800322307EE903AB8EEE7BADFEDD67A87EE23
:109958008BBA01E09FEDD4BAD44BDFEDD5BA1B88A2
:10996800D44CDFF86493002B08BF012307EE903A2C
:10997800B8EEE79A238869EE2BBA13F0020F3BEE94
:109988002BBA8BEE8BBA26D0B9F90030B9F9022080
:1099980083EAE37182EAE270A1EBE371A0EBE27083
:1099A80088420546B8BF0D46B5F5E17F16DA88420C
:1099B800DFEDC1AA05DD002AD8BF524207EE902A82
:1099C80004E0002BD8BF5B4207EE903AF8EEE77A46
:1099D800C7EEAAAA04E0DFEDB9AA01E0F7EE00AAF3
:1099E800DFEDB69AB64A59464FF0000AB0EE69AABA
:1099F800B448B54D30F81A00B4F800E003B207EEE9
:109A0800903AF8EEE77AB5EE047A67EE877A35F998
:109A18001A309FEDAE7AFDEEE77A06EE903AF8EE50
:109A2800E77A1EF0030F5FFA8AF64FEA4A0767EEF5
:109A3800877AF8EEE66A6FD036EEA67A019BBDEE1D
:109A4800C77AC3F1000817EE105A454503DBAB424D
:109A5800A8BF2B4698469E4D039B7D5F9FED9D5A60
:109A6800C5EB080833F91A509BF81C30454407EE3B
:109A7800105A0AEE103A9BF80830B8EEC76A07EE9B
:109A8800103AB8EE477AB8EE4AAA26EE077AF1EE0F
:109A9800045A27EE057A6AEE255ABDEEC77A17EE04
:109AA800108AB1EE657ABDEEC7AA1AEE103A98454B
:109AB80008DBBDEEE5AA1AEE103A4345A8BF4346B7
:109AC8000AEE103A844D05EB8A0595ED007AA6EE6C
:109AD8002B7ABBEE0E6AB4EEC67AF1EE10FAB8EE47
:109AE800CAAA09D4B3EE0E6AB4EE467AF1EE10FAB9
:109AF800C8BFB0EE467A01E0B0EE467A85ED007A4E
:109B08009BF8123009EE903AF8EE699A27EE297A16
:109B1800DFED729A67EE299A1EF0010F50D100B25C
:109B28000028B8BF4042B0F5206F02DD0020106069
:109B380025E09FED6B6A4B7826EE867A06EE103AA2
:109B4800B8EE466A87EE066A92ED007A36EE676AE4
:109B5800A6EE2B7A9FED636AB4EEC67AF1EE10FAA0
:109B680009D49FED616AB4EE467AF1EE10FAC8BFE7
:109B7800B0EE467A01E0B0EE467A82ED007ACB7A12
:109B880092ED007A08EE103AB8EE488A1EF0020FFD
:109B980028EE077A9FED558A27EE088A14D076EECC
:109BA800CA6AB0EE4A7AAAEEA67A38EE698AF0EE68
:109BB800476AB0EE697AAAEE887AB0EE478A03E07F
:109BC800B0EE698AF0EE4A6A49489FED4A6A1AF887
:109BD8000030059207EE103AB8EEC77A4FEA8A08C5
:109BE80027EE677A051D4544E7EE066A049195ED70
:109BF800007AC5ED007A37EEC77A00F10C0587EEDA
:109C08002B7A454414301AF80030D5ED007A37EE37
:109C1800677A08EE903AEBEE077AF8EEE88AC5ED37
:109C2800007A67EEA87ADFED348A344D67EEA88AA9
:109C380036EE880AB0EE66CA30EE680A09F01EFEF3
:109C4800E85320880499059A10F4006F08D02C482E
:109C58000078400704D53046FEF7E8FE059A0499D7
:109C68002848294FFDEECC6AFDEEC87AF1EE688AE5
:109C780016EE903A17EE906AFDEEE88A48F8003042
:109C880048F8076018EE903A204E049648F80630D7
:109C9800043201318046BAF1000F3BD14FF0010A7E
:109CA800A6E600BF83F9223EAF4C593C880E00203F
:109CB800BD378635980E00200000E1430000000003
:109CC800EC120020C20E00203C190020CDCC4C40E4
:109CD800F40E00206F12033CF81200200AD7A33DAF
:109CE8000000A043000040C3000040430AD7233CC3
:109CF80000130020A69B443BF7CC9238841900201F
:109D0800942A00208C19002098190020A4190020FA
:109D180000803B45BDEEC99A5FED037A9BF853601E
:109D28009049DFF864A219EE103A23F0030309EE14
:109D3800103A029BB8EEC99A9B7989EE279AB5EE3C
:109D4800000A002E6DD0B9F904209BF80300002A00
:109D5800B8BF52425A43844B92FBF3F364336422F4
:109D6800434393FBF2F308EE903AB1F9043007EE5F
:109D7800903AF8EEE77AF8EEE88A27EE800A09F0DA
:109D88007DFD07EE900AF8EEE77AB9F9043067EE40
:109D9800A88ADFED767AC8EEA78A80EAE072A2EB9D
:109DA800E072B2F5207F07EE903AF8EEE77A77EEA8
:109DB800E88A05DC83EAE372A2EBE372642A03DD36
:109DC8000023CAF80830A2E003EB83031A019BF8CA
:109DD800033092FBF3F31B1A07EE903AF8EEE77A9A
:109DE800DAF8083067EE897AFDEEE77A17EE902AFE
:109DF8001A441346B2F57A5F5D4AA8BF4FF47A5306
:109E08009342B8BF1346CAF808307D2293FBF2F399
:109E18009BF80D2053439B1107EE903AB8EEE78A62
:109E280075E0544A5B00B2F90490283303FB09F942
:109E3800B1F9043007EE903AF8EEE77A4FEA69197B
:109E480027EE800A09F01AFDB9F1000FC0EB0900EE
:109E580007EE900AB8BFC9F10009B9F1320FB8EEA0
:109E6800E77A02DDCAF808601BE09BF80D3007EEC0
:109E7800903AF8EE677ADAF8083067EE277A67EEF4
:109E8800897AFDEEE77A17EE902A13443A4A93420C
:109E9800A8BF1346394A9342ACBFCAF80830CAF87B
:109EA8000820DAF808305B13B3F5807FA8BF4FF4B9
:109EB80080736FF0FF029342B8BF134607EE903AE3
:109EC800B8EEE78AFDEEC77A9BF8032017EE903AC2
:109ED80053439B1107EE903A294B1B78032BF8EE5E
:109EE800E78A14D9BBF84E20B2F5FA7F0FD2FDEEFF
:109EF800E87A534217EE901A994204DB914217EE22
:109F0800903AA8BF134607EE903AF8EEE78A78EE43
:109F1800887AFDEEE77ACDED017ABDF80430AB80A2
:109F28001BB200EE103AB8EEC00A09F0A7FC23886D
:109F3800A8801A0506D5134B1B785B0702D50220AB
:109F4800FEF774FDFDEEE88ABDEEC88A049AC8EDF6
:109F5800028A002387ED028A936007B0BDEC0A8B62
:109F6800BDE8F08FC20E00200CFEFFFF0000A042EB
:109F780080C1FFFF3C190020FEFFFF0F020000F028
:109F880024260020942A0020541900202DE9F04F9F
:109F980087B000260593BA4B0491B3F90270B3F960
:109FA80000300292002FB8BF7F42002BB8BF5B423F
:109FB8009F42B8BF1F46B7F5FA7F8046A8BF4FF447
:109FC800FA770090B3460196B2463446AD4B1988ED
:109FD80011F003023DD0AA4B33F91400029B400054
:109FE8005B4298424FEA440503DB029B8342A8BFC9
:109FF8000346A5482D5E05985B1B30F914501D4497
:10A0080098F8083064206B4393FBF0F398F81C0031
:10A018006FF0040A0AFB00FA534504DB00EB800AE0
:10A028009A45A8BF9A46994850F824302B4442F2E2
:10A038001075AB42A8BF2B46954DAB42B8BF2B4617
:10A0480040F8243098F8120043431B13012A019367
:10A0580038D08B4B8F4833F914B0009B50F824E06C
:10A0680093F801C08C4B33F9145085EAE573A3EBE0
:10A07800E573B3F5206F4FEA840616DC0BEB8B0310
:10A088001A0192FBFCF3042295FBF2F55D1BAE442A
:10A09800BEF57A5FA8BF4FF47A5E804B9E45ACBF91
:10A0A80040F824E040F8243002E0002340F824304F
:10A0B80083597D2693FBF6F6009BDB7A7343402693
:10A0C80093FBF6F6880711D50198C7F5FA7307FBD5
:10A0D8000BF907FB06F54FF4FA7103FB0A9903FB2A
:10A0E800005599FBF1F295FBF1F505E0C9074DBF65
:10A0F800019D35465A465246630069490393664BAB
:10A10800605C33F814E020310FFA8EF34FF0040C42
:10A1180093FBFCF909FB00F06FF04F0990FBF9F98C
:10A12800914431F9142021F814E098F850109B1A42
:10A1380093FBFCF379B107EE903A5A485A4BB8EEC4
:10A14800E70AD3ED000A00EBC400FEF709FEFDEEB6
:10A15800C07A17EE903A554A554912F804C0039848
:10A1680003EB430309EB05020CFB03F34FF0200C50
:10A1780093FBFCF3D21A4252424A1288120508D5C0
:10A188004C4A1278500704D520460393FEF74EFC3C
:10A19800039B494A49494A4841F824905B4242F89E
:10A1A8002430009B40F82450013300930D4681462B
:10A1B8000CB901240AE7324B3648B3F90410049B62
:10A1C80086689B790F335B004B435B113249002B48
:10A1D8004FF00404B1F9041091FBF4F1A3EB010171
:10A1E800B8BF5B42322B98F80D400BDC354B04FBB3
:10A1F8000164A342A8BF2346334CA342ACBF83608B
:10A20800846001E000238360304B98F803401B789A
:10A218004C43032B4FEAA4140CD9B8F84E30B3F5CD
:10A22800FA7F07D259428C4203DB9C42A8BF1C46E6
:10A2380000E00C46866846F34F36B6F5807F6FF02F
:10A24800FF03A8BF4FF480769E42B8BF1E46184B46
:10A25800A11999800B4B1B88190508D5154B1B783C
:10A268005B0704D502200092FEF7E0FB009AAC6081
:10A278000023C9F80860936007B0BDE8F08F00BFFD
:10A288003C190020980E0020F40E0020181300201E
:10A29800F0D8FFFF54190020C20E002080C1FFFF34
:10A2A800001300206C1900205019002014130020FE
:10A2B80084190020942A0020A41900208C19002059
:10A2C80098190020FEFFFF0F020000F0242600204E
:10A2D8002DE9F04F87B080460493A94B03911C8861
:10A2E800029204F00204A4B294B1A64BB3F902405E
:10A2F800B3F90030002CB8BF6442002BB8BF5B42F2
:10A308009C42B8BF1C46B4F5007FA8BF4FF4007448
:10A31800C24600259B4B9C4E33F915E09B4B33F806
:10A3280015300193BDF9040056F8253080EAE0772E
:10A33800A7EBE0770421B7F5206F90FBF1F189B224
:10A348004FEA450B4FEA4E0C0AB24FEA85090FDC7B
:10A35800C2EB0C021344B3F57A5FA8BF4FF47A53EB
:10A368008B4A9342ACBF46F8253046F8252002E0D8
:10A37800002346F8253056F809709AF80B30804AC1
:10A38800FF115F4312889AF80130960703FB0CF31C
:10A398004FEAA7174FEAA31340D0029A4FEA4E0E8E
:10A3A8005242964503DB029A7245A8BF7246794E1F
:10A3B800DFF814E23BF90660961B049A32F915207F
:10A3C800164459F80E2042F2107C32446245A8BF68
:10A3D8006246DFF8F8C16245B8BF624649F80E2008
:10A3E80098F808E00EFB06F698F81CE00EEB8E0EC7
:10A3F800F611CEF1000C664503DB7645A8BF76461C
:10A40800B44698F8126072431213BF1ACCEB0303D8
:10A418006743634302EB67270CEB63235E4A565D91
:10A42800243211FB06F6A3EBA6163BF9023098F886
:10A438005010C01A042390FBF3F0BDF804302BF839
:10A44800023079B107EE900A544B5548D3ED000A13
:10A45800B8EEE70A00EBC500FEF782FCFDEEC07A15
:10A4680017EE900A4F4B504A5B5D00EB4000584393
:10A478004311F119C91A2BF802104149088810F440
:10A48800006F8B460AD049490978490706D52846FE
:10A4980005920193FEF7CAFA059A019B444845497B
:10A4A80049F80060444E49F801705B4249F80630AB
:10A4B8000AF1010A074689460DB901252AE7314BF9
:10A4C80098F80D00B3F90410039B9B790F335B00D8
:10A4D8004B435B112D49002BB1F904104FF00405D3
:10A4E80091FBF5F52849A3EB0505B8BF5B42322B74
:10A4F8008C680BDC314B00FB05408342A8BF034648
:10A508002F488342ACBF8B60886001E000238B60DA
:10A5180098F803305D432B4B1B78032B4FEAA515A6
:10A528000CD9B8F84E30B3F5FA7F07D258428542B5
:10A5380003DB9D42A8BF1D4600E005468C6844F336
:10A548004F34B4F5807F6FF0FF03A8BF4FF48074D9
:10A558009C42B8BF1C462B199380BBF800301A05E3
:10A5680006D5124B1B785B0702D50220FEF75EFA70
:10A578000023BD60C9F80840B36007B0BDE8F08F9C
:10A58800980E00203C19002054190020C20E00200B
:10A5980080C1FFFFF40E0020001300205019002096
:10A5A8006C1900201413002084190020942A00201C
:10A5B8008C19002098190020A4190020FEFFFF0F15
:10A5C800020000F02426002018130020F0D8FFFF16
:10A5D8002DE9F04F2DED028B85B000260293A44B98
:10A5E8000192B3F90270B3F900300090002FB8BFA0
:10A5F8007F42002BB8BF5B429F42B8BF1F46B7F5EA
:10A60800FA7F8346A8BF4FF4FA77B046B146B24600
:10A618003446984B1B8813F0030045D0022C43D0D6
:10A62800934A32F91410019A4900524291424FEA72
:10A63800440503DB019A8A42A8BF0A468E4935F9C8
:10A64800019002999BF81C5031F91410C9EB0202D1
:10A6580002EB01099BF8081001FB09F2642192FB47
:10A66800F1F16FF0040202FB05FA514505DB05EB39
:10A6780085029142A8BF11468A46804D804A55F806
:10A68800241042F2107E49447145A8BF7146914298
:10A698009BF81290B8BF114609FB01F9012845F84B
:10A6A80024104FEA293942D0764D714935F91450B2
:10A6B800009A754831F9148092F801E050F8242086
:10A6C80085EAE576A6EBE576B6F5206F4FEA8401D4
:10A6D80020DC022C18D008EB8800000190FBFEFE5D
:10A6E800042095FBF0F5C5EB0E0E02EB0E0CBCF545
:10A6F8007A5F6548654DA8BF4FF47A5CAC45ACBF3E
:10A7080041F800C00D5007E088EAE876A6EBE87645
:10A71800642EE0DD002545505B48009A09587D26E7
:10A7280091FBF6F6D17A7143402691FBF6F69D0728
:10A7380012D5022C10D0C7F5FA7307FB06F507FBF4
:10A7480008F103FB0A114FF4FA7003FB095391FB5C
:10A75800F0F193FBF0F508E0D80704D5022C02D0FD
:10A768004D46514601E035464146464B33F9140003
:10A77800042390FBF3F34648205C022C03FB00F310
:10A788006FF04F0093FBF0F30B444FEA440C08EED4
:10A79800103A0ED13F4B4048D3ED000ACDF80CC01B
:10A7A800B8EEC80A1E21FEF7DBFADDF80CC0BDEED4
:10A7B800C08A344B39493CF803003CF901302CF885
:10A7C80001009BF850100FFA80FEC3EB0E034FF008
:10A7D800040E93FBFEF399B107EE903A30482D4BE7
:10A7E800CDF80CC0B8EEE70AD3ED000A00EBC400C0
:10A7F800FEF7B6FAFDEEC07ADDF80CC017EE903A17
:10A808002849294811F804E018EE102A03EB4303FD
:10A8180051190EFB03F34FF0200E93FBFEF3C91AF8
:10A828002CF8001013490988090508D51F4909782B
:10A838004A0704D5E0B20393FEF7F8F8039B1C49D6
:10A8480018EE102A41F824201A4941F824501A49D0
:10A858005B4241F82430009B01340133032C009300
:10A868007FF4D7AE05B0BDEC028BBDE8F08F00BF1A
:10A878003C190020980E0020F40E00201813002028
:10A88800F0D8FFFFC20E00205419002080C1FFFF3E
:10A898000013002050190020481900202813002018
:10A8A8006C1900201413002084190020942A002019
:10A8B8008C19002098190020A4190020284B294A37
:10A8C8001B68126810B51A60274A116859605168E8
:10A8D8009268DA60254A996011681961516892682E
:10A8E8009A61234A59611168D961516892685A621C
:10A8F800204A196211881985518859859188D2880A
:10A90800DA851D4A99851188198651885986928851
:10A918009A861A4A1188D9865188198719469288C1
:10A9280021F83A2F164A10780022824206DA154C8E
:10A9380034F8124021F8024F0132F6E7124A128821
:10A94800A3F86420114A1288A3F86620104A1288D6
:10A95800A3F868200F4A5289A3F85E2010BD00BFF3
:10A96800D8270020782A00208C1900209819002068
:10A97800A41900203C190020C20E0020BC0E0020A3
:10A9880024260020DC0E00204C1100206C0E002034
:10A99800FA0E0020C80E0020A0F17D03012B70B52F
:10A9A80004460D460A4E05D830687D2104F0F3FBB5
:10A9B80084F020043068214604F0EDFB35B12B8883
:10A9C8001C4404EB142404F0FF042C8070BD00BF69
:10A9D800A407002010B50A4C5E280146206805D15E
:10A9E8005D2104F0D8FB20683E2105E05D2903D1F4
:10A9F80004F0D1FB20683D21BDE8104004F0CBBB3A
:10AA0800301300202DE9F8430E4B93E880030546E8
:10AA18000E460024B44213DA7B1933F9140008EB0C
:10AA2800050333F9142009EB050333F914301344F3
:10AA3800022293FBF2F3C01A03F0DDFA0134E9E7CE
:10AA4800BDE8F883D827002010B5134B93F8D0370A
:10AA5800012B014619D1114B114C1878421CD2B266
:10AA68001A70120644BF00221A700E4A1B78127818
:10AA78002154934236BFC2F180029B1A9B183F2B88
:10AA880009D9BDE8104002F001BB074BBDE81040F2
:10AA9800186804F080BB10BD401D0020F81B002082
:10AAA800FA1B0020F91B0020C02700207FB5264C88
:10AAB800264E274D2749284A284B20B12848008888
:10AAC800B0F5805F32D230881F4E91F8201012788E
:10AAD800ADF8040028788DF80600351D8DF80710AC
:10AAE8008DF808201B788DF8093001A82946062220
:10AAF80008F09AFC30B30198BDF808307060AB805C
:10AB08005320FFF7A1FFA08803F065FAA07903F0AE
:10AB180062FAE3790193237A029301A8637A039393
:10AB280003F0C8F90E4B00221A800BE03088A08091
:10AB380091F82010287812781B78A071E1712272A0
:10AB48006372DDE704B070BD30130020980E00205A
:10AB5800A81A0020482A00206C0D0020D20D0020E1
:10AB68004C2900200A4A138801331380094A1368C4
:10AB780001331360084A138801339BB2202B01BFAD
:10AB880000231380054A138808BF013313807047D8
:10AB98004C29002034290020382900203A29002097
:10ABA80038B5294B1B78083B012B05460C464AD87B
:10ABB8004520FFF749FF2846FFF746FF0E2D33D003
:10ABC80003D83DB10D2D07D038BD142D20D0FF2D51
:10ABD80032D038BD20682BE0637820789BB180F0B4
:10ABE8008000FFF731FFA568E8B2FFF72DFFC5F336
:10ABF8000720FFF729FFC5F30740FFF725FF280EB9
:10AC0800FFF722FF04E0FFF71FFF606803F0F3F986
:10AC18002078FFF719FF606803F0EDF92489E0B2A6
:10AC2800FFF712FF200A0BE0206803F0D4F96068F0
:10AC3800BDE8384003F0CFB9044803F0E0F900203C
:10AC4800BDE8384000E738BDBE270020CB710108B9
:10AC58002DE9F04FB44BB54F1A8889B01C46002A2D
:10AC680040F09680B7F8CE07B14D42F20103C41AFE
:10AC780060426041FFF71AFFFFF720FE2C68492069
:10AC8800FFF7E2FEAB4B2646186803F0A4F956F826
:10AC9800040B03F0A0F9304603F0D3FB04F11000D5
:10ACA80003F0CFFB04F11C094FF01008A24E01235A
:10ACB800326803FA08F3134203D0D9F8000003F00E
:10ACC8009AF908F10108B8F1130F09F10409EDD157
:10ACD80004F1280003F0A5FBB7F84031B4F92E00C1
:10ACE800C01A03F078F93368D90408D5934BB4F83F
:10ACF80064001B88181AC0F30D0003F06CF9336860
:10AD08009A0403D5B4F8660003F065F933681B04A8
:10AD180003D5B4F8680003F05EF904F13000A046EA
:10AD280003F07FFB04F1360003F07BFBB7F84031FA
:10AD380038F93C0FC01A03F04EF90127804B1B78F5
:10AD48009F4208DA38F9020FB4F93C30C01A03F010
:10AD580052F90137F2E73368980505D5B4F95E0072
:10AD6800A0F2DC5003F047F92A6876486A60AA60C6
:10AD7800121A9110744A4A43531C032293FBF2F2AD
:10AD880002EB42029A1A6C2303FB02032B6070E168
:10AD98006E4B6F4A1B6811688B4206D008A90020C9
:10ADA80041F8203D1360FFF7FBFE97F8CE17238884
:10ADB80097F8CF070B44013BB3FBF0F200FB1233CB
:10ADC8008B4280F056815A4E0120FFF76FFEFFF745
:10ADD80075FD5020D6F800807768FFF735FEB26819
:10ADE800336810681B68726803441068A3EB40005E
:10ADF80003F001F97A68D8F804309B1A0093BA680E
:10AE0800D8F808309B1A0193FA68D8F80C306846CD
:10AE18009B1A029303F015FB3A69D8F810309B1A75
:10AE280000937A69D8F814309B1A0193D8F818302F
:10AE3800BA6968469B1A029303F03CF808F11C0AA9
:10AE480007F11C0510243C4901230A68A34013425A
:10AE5800894605D0DAF800002B68C01A03F0CBF851
:10AE68000134132C0AF1040A05F10405EBD108F1A9
:10AE7800260007F12601002330F9022F31F9024F8D
:10AE8800121B4DF823200133042BF5D10322002592
:10AE98005DF82230AD00EDB26BB103F108010F2966
:10AEA80002D845F0010506E08033FF2B94BF45F03A
:10AEB800020545F0030512F1FF32E9D22846FFF7F3
:10AEC800C3FD0024EB46A24605F00303022B16D06F
:10AED800032B1DD0012B4ED1BAF1000F05D1DBF8A1
:10AEE80000402401E4B29A4645E0DBF8000000F097
:10AEF8000F002043FFF7A8FD4FF0000A3BE0BAF12E
:10AF0800000F0CD0DBF80000C0F3031020432CE046
:10AF1800BAF1000F1ED19BF80100FFF795FD9BF8D1
:10AF28000000FFF791FD26E038290020401D002091
:10AF3800D8270020342900202C2900202829002087
:10AF480024260020E427002013DA4B68402900203B
:10AF58003C290020DBF80000C0F303302043FFF752
:10AF680073FDDBF80000C0F30710FFF76DFDDBF899
:10AF780000402401E4B20BF1040B04AB9B454FEAFB
:10AF88009505A1D1BAF1010F02D12046FFF75CFD6A
:10AF9800D9F8003013F480541FBFB8F86420B7F80C
:10AFA8006410521A009218BF012499040AD508AAFD
:10AFB80002EB8401B7F86600B8F86620121A41F867
:10AFC800202C01341A040BD508AB03EB8402B7F824
:10AFD8006810B8F868305B1A42F8203C013400E089
:10AFE800DCB1012C03D1009803F005F815E0631ECD
:10AFF80000205DF823204000C0B20AB140F00100F3
:10B00800013BF6D5FFF720FD00255DF8250008B1C6
:10B0180002F0F1FF0135A542F7DB30200321FFF7ED
:10B02800F1FC36200321FFF7EDFC144B3C20197886
:10B03800FFF7E8FCD9F800309B0506D5B8F95E00A3
:10B04800B7F95E30C01A02F0D6FF32680C48736850
:10B058007260121A91100B4AB3604A43531C0322C0
:10B0680093FBF2F202EB42029A1A6C2303FB0203EF
:10B07800336002F00DFF09B0BDE8F08F24260020F0
:10B08800E427002013DA4B682DE9F84F0C9E3A4C60
:10B09800C2EB030B0B9BF61A6368002914BF4FF031
:10B0A800060A4FF0040A01330546904613D1236877
:10B0B80053455ED2314A324852F82320032B98BFB9
:10B0C800294603F007F86368013363602D4B0022BB
:10B0D80005469A7213E0002511E02B4A1278954232
:10B0E80040DA0B9BE3B109FB06F2995C01228A4026
:10B0F800264909680A4213D1636801336360D4F8AA
:10B1080004900A9B1C4F9945E7DB2BD10A20FFF7D7
:10B118009BFC3B6801333B604FF0FF337B6021E0D1
:10B12800184A917A21B12C20FFF78EFC013501E0F5
:10B1380001219172226809FB0BF308EB030752B94E
:10B1480058F8030002F05BFF97F904104B1C054404
:10B15800D2D00F4802E03A440E48117902F0BAFF03
:10B168000544C9E7206850452CBF00200120BDE8F0
:10B17800F88F0020BDE8F88F4429002014500108FA
:10B18800D671010830130020090100202C29002065
:10B19800E57101085D71010830B585B004AC002582
:10B1A80024F8025D0091ADF8060021461020FFF753
:10B1B800F3FB9DF806002146FFF7EEFB9DF807001C
:10B1C8002146FFF7E9FB9DF800002146FFF7E4FB65
:10B1D8009DF801002146FFF7DFFB9DF8020021469C
:10B1E800FFF7DAFB9DF803002146FFF7D5FB9DF832
:10B1F8000E00C043C0B22946FFF7CEFB05B030BDF4
:10B2080010B5054C206803F0C3FF18B1206803F09F
:10B21800BCFFF6E710BD00BF7C07002030B5002852
:10B22800104C114AB8BF40423C2590FBF2F304FB96
:10B23800030068430D4D90FBF2F22D682D7B25B974
:10B2480003EB830303EB830301E0C3EB031302EB7C
:10B2580083030B8004FB02024FF47A7392FBF3F230
:10B268004A8030BD806967FF8096980034070020C7
:10B2780010B50446C0B2FFF7ADFBC4F30720BDE824
:10B288001040FFF7A7BB024B5E21186803F083BF8D
:10B298003013002038B5064C05465E21206803F0BF
:10B2A8007AFF20682946BDE8384003F074BF00BF24
:10B2B80030130020026BC168034610B5406942B1E3
:10B2C8001A6C8C1A013A005D08BF0A46C0B21A64AB
:10B2D80010BD1A6A805C01328A4228BF0022C0B2BF
:10B2E8001A6210BD436B13B190F844007047836A2B
:10B2F800406A1B1A584258417047036B13B15B6888
:10B30800016C01E0C369016A8B423CBFC2689B18AB
:10B31800581AC0B27047836A8169426B1944D16078
:10B32800416A99429DBF0169CB1A5360CB1A96BFF7
:10B338000023536083624FF0000380F844301368A1
:10B3480088BF816243F0010313607047436A8269D2
:10B35800D154436A02690133934228BF00234362F0
:10B36800436B1BB11B68DB0705D4D4E7026D136878
:10B3780043F08003136070474171F9F729BF81607A
:10B38800F9F726BF026D036B70B50446D5699BB902
:10B39800A90611D5C36A1BB1908C80B298470BE0FF
:10B3A800E169928C40694E1CD2B2E6614254E1696F
:10B3B800E268914228BFE361616BA1B92A0612D500
:10B3C800636AA26A9A42236D09D0501CA669A062DA
:10B3D800B25C1A852369984205D3A16203E01A6812
:10B3E80022F080021A602B0742BF236D08221A62DE
:10B3F80070BD0D4B0D484FF400525A600C4A11684D
:10B408004FF6FE730B401360426B11684FF6FE73E4
:10B418000B401360426A836A9A4200D07BE701239B
:10B4280080F84430704700BF00000240A41B002091
:10B43800440002402DE9F0471E469F4B8CB09842CD
:10B44800894690469DF850507ED19C4B9C4A1A6084
:10B458009C4A5A6102F580729A614FF48072DA60F0
:10B468001A61994A1A63143A5A63A2F54842203A73
:10B47800DA6404329A64C3F808801865934B9A69B1
:10B4880042F480429A615A6942F001025A610223E9
:10B498008DF80830032315F0010A8DF809304FF0B4
:10B4A80000038DF80A3014BF022301232C078DF8FE
:10B4B8000B3017D5864C402701978AF001038DF889
:10B4C8000A30236A23F070632362236A43F0E0633F
:10B4D8002362204601A9FAF78BFFBAF1000F23D1A6
:10B4E800A76121E0B0070ED50CA9402341F82C3DF7
:10B4F8007748036A23F070630362036A43F0E063EA
:10B508000362FAF775FFF1070ED50CA9802341F8FD
:10B518002C3D6F48036A23F070430362036A43F0CB
:10B52800E0430362FAF764FF0E238DF8003000222F
:10B53800012368468DF801308DF802208DF803301C
:10B548005E4C02F07FFE04E1624B984270D1624B80
:10B558005B4A1A604FF48072DA601A615F4A5A6176
:10B5680002F580729A61594AC3F808801865D36950
:10B5780043F40033D36102238DF80830032315F018
:10B58800010A8DF809304FF000038DF80A3014BF16
:10B59800022301232A078DF80B3017D54C4C0827B6
:10B5A80001978AF001038DF80A30236A23F4704367
:10B5B8002362236A43F4E0432362204601A9FAF791
:10B5C80017FFBAF1000F23D1A76121E0B3070ED509
:10B5D8000CA9082341F82C3D3D48036A23F4704325
:10B5E8000362036A43F4E0430362FAF701FFF707D3
:10B5F8000ED50CA9102341F82C3D3548036A23F4D5
:10B6080070230362036A43F4E0230362FAF7F0FE4F
:10B6180026238DF800300022012368468DF801307A
:10B628008DF802208DF803302B4C02F00BFE90E0D1
:10B638002B4B984240F00E812A4B214A1A604FF456
:10B648008072DA601A61284A5A6102F580729A613A
:10B658001E4AC3F808801865D36943F48023D36170
:10B6680002238DF80830032315F0010A8DF80930FC
:10B678004FF000038DF80A3014BF022301232C0772
:10B688008DF80B3032D5124C4FF4806701978AF051
:10B6980001038DF80A30636A23F470636362636A96
:10B6A80043F4E0636362204601A9FAF7A1FEBAF108
:10B6B800000F3FD1A7613DE000380140A41B0020E6
:10B6C8002C5001083C130020580002400010024092
:10B6D8000004004800440040501B00203C15002096
:10B6E80000480040FC1A00203C170020B0070FD586
:10B6F8000CA94FF4806341F82C3D5848436A23F461
:10B7080070634362436A43F4E0634362FAF770FE8E
:10B71800F1070FD50CA94FF4006341F82C3D4F48B1
:10B72800436A23F470434362436A43F4E043436249
:10B73800FAF75EFE27238DF80030002201236846C1
:10B748008DF801308DF802208DF8033002F07AFD73
:10B75800434CC4F82C900027012384F84430276216
:10B76800E761A76267626671C4F80880A571204620
:10B77800F9F72EFDF20734D5236B002B2AD001A848
:10B78800FAF7D2FBE36C01934FF480530A938023BA
:10B798000693E368ADF8103020230993206B6369A2
:10B7A80002930B970597079708970397FAF7E7FB14
:10B7B80001A9206BFAF7C5FB236B216D1A6842F0CB
:10B7C80001021A608A6842F040028A605B689BB294
:10B7D800236406E0236D20221A621A6842F02002D0
:10B7E8001A60B3072FD5636B43B301A8FAF79CFB24
:10B7F800A36C01934FF480530A9380230693236923
:10B80800ADF8103000251023606B03930B95059558
:10B81800079508950995FAF7B2FB606B01A9FAF745
:10B8280090FB636B1A6842F002021A60226D5D6039
:10B838005D60936843F08003936004E0226D1368B1
:10B8480043F080031360226D136843F00103136013
:10B85800204600E000200CB0BDE8F0870004004856
:10B86800FC1A00202DE9F04F2DED028B85B08146A2
:10B8780003938A4B02921B889D0737D5109B8848F3
:10B88800DC89B0F900301B1B03F2F31540F2E632F5
:10B89800954203D8002BB8BF5B4201E04FF4FA731E
:10B8A800B0F90220121B02F2F31440F2E63084428F
:10B8B80003D8002AB8BF524201E04FF4FA7293420B
:10B8C800B8BF1346C3F5FA73052293FBF2F30A22B5
:10B8D800643B534399F81C20D2105343642293FBD2
:10B8E800F2F3134423EAE373DBB200E0642300932A
:10B8F800CB1C0193C8460025019B6A4813F8011F19
:10B908000193022D4FEA450A06D1B0F9040001F16E
:10B918001B04444363112DE030F91520029B5000AD
:10B928005B42984203DB029B8342A8BF03465E4802
:10B9380030F90A40039830F915001B1B1844574B7F
:10B948001E88F40712D401F11B035A43B1074FEACA
:10B9580022130FD599F812409DF9001044434C4327
:10B96800642294FBF2F203EB221303E099F8083007
:10B9780043431B114D4A042432F90A2092FBF4F484
:10B988001C1B484B03F108026421AF5C98F80120A6
:10B9980062437A43022D92FBF1F24FEAE21208EE7B
:10B9A800102A0AD1B8EEC80A03F10C001E21D3ED03
:10B9B800050AFDF7D5F9BDEEC08A3A4A3C4B98F81E
:10B9C8000B601B8802F1180E03FB04F05EF82510CB
:10B9D800C01206FB0016B6F5001F3649A8BF4FF483
:10B9E800001602F124008E42B8BF0E4650F825100A
:10B9F80040F82540611A1B094FF6FF70B0FBF3F3BE
:10BA08004B4399F850104EF825604FEA850B761392
:10BA18009B1179B107EE903A02F13000B8EEE70ACF
:10BA280000EBC500D2ED050AFDF79AF9FDEEC07AE4
:10BA380017EE903A98F815101F4A03EB43034B434F
:10BA48005F43642397FBF3F718EE103A3F12334431
:10BA58003B4422F80A30114B1B881A0506D5174BB0
:10BA68001B785B0702D5E8B2FCF7E0FF144B18EE31
:10BA7800102A01354BF8032003F10C021833032D6B
:10BA88004BF802604BF8037008F101087FF434AFFB
:10BA980005B0BDEC028BBDE8F08F00BF980E00200A
:10BAA800821C00203C190020F40E0020C20E002049
:10BAB800000F00200000E0FF84190020942A0020D5
:10BAC8008C1900202DE9F04F2DED0A8B97B011F05D
:10BAD800FD0806460191A94C06D0A94B1B689A0798
:10BAE80000F1B08000F041BCA36FA648DFF8949243
:10BAF80098470028F1D0A44F94F888204846494632
:10BB0800FAF7B2FC3B8804F1D802002B70D0D4F8C5
:10BB18008C301B7808EE103A04F1900A04F19C0569
:10BB2800B7F800B039F91800BBF57A7F02BF0023D7
:10BB3800CAF800302B61DAF800300344CAF8003044
:10BB48002B6907EE900A0133012B4FEA4801F8EE02
:10BB5800E77A2B6106D10023C5ED017AC5ED007A9D
:10BB6800AB601BE0D5ED006A07EE103A37EEE66AE7
:10BB7800B8EEC77A86EE077A36EE877AD5ED026A8E
:10BB880085ED017A77EEC77A85ED007AE6EE276AC9
:10BB9800F0EE667AC5ED036AC5ED026A0023BBF1D3
:10BBA800010F29F8013053522DD12B690392012B33
:10BBB800C3BF03F1FF3300EE103AD5ED037A9FEDD2
:10BBC800730A0291C4BFB8EEC00A87EE800A07F074
:10BBD800FDFE0299039A18EE103A5BB1F8EEC87AA6
:10BBE800B4EEE70AF1EE10FA04DD4FF47A733B8005
:10BBF80000231CE0DAF800304FF47A7003F5FA738A
:10BC080093FBF0F3535208F10108B8F1030F0AF15E
:10BC1800040A05F1140583D1BBF1010F04D158467C
:10BC2800029203F02DFA029A3B88013BDFE739F8CC
:10BC3800131032F81300091A29F813100133032BD3
:10BC4800F5D14AE7019B002B00F08F8394F8DE7052
:10BC58004A4D6FB1012F40F0808305F59470D5ED02
:10BC6800486A95ED497A05F59A730021804613E1F3
:10BC780003F0B2F9D5F8E8309FED457AC5F8E00051
:10BC8800C31A07EE903AF8EE677A424BC5F8E80017
:10BC980067EE877A5B68C5ED397A05F1EC0098475D
:10BCA80005F1EC08002800F0F1803B4B40461A787B
:10BCB8004146FAF7D9FBB5F8F230002B42D0D5F857
:10BCC800F4103B46B4F8F22038F913702B4DB2F556
:10BCD800C87F324A04BF002042F823004FEA830E8F
:10BCE80052F80E00384442F80E00002028F81300DD
:10BCF80021F813000133032BE4D1B5F8F230012BFE
:10BD08001BD1D5F8F8304FF4C87703F1C80292FB7D
:10BD1800F7F20A80D5F8FC20C83292FBF7F24A8085
:10BD28001F4AD5F800311288C83393FBF7F39B1AE2
:10BD38008B8030807080FDF7EBFDB4F8F230013B6A
:10BD4800A4F8F230174B1B685B0740F18B80B4F8FE
:10BD580004210A4B322A27D1D3F8F4201188A3F8FA
:10BD6800061151889288A3F80A213288A3F80C2179
:10BD78007288A3F80811A3F80E2117E03C190020D7
:10BD8800940E0020C20E0020902A0020000000001F
:10BD9800BD378635A8250020962A0020341A0020B1
:10BDA80008000020382A0020002A3BD0D4F8F400EC
:10BDB8000023B4F8042138F913E0C64D322AC64AE4
:10BDC80004BF002142F823109F00D1597144D1517A
:10BDD800002228F8132020F813200133032B1146E2
:10BDE800E7D1B5F80431012B17D10C2085F81C21B7
:10BDF80085F81D3103F044F9D5F8F430B5F806217B
:10BE08001A80B5F808215A80B5F80A219A80B5F841
:10BE18000C313380B5F80E317380B4F80431013B2E
:10BE2800A4F8043194F81E31AA4ADBB1D2F8F40020
:10BE3800D2F81031002182F81E11322593FBF5F358
:10BE48000380D2F8143193FBF5F34380D2F818310C
:10BE5800A24A93FBF5F312889B1A83803180718084
:10BE6800FDF756FDD4F8F420B4F8EC3011885B1ACD
:10BE7800A4F8EC305188B4F8EE305B1AA4F8EE3030
:10BE88009288B4F8F0309B1AA4F8F03094F8DE30B9
:10BE9800013384F8DE30D9E68E4D914F05F1EC027E
:10BEA80032F8112027F8112012B207EE902A8D4A95
:10BEB800F8EEE77A32F9112067EEA67A0131E0EC64
:10BEC800017A07EE902AF8EEE77A032967EE877A77
:10BED800E3EC017AE0D105F59A7005F5A071024608
:10BEE80003F065FB05F59A7005F5A67104AA03F041
:10BEF8005EFB04A895ED390ADFF8D8A1014603F0E6
:10BF08006FFBDDED054ADDED047A9DED065A95EDF2
:10BF1800594AD5ED583A95ED563AB6EE007A64EEA0
:10BF2800874A67EE875A64EEA47A25EE075AE5EE4B
:10BF3800A57A07A80146B7EE008AE5EE057A0AAAAF
:10BF48000DAFF0EE482AE7EEC72A0AF5BC7965EE90
:10BF5800846AD5ED577AE2EEA36A25EE236AE4EE09
:10BF6800836A23EEE57AB1EE452AE2EE276AA2EE6D
:10BF7800A76AA4EEA77A67EEE57AF1EE641AE2EE14
:10BF8800837AA1EE846AA2EE847AE1EEA37AA5EE22
:10BF9800836AA5EE037AE2EE047A85ED576AC5ED69
:10BFA800567AB1EE466AC5ED586A85ED597AF1EED2
:10BFB800666AB1EE477A8DED097A8DED076ACDEDA7
:10BFC800086A03F0F4FA95ED560A474810A903F0F9
:10BFD80007FB07A8444913AA03F0CAFA13A810A933
:10BFE8003A4603F0E4FA0AA8394613AA03F0C0FA5D
:10BFF8003D4813A93A4603F0DAFAD5ED5A7A9DED91
:10C008000F7A95F86C31B4EEE77AF1EE10FACCBFFE
:10C0180043F0080323F0080385F86C31D4F8703135
:10C028001B78F0EE489A0AF5C4753BB3DAED5D8AE1
:10C038004846B0EE680A10A903F0D2FA9AED618A70
:10C048000AF59470B0EE480A13A903F0C9FA4A46F3
:10C0580010A813A903F0ABFA2846B0EE680A10A995
:10C0680003F0BEFA384613A9B0EE480A03F0B8FA4E
:10C0780010A813A92A4603F09AFA07E098E80700DF
:10C0880089E8070097E8070085E80700D4ED4B7AB0
:10C09800D4ED4A6A94ED4C7A0E4D67EEA77A0023E8
:10C0A800E6EEA67AE7EE077A9FED107AF4EEC77A05
:10C0B800F1EE10FA06DC9FED0E7AF4EEC77AF1EE97
:10C0C80010FA19D5C4F84C31C4F85031C4F85431B9
:10C0D80025E000BF3C1900204C1A00200800002071
:10C0E800BC0E0020C20E00204C500108B81E8D3F27
:10C0F8003D0A673F6F12833A05F5BC7005F5C471B8
:10C1080005F5A67203F034FAD5ED397A1FED070A62
:10C1180005F5A67080EE270A014603F061FAB4F827
:10C128009431984D01339BB2B3F57A7FA4F89431DA
:10C138002ED195ED570AD5ED566A95ED587AD5ED7D
:10C14800597A20EE000AA6EEA60AA7EE070AA7EE7D
:10C15800A70A07F03BFC89EE800A0023A5F8943172
:10C16800D5ED576A95ED587AD5ED597A95ED566A19
:10C1780060EE266A20EE077A60EE277A26EE000A3D
:10C18800C5ED576A85ED560A85ED587AC5ED597A99
:10C19800D4ED578A94ED59AA94ED56BAD4ED58AA1D
:10C1A8009FED799A68EECA7AB7EE007AEBEE2A7AB2
:10C1B80077EEA77AF4EEE97AF1EE10FA0EDCFFEEEC
:10C1C800006AF4EEE67AF1EE10FA24D4F4EE477A37
:10C1D800F1EE10FAC8BFF0EE477A01E0F0EE477AC8
:10C1E80017EE900A04F022FA41EC100B07F08CFBD2
:10C1F80051EC100B04F06EFA08EE100AB5EEC08A86
:10C20800F1EE10FA09DD78EE497AF5EEC07AF1EE32
:10C2180010FA10DC23E09FED5D8AF1EE487A77EEA4
:10C22800C97AF5EEC07AF1EE10FAB5EEC08A13DDE0
:10C23800F1EE10FA06DD38EE499ADFED557AB4EEE4
:10C24800E79A03E09FED527AF4EEC77AF1EE10FA1E
:10C258004CBF0123002312E0F1EE10FA06DD38EEA0
:10C26800499ADFED4C7AB4EEE79A03E09FED497AFC
:10C27800F4EEC77AF1EE10FACCBF0123002353B1D4
:10C28800B0EE4A0AF0EE4B0AFCF7BEFF9FED42CA39
:10C2980070EE008A41E02AEE8A0A6AEEAABAABEE8C
:10C2A800280AB0EE6B7A30EE000AA8EEA87AB5EE4E
:10C2B800400AF0EE007AF0EE690AF1EE10FAE7EEC5
:10C2C800670AB0EE679A04D1F5EE400AF1EE10FA6B
:10C2D80004D0FCF799FFB0EE40CA01E09FED2ECAEA
:10C2E80028EEAA0AEAEE0ABAABEE0A0AF0EE690AE2
:10C2F80030EE000AEBEEC90AB5EE400AF1EE10FA8C
:10C3080004D1F5EE400AF1EE10FA04D0FCF77CFFF8
:10C31800F0EE408A01E0DFED208A9FED209A204D63
:10C328002CEE090A07F0AAFA28EE090A288007F075
:10C33800A5FADFED1C7A1C4A688068EEE78AFDEEF4
:10C34800E88ACDED018ABDF8043013F4004F18BF18
:10C3580003F5B4731380002300E00123002284F85E
:10C36800DE20002B7FF472AC06E00023A4F8EC304A
:10C37800A4F8EE30A4F8F03017B0BDEC0A8BBDE895
:10C38800F08F00BF3C190020DB0FC93FDB0FC9BF8E
:10C3980035FA0E3C35FA0EBC000000004D3D0F4446
:10C3A800F40E0020E12E6542F80E002001380A4BF9
:10C3B800042804D8DFE800F00507090B0D00074A38
:10C3C80008E0074A06E0074A04E0074A02E0074A8D
:10C3D80000E0074A1A60704700010020D9A500084C
:10C3E8006DB80008F1FC0008D9A20008959F000864
:10C3F8002D990008704708B50B4B002093F82C10B6
:10C40800F9F7D2FC094B1B68187A082801BF084BBA
:10C418004FF480521A80102208BF5A80A0F10903F5
:10C428005842584108BD00BFD00000207C1C0020A5
:10C43800D41A0020704770477047FEE7FEE7FEE712
:10C44800704730B50024E3B293420DD2030F092B95
:10C4580094BF3033373301F8143001EB440300251F
:10C4680000015D700134EEE730BD30B5002202F105
:10C47800805303F5B8539B0042F400441D6840F60E
:10C488000F7144F08004294001322143042A1960C5
:10C49800EDD1024B40F08000186030BD4C5C00408C
:10C4A8002DE9F347884D894C2B68894E9BB2A380B0
:10C4B800A28831880A40970507D54FF6FF53854A69
:10C4C8002B6013780133DBB21370A3880B40180478
:10C4D80040F100830023ADF802302B687B4F9AB2FD
:10C4E8001804A28040F1F682BB8803F00F03BB71E9
:10C4F800002B40F0C182784A13689BB23B803B888E
:10C5080003F030037B803B8803F440533B80116881
:10C518004BF6BF730B4083F4005383F0200343F4BE
:10C52800004343F080031360BB88D90621D4116807
:10C5380048F60F730B40694913600B681A7A022A90
:10C54800884601D0042A02D1F9F7BAFB5AE2062A32
:10C5580040F06B825A78052A08D11A78520605D11C
:10C56800D878FFF782FFBB681B6A9847E3689B6827
:10C578005AE213689BB2ADF80230BDF802301F05CD
:10C5880040F1D0811168554F40F68F730B405449E4
:10C5980013600A68534B92B213445B0088461A68CA
:10C5A8003B68187A092817D092B2520002F18042EB
:10C5B80002F5C04211781970517859709188C8B243
:10C5C800090A41EA002159801189C8B2090A41EAD9
:10C5D800002199809289DA8001221A72DA8893F808
:10C5E8000190002A40F0DC801A7812F07F024AD1CC
:10C5F800B9F1090F0FD1DA78012A00F2B8809978D9
:10C60800002940F0B4809988002940F0B0809A72DF
:10C61800A3685B68A9E0B9F1050F10D193F903206D
:10C62800002A01DA0823B9E09A78002AFAD19A8810
:10C63800002AF7D19B7A002B00F0A280F2E7B9F12B
:10C64800030F0ED1DA78012A40F091809A88002AE7
:10C6580040F08D805A7A42F020025A72A368DB6952
:10C6680083E0B9F1010F40F08280DA78012A7ED1A7
:10C678009A88002A7BD15B7A980678D5F9F7B6FBB9
:10C6880000287DD073E0012A2ED1B9F10B0F6ED1AD
:10C69800E26858799269D97890473B689A7A002A73
:10C6A80065D0002863D11A79002A60D19B78002BC5
:10C6B8005DD1064B9B68DB689847084B1B685A7925
:10C6C800DA72DA781A735BE0445C0040D41A00200E
:10C6D800B8270020982A0020005C00407C1C00201D
:10C6E800505C004004300020022A40D1B9F1010F0B
:10C6F800C4D0B9F1030F3AD1587920F0800E4FEA2F
:10C708008E0202F1804101F5B84110F0800F0968EE
:10C7180014BF01F0300101F44051BEF1030F26D8D7
:10C72800B3F802E0BEF1000F21D101B39B7AF3B157
:10C7380002F1804202F5B842010613684BBF23F4A8
:10C74800E04323F4804323F0400323F070034BBFFE
:10C758009BB29BB283F0100383F4805343F40043ED
:10C7680043F080031360A3689B69984708E0E36877
:10C7780048465B69984703280FD000287FF452AFDA
:10C78800D8F80020A14B92B213445B001A6800222B
:10C798001A6030236380062300E009233A6847E1E2
:10C7A800B9F1060F12D11A78520678D19B78012B6D
:10C7B80002D1E368DB6967E0022B02D1E3681B6AF8
:10C7C80062E0032B6BD1E3685B6A5DE0B9F1000FAF
:10C7D80038D15988002962D15A6822F47F42B2F5CB
:10C7E800003F5CD11A7812F07F0204D19B88002B9D
:10C7F80000F0D58153E0012A08D1E268587992699E
:10C80800904700284BD13B689B7A17E0022A46D113
:10C818005A7902F00F010BB29B0003F1804303F534
:10C82800B84312F0800F1B6814BF03F0300303F401
:10C838004053032933D812F0700F30D1002B40F049
:10C84800AE812CE0B9F1080F04D11B785B0600F02B
:10C85800A88124E0B9F10A0F21D11A7802F07F02E9
:10C86800012A1CD19A7AD2B15988C1B95A6822F4DE
:10C878007F42B2F5803F12D1E268587992699047B9
:10C88800002800F090810AE04BB13A684FF00008A8
:10C89800A2F8128093614046984740460BE0E3684F
:10C8A8003A681B6950789847032804D1584B1B688D
:10C8B80009221A72BDE03A68138A4FF6FF718B425B
:10C8C80001D10923B4E0022800D00BB90823AFE056
:10C8D80092F9001000291FDAD1880191019883424A
:10C8E80002D9019B138210E08B420ED2E16891F8C5
:10C8F8002C00834201D2002105E093FBF0F100FBFC
:10C90800113313B90121434B1970E36893F82C30A4
:10C918009382F9F7D5F98CE0032313724FF440534F
:10C92800238086E0BDF802301BB2002BBFF6D5ADE0
:10C93800116840F68F730B401360354A17683B7ACD
:10C94800022B904671D0042B6FD0032B01D0052BFE
:10C9580066D1BB693A8A8BB9398A00293BD04FF432
:10C96800405323802C4B1A68284B92B213445B0027
:10C978001A6800221A60302363802CE0002AEBD06A
:10C98800B7F81490914528BF91461FFA89FA504686
:10C9980098473B8ACAEB03033B827B8A53447B82DA
:10C9A8001D4B1A681D4B92B213445B0009F101023A
:10C9B8001B689BB203F1005303F5405352105B0010
:10C9C8004FF0000E9645C7D053F82E1020F81E10D1
:10C9D8000EF1010EF6E7BB8A8B42D8F8003001D879
:10C9E800032201E011B105221A720BE006221A7225
:10C9F800094B1A68054B92B213445B001A68196018
:10CA080030236380D8F800301B7A0FE00230002012
:10CA18007C1C0020972A0020505C00400430002035
:10CA2800072B02D1E368DB6898470823D8F8002071
:10CA38001372FFF7E0FC5E4B1A684BF6BF731340A6
:10CA48002288D704228848BF83F4805390046288E0
:10CA580048BF83F40053D106628848BF83F01003AF
:10CA6800920648BF83F0200343F4004343F0800359
:10CA78004F4A9BB213602DE09A0002F1804202F502
:10CA8800B842116889B2ADF80210BDF8021009B2B7
:10CA9800002909DA106840F68F7101401160013BE6
:10CAA800444A52F823309847BDF802301F067FF5F4
:10CAB80014ADA1798B0003F1804303F5B84348F620
:10CAC8000F72186802401A603A4B03EB81039B69A6
:10CAD800984702E5A28833881340590505D54FF6D3
:10CAE800FF332B60344B5B689847A28831880A4033
:10CAF800920444BF4DF6FF732B60A3882F4A0B4066
:10CB0800DB0452D54EF6FF732B6000231374137C9D
:10CB1800052B41D8DFE803F0030D1418222D6369B3
:10CB2800264D1BB901F0B2FD062300E005232B7446
:10CB38003BE001F0ABFD042323740123636134E07F
:10CB480002236374032328E0637C013BDBB2637434
:10CB5800637C53BB194B04221A7426E0184A1368E5
:10CB68009BB243F010031360052323740A236374F4
:10CB78001BE0637C114A013BDBB26374637C03F006
:10CB8800FF0093B90E490C684FF6EF7323400B6012
:10CB980006231374506108E00623237405E0094B4B
:10CBA80073E6094B71E6094B6FE602B0BDE8F08702
:10CBB800005C004058500108D0000020D41A002022
:10CBC800405C004071590008295A0008055A0008BD
:10CBD800012380F8453070472DE9F04390F8441060
:10CBE800002380F84430002953D02E4C2268002AB4
:10CBF80052D02268052A52D12B4C20290D4628BF35
:10CC080020256E1C27687610DFF8A8E0DEF80030D3
:10CC18009BBBDFF8A4C000F13203324613F8019C35
:10CC280013F8028C013A48EA09282CF8048C03F11D
:10CC380002030CF1040CF1D11C4B1A681C4B92B284
:10CC480013445B002A46D3F800C01D60DEF80030AC
:10CC58002B44CEF80030DFF864E0DEF8003023F42F
:10CC6800E04323F040039BB283F0300343F40043D6
:10CC780043F08003CEF8003000E000228A4203D05F
:10CC88002368DB1B312BBFD9531A58425841BDE8E2
:10CC9800F0830120BDE8F0831046BDE8F083184614
:10CCA800BDE8F0837C2A0020442A0020505C004024
:10CCB8000A300020B427002084610040045C004052
:10CCC800002280F8452087E790F84420531C02444E
:10CCD800DBB280F8443082F8301090F845200AB171
:10CCE800132B00D978E77047014B1868C0B270471A
:10CCF800702700200120704770477047F7B51C4B1C
:10CD08001A680AB91C6800E001241A490E78002242
:10CD1800D0B2A04202F1010207D202AD2F18164D7F
:10CD28003544285C07F8040CF2E71A68121B1A60ED
:10CD38000A781D6822440A709DB903204021F9F73A
:10CD480033F80E4A136823F4804323F070039BB230
:10CD580083F4405343F4004343F080031360054BCE
:10CD68001D70002CCBD09DF8040003B0F0BD00BFAF
:10CD780070270020EC1A0020742700200C5C00406B
:10CD880070B5044600F0BBFBB4F5807F0ED0BB2C19
:10CD98000ED8612C0ED8292C0ED8132C0ED8092C9D
:10CDA8000ED8002C14BF062500250AE0002508E04F
:10CDB800012506E0022504E0032502E0042500E041
:10CDC8000525154C8021A3686B209847642002F044
:10CDD8001FF9A36803216B209847104AA3681178AC
:10CDE800192098470F2002F013F9A36829461A2042
:10CDF8009847A36818211B209847A36810211C2076
:10CE08009847A368022137209847A3683820012152
:10CE1800BDE87040184700BFD4090020E40900208D
:10CE280008B500F06CFB074B5B7813B1012B03D0FE
:10CE380008BD4FF4006201E04FF48052024B1A80A3
:10CE480008BD00BFD009002008000020094A137857
:10CE58001844C0B210F0800F18BF80381070134605
:10CE6800054A19781378994201BF00231370014AC3
:10CE780013707047F91B0020F81B002010B50A4BEF
:10CE88000A4A1B7842609C18094A046012789A4240
:10CE980025BFD31A0B60C3F1800300232EBF4B605C
:10CEA8000B604A6010BD00BFF91B0020FA1B002070
:10CEB800F81B00201FB5684602A9FFF7DFFF044BE7
:10CEC80002981B6803440398184405B05DF804FBF6
:10CED800400D00200F4B73B518781C4698B10523F8
:10CEE8000D4D8DF800304FF4805600238DF8013039
:10CEF80001A82E856946022201F06EF9AE619DF8FF
:10CF0800050000F0010000F00100207080F0010031
:10CF180002B070BD3D0D002000040048064B70B5FE
:10CF28001D6806461C46FFF7D5FF18B923685B1B2A
:10CF3800B342F8D970BD00BF442A00202DE9F04F54
:10CF480089B0824601930023029103929946039A7D
:10CF5800934205DA029A52F8232001339144F6E706
:10CF6800019B4D46002B56D1FFF7B4FF002852D144
:10CF780001987CE002223F4E8DF81C201A0C4FF4D9
:10CF880080578DF81D2006201A0A8DF81E208DF86E
:10CF98001F30FFF7C3FF3785062001F0F5F8364B41
:10CFA800B76101221A700020378507A9042201F011
:10CFB80013F9029FD04626464FF0000B039B9B4572
:10CFC8001EDABC4657F8042B4FEA8B03002A47D0D9
:10CFD800B24235D332465AF80310CDF814C00020B7
:10CFE800049301F0F9F8049BDDF814C05AF8032003
:10CFF80032444AF80320DCF800309E1BCCF800606D
:10D008001C4B4FF480529A611C4A13682D1B1C4418
:10D01800019B14604BB345B3184B1B68DCB22A194B
:10D02800B2F5807F164AD2688CBFC4F580742C464E
:10D0380093429FD3134A00231370134A137014E0CA
:10D048000020D8F8001001F0C7F857F8043CD8F8C9
:10D058000020F61A1344C8F80030002347F8043CAF
:10D068000BF1010B08F10408A8E7C5EB090009B0AA
:10D07800BDE8F08F000400483D0D0020400D002061
:10D088000C000020F81B0020F91B002030B50E4DC5
:10D098000E4C2A7823789A4285B011D0684602A9A6
:10D0A800FFF7ECFE002302A902226846FFF746FFBD
:10D0B800FFF7CCFE20782B781B1A5842584100E025
:10D0C800012005B030BD00BFF91B0020F81B00206F
:10D0D80038B50E4C4FF4805545F20820FFF71EFF77
:10D0E8002585062001F050F8094BA56101221A7028
:10D0F800C720258501F048F8064AA561002313706A
:10D10800054A1370054A136038BD00BF0004004883
:10D118003D0D0020F81B0020F91B0020400D0020C9
:10D12800F7B503238DF80430030C8DF805308DF81E
:10D138000700030A06200F4614468DF80630FFF74D
:10D14800EDFE78B1084D4FF4805601A904222E85D2
:10D15800002001F041F838460021224601F03CF851
:10D16800AE61204603B0F0BD0004004810B5D420DD
:10D1780000F0C0F9802000F0BDF9A82000F0BAF94D
:10D188003F2000F0B7F9D32000F0B4F9002000F0F8
:10D19800B1F9402000F0AEF98D2000F0ABF9142071
:10D1A80000F0A8F9A12000F0A5F9C82000F0A2F924
:10D1B800DA2000F09FF9122000F09CF9812000F09D
:10D1C80099F9CF2000F096F9D92000F093F9F120D1
:10D1D80000F090F9DB2000F08DF9402000F08AF98A
:10D1E800A42000F087F9A62000F084F9AF2000F011
:10D1F80081F9A62000F07EF9AE2000F07BF920200E
:10D2080000F078F9002000F075F9B02000F072F90C
:10D21800402000F06FF9002000F06CF9102000F0B9
:10D2280069F94FF48064013C0020A4B200F05DF974
:10D23800002CF8D1812000F05DF9C82000F05AF9DF
:10D24800AF2000F057F9012010BD70B500EB800049
:10D25800094CA0F1A1059C3825440444074B15F856
:10D26800010F1E78704000F040F9A542F6D1304613
:10D27800BDE8704000F039B994500108992A00209F
:10D2880010B5441E14F8010F10B1FFF7DEFFF9E7DF
:10D2980010BD08B55038C0B200F02CF9002000F0DD
:10D2A80029F91020BDE8084000F024B9054B1A7888
:10D2B80002F0FF0122B10122027000221A707047A9
:10D2C80001707047F01A002037B5104B04465D68AE
:10D2D800187806216A46A847A8B19DF800209DF84D
:10D2E800013043EA022323809DF802209DF8033091
:10D2F80043EA022363809DF804209DF8053043EA41
:10D308000223A380012003B030BD00BFD409002050
:10D3180013B5104B04465B683B2006216A469847C4
:10D32800A8B19DF800209DF8013043EA022323802C
:10D338009DF802209DF8033043EA022363809DF89C
:10D3480004209DF8053043EA0223A380012002B09F
:10D3580010BD00BFD409002003460A4668201946BC
:10D36800F8F79EBAF8B52F4D2F4C06464FF42043D8
:10D378002868636087693F0404D51F46013B002F76
:10D38800F8D111E04768294B3B4043F4903343F010
:10D39800D00343604FF4204363608769BF070AD412
:10D3A8001F46013B002FF8D16360F8F767FA003099
:10D3B80018BF0120F8BD4FF4204386626360866978
:10D3C800770604D41E46013B002EF8D1ECE76360D3
:10D3D800164E43681E40164B334343EA01434360ED
:10D3E8004FF420436360286859B1866976070CD4E6
:10D3F8001E46013B002EF8D1D6E71A46013B002A0B
:10D40800D2D082699206F8D506E063600139436A92
:10D4180002F8013BC9B2E3E763602023C36101203E
:10D42800F8BD00BF8C0E0020F01A0020009800FC08
:10D43800D0240002094B1B681869094B20F01F0211
:10D4480010B5D258012400F01F0304FA03F31A425E
:10D4580003D0F8F75DFD034B1C7010BDE0090020F8
:10D4680014040140F01A00202DE9F0410369C7684F
:10D4780005460E461F40002F35D0B7FA87F24FF009
:10D488000043D340DB432B611F40A2F11B03042B55
:10D49800F1D8DFE803F0221F1C190300746A24B1D5
:10D4A800013C0023A4B2736201E0EC6AA4B2D6F88E
:10D4B8002080B8F1000FDED0D8F800304046214671
:10D4C8009847D8F80480F4E73068696B07E070681B
:10D4D800A96B04E0B068E96B01E0F068296C0368A7
:10D4E80089B29847C7E7BDE8F081024640213C2051
:10D4F800F8F7D6B9024680213C20F8F7D1B9F0B543
:10D50800324D2B7A85B0002B5DD1314C2368002B2E
:10D5180059D01A682F4E12B171690A4372619A88FC
:10D528009868ADF800206946022200278DF803208C
:10D538008DF80270F8F78CF8B36943F00103B36112
:10D548002368187B1B7D03F0030203F0FC0303F13F
:10D55800804303F5803392009E680F21914026EAAC
:10D5680001019960996800FA02F20A439A601A4B1D
:10D578001A681AB1384601F0BDFD01E0174A1A6071
:10D5880023681869F8F7C4FC23681B690293082309
:10D5980001260DEB030000278DF80D308DF80C7077
:10D5A8008DF80E6000F098FE23688DF806705B7D9C
:10D5B8008DF8043001A803238DF805308DF8076035
:10D5C80000F040FE2E7205B0F0BD00BFF01A00203A
:10D5D800E009002000100240E02500203DD40008AA
:10D5E800094B1B681869094B20F01F0210B5D25867
:10D5F800012400F01F0304FA03F31A4203D0F8F7DA
:10D6080087FC034B1C7010BDE00900201404014086
:10D61800F01A00200148024926E700BF00480140EF
:10D62800C8260020014802491EE700BF004001400B
:10D63800A02600200148024916E700BF0004004068
:10D64800782600204FF0804000490DE75026002042
:10D658000148024908E700BF002C014028260020A5
:10D668000148024900E700BF002C0140282600209D
:10D67800224B10B5224C5A43224BB3FBF2F20388DB
:10D688000139013AA04289B292B29BB20ED004F598
:10D698000064A0420AD0B0F1804F07D0A4F59834B6
:10D6A800A04203D004F58064A04202D123F07003A5
:10D6B8009BB2154CA04206D004F58064A0421CBF62
:10D6C80023F440739BB203800D4BC16298420285DC
:10D6D8000FD003F5006398420BD003F540639842DE
:10D6E80007D003F58063984203D003F5806398421E
:10D6F80001D1002303860123436110BD40420F007E
:10D70800002C014000A24A04001000400E4B800A81
:10D71800984216D007D8B0F5801F0CD04A3B9842E3
:10D728000DD102207047094B984206D00233984227
:10D7380005D1042070470120704703207047FE2060
:10D7480070470020704700BF4B00100050001000C9
:10D75800F8B50468064620460F461546FFF7D6FF7B
:10D7680004284BD8B27A910847B902238B40D4F8E1
:10D778000CE0DB439BB203EA0E03E3600A23204A72
:10D7880003FB001342F82370043342F82350154674
:10D798003FB1B17AE268890802238B409BB21343F8
:10D7A800E360282202FB00522032EFF31286502356
:10D7B80083F3128803B203EB8303DB0003F10C014C
:10D7C8001C3329442B4451F8047F17B117600A68A9
:10D7D80004329942F7D100231360F3B283F311881E
:10D7E800282303FB0050036A1BB1E36843F00103DD
:10D7F80003E0E2684FF6FE731340E360F8BD00BF34
:10D80800282600200148FDF7BDBD00BFFC1A0020F6
:10D818000148FDF7B7BD00BF501B00200148FDF7C8
:10D82800B1BD00BFA41B00200846FDF70DB90F4B82
:10D838001A786F2A17D1598840F2DC72914212D1B6
:10D848001A79BE2A0FD193F8D827EF2A4FF0000093
:10D858000BD113F8012B5040054A9342F9D1B0FA85
:10D8680080F04009704700207047704700F00308B7
:10D87800DCF703082DE9F04F2DED028BF04C85B055
:10D88800002140F2DC72204605F0E9FDED4B04F57D
:10D8980038721A60EC4B00261E70EC4B04F2AA7228
:10D8A8001A606F232370012003236371FBF7AEFD19
:10D8B8000220FBF7ABFD4FF48070FBF7A7FD202299
:10D8C8004FF4167384F868216E22A4F8643184F842
:10D8D8007A21FA230A22A4F8663184F87B214FF4CE
:10D8E800FA732B22A4F86C3184F87D2101232122BC
:10D8F80084F85E3184F8693184F86A3184F87C31BF
:10D9080084F87E2184F884312322002384F87F213F
:10D91800C4F81432C4F818324FF4C872052384F8D6
:10D92800A867A4F87061A4F86E61A4F8726184F81D
:10D93800556184F8566184F85761A4F85861A4F8D1
:10D948005A61A4F85C6184F85F61A4F88261A4F864
:10D958008021A4F8866184F8116284F8106284F842
:10D968001C6284F81D6284F81F3240F2DC53A4F86C
:10D97800963140F24C43A4F8983140F26C73A4F805
:10D988009A3140F27533A4F89C3140F64303A4F869
:10D998009E3184F81E6284F8906184F8916125466E
:10D9A8002346032ECCBF0122002206F1010683F88C
:10D9B800A02114BF1E220522122E83F8A12103F1F3
:10D9C8000203EED140F27E42A4F8402140F23A72BE
:10D9D8004FF4FA63A4F8422140F27E52A4F8C6310B
:10D9E800A4F8CA31A4F8CE31A4F8D231A4F8482159
:10D9F800052340F2EA5284F8E031A4F84A21C8230A
:10DA080040F2B452002601274FF47A7A4FF01E0BE9
:10DA180040F2DC504FF01909A4F8E431A4F84C2185
:10DA28004FF4C8733222A4F8E831A4F846010390F1
:10DA3800A4F84E21A4F8503184F893B184F8DF712A
:10DA480084F8E19184F8E27184F8E37184F8E6716E
:10DA580084F8EC7184F8926184F89461A4F8C4A104
:10DA6800A4F8C8A1A4F8CCA1A4F8D0A184F8D461E2
:10DA780084F8DE6184F8EA61A4F844A1A4F852218C
:10DA8800019284F8546100F029FDDFF8B8C12673CB
:10DA9800DCF80030019A83F80BB04FF05F0E83F882
:10DAA80003E04FF00F0E83F805E04FF0220E83F8E5
:10DAB80006E04FF00E0E83F810E04FF0350E83F8B5
:10DAC8001AE04FF0210E83F811E04FF0530E83F85F
:10DAD8001BE04FF05A0E83F808E04FF0780E83F8F9
:10DAE8000AE04FF02D0E4FF02808142183F80CB0EF
:10DAF80083F807904FF00A0B4FF0640983F814E09D
:10DB08004FF4FA7ECDF808C01F70597599755A738D
:10DB18001A719F7783F8018083F8028083F817B021
:10DB28009E731E76DE735E7683F812B083F81C90BF
:10DB380083F80980A3F84EE0DFF82CE1C3F838E059
:10DB4800C3F83CE0DFF824E1C3F828E0DFF820E17F
:10DB5800C3F834E0DFF81CE1C3F848E0DFED3C7AB5
:10DB68009FED3C8AC3ED0B7A4FF04B0E83F84CE0E7
:10DB78004FF4E17EC3ED0C7AA3F85CE0B7EE087AC7
:10DB8800F1EE047A4FF0100E83F85EE083F85080CF
:10DB980083ED087A83ED097A83ED108AC3ED117A53
:10DBA80083F8536083F854B083F855B083F856B0BF
:10DBB80083F8579083F8589083F8599083F85A60FF
:10DBC800039884F8AC274FF0460E042284F8B21765
:10DBD800019184F8ABE7A4F8B40784F8AA9784F80D
:10DBE800AD6784F8B16784F8AE6784F8AF6784F8E6
:10DBF800B06783F86820152283F87420164A9A675C
:10DC0800164ADA67164AC3F8802083F88470A3F8A6
:10DC18006460A3F86660A3F86260C3ED1B7A83F8BA
:10DC2800708083F871800F4800F098FCDDF808C018
:10DC38000199DCF800204FF4487382F820711BE04A
:10DC4800401D0020D80E00207C250020040F002055
:10DC5800CDCCCC3E000000009A99193FF6287C3FB5
:10DC68003D0A773F097201088FC2F53C0000604009
:10DC78006666663F0000404082F81D6182F81E61BA
:10DC880082F81F8182F82461A2F82231674684F85D
:10DC9800D71184F8D6B1A4F8D8A184F8DA61A4F829
:10DCA800DC9111460E2303FB06236FF0170083F85F
:10DCB8002501032083F826016FF02F0083F8270140
:10DCC800072083F828016FF0230083F82901052035
:10DCD80083F82A01642381F82B3101365A2381F80D
:10DCE8002C3181F82D31082E4FF0FF0381F82E31A9
:10DCF80001F10E01D6D1002382F895312D4B18EE93
:10DD0800102A45F8102F9D42F9D12B4800214022B6
:10DD180005F0A5FB0023294D294C59591A1904333C
:10DD28000868C2F8A002382BF5D104F50870002164
:10DD3800802205F094FB05F13801702204F5087083
:10DD480005F082FBFAF718FE3E68002301253146EC
:10DD580004F58F604FF4CC7284F8D03784F8CE572E
:10DD680084F8CF5705F070FB04F5C26031464FF4D4
:10DD7800CC7205F069FB134B1B681A68C4F8B62708
:10DD88005A68C4F8BA279A68C4F8BE271A68C4F84B
:10DD9800C2275A68C4F8C6279A68C4F8CA27022353
:10DDA80084F8D85484F8703605B0BDEC028BBDE811
:10DDB800F08F00BF001E0020E01F0020385301082C
:10DDC800401D0020040F00201549D1F8883043F485
:10DDD8007003C1F88830134B1A6842F001021A60C8
:10DDE8005868114A02405A601A6822F0847222F474
:10DDF80080321A601A6822F480221A605A6822F463
:10DE0800FE025A60DA6A22F00F02DA62186B074AD9
:10DE180002401A6300229A604FF000638B607047DB
:10DE280000ED00E0001002400CC07FF8CCFC00FFC1
:10DE3800074B93F8D037012B08D1064A064BD06818
:10DE48001B68834234BF00200120704700207047C0
:10DE5800401D00200C000020400D002038B5094B63
:10DE680093F8D05765B9084C2068F8F7CDFF074BF1
:10DE780025601B78022B03D1BDE8384000F0EEBACC
:10DE880038BD00BF401D0020C0270020BF2700204C
:10DE9800064B93F8D0371BB1012B05D1FFF7F6B825
:10DEA800034B186801F06EB900207047401D002030
:10DEB800C0270020F8B5011F06460023083051F896
:10DEC800042F02F120043F2C3BD802F108040F2C48
:10DED80006D80232032A04D9002B08BF012300E028
:10DEE80002238142EBD1012B30680ED0022B1AD0CD
:10DEF800736803F003039B0000F0030043EA00107B
:10DF0800B36803F00303184317E000F00F0040F074
:10DF18004000FCF799FDB068736800F00F0040EA14
:10DF28000310C0B209E000F03F0040F08000FCF7A9
:10DF38008BFD3079FCF788FD307ABDE8F840FCF7B6
:10DF480083BD06F10C0734463A46002552F8043DD5
:10DF580003F18001FF294FEA850510D903F5004137
:10DF6800B1F5803F02D245F0010508E003F5000352
:10DF7800B3F1807F34BF45F0020545F00305B24296
:10DF8800E4D165F03F00C0B2FCF75EFD05F0030385
:10DF9800022B207807D0032B0CD0012B13D1FCF7D0
:10DFA80053FD60780FE0FCF74FFD6078FCF74CFDFF
:10DFB800A07808E0FCF748FD6078FCF745FDA078FC
:10DFC800FCF742FDE0780434FCF73EFDBC424FEA22
:10DFD800A505DBD1F8BD10B504467F2C06D964F041
:10DFE8007F00C0B2FCF730FDE409F6E7E0B2BDE817
:10DFF8001040FCF729BD430083EAE070EBE72DE908
:10E00800F047314B93F8D037012B86B0074601D043
:10E0180004464AE005F067FA03A90546064668463D
:10E02800FEF72CFF039B049A029713442B443F2BC3
:10E03800059519D90023684603A90322FEF77EFF38
:10E04800039B3BB9049B2BB9204A13705370059B63
:10E05800ABB301E0FEF7FAFE039B049A059E134456
:10E0680033447F2B2BD8029FDFF86090CA4639468D
:10E078001AF8024BC4F18008B04528BFB0460AEB35
:10E0880004004444E4B2424605F0DEF9802C89F8E5
:10E09800004014D1C8EB0606504607EB080132468B
:10E0A80005F0D2F989F8006009E0254614F8011B4B
:10E0B80021B1074B186801F06EF8F6E7ED1B28460A
:10E0C80006B0BDE8F08700BF401D0020F81B002007
:10E0D800C02700200FB407B504AB064953F8042B3A
:10E0E80001930020FAF76EFF03B05DF804EB04B06B
:10E0F800704700BF31D8000820B9034B1B680822BD
:10E108001A827047014870477C1C00207400002068
:10E1180020B9034B1B6808221A82704701487047D0
:10E128007C1C00207400002021B901288CBF02202B
:10E13800002070470220704710B5094B1A68D37841
:10E14800042B0BD8074C518ADB00234418B99B8950
:10E158005B1A138210BD9B68581810BD002010BDB3
:10E168007C1C002074000020054B1968054B4A8A66
:10E1780018B99B8D9B1A0B827047986A1044704798
:10E188007C1C00207400002040F2E9330F4A1289F9
:10E19800920704D4013B9BB2002BF7D10BE00C4A49
:10E1A80040F2E933107009490989C9070AD4013BCB
:10E1B8009BB2002BF7D1074A938801339BB2938017
:10E1C800FF2070471078C0B2704700BF0038004089
:10E1D8000C3800407C1C002030B5174B9B894FF44D
:10E1E8007A733AB311B10D78013107E0FF2505E0E4
:10E1F800013B9BB24FF6FF74A3420FD00E4C24890B
:10E20800A407F5D50D4C25700B4D2D89ED070BD4C2
:10E21800013B9BB24FF6FF75AB42F5D1084A938894
:10E2280001339BB2938005E0247808B10470013073
:10E23800013AD6E7012030BD003800400C380040D4
:10E248007C1C00200C4B0D49DA684378D243C2F39A
:10E258000222C2F10402934002781B010A44DBB295
:10E2680082F8003303780122580903F01F0302FAE9
:10E2780003F341F82030704700ED00E000E100E0D2
:10E2880073B50546002100680122FFF7F1F92A68F5
:10E2980013889BB243F001031380EB7A8DF80430A6
:10E2A8000124002601A88DF805408DF806608DF838
:10E2B8000740FFF7C7FFEB7A1B2B0BD1192301A8E7
:10E2C8008DF804308DF805408DF806608DF807400C
:10E2D800FFF7B8FF02B070BD036823F01F0202F118
:10E2E800804202F5823270B503F01F0114680123E1
:10E2F80003FA01F124EA0101116002682A4C22F0B4
:10E308001F0502F01F02295903FA02F221EA02024C
:10E318002A510279016802F1804221F01F0402F5B6
:10E32800823201F01F01155903FA01F129431151F5
:10E3380002681E4D22F01F0402F01F02615903FA01
:10E3480002F221EA020262510268194C22F01F0609
:10E3580002F01F02315903FA02F221EA020241795E
:10E3680032511029026812D122F01F0102F01F0257
:10E378004E5903FA02F232434A51026822F01F0151
:10E3880002F01F020859934003430B5170BD01F17D
:10E39800804122F01F0001F5823102F01F020C5863
:10E3A800934023430B5070BD04040140080401400E
:10E3B8000C040140104B10B50446185CFEF745FFED
:10E3C8000E4800EB4400B0F90610B1F57A7F05DB82
:10E3D800B1F5FA6FA8BF4FF4FA6101E04FF47A7112
:10E3E800A1F57A710A23092091FBF3F1BDE81040E9
:10E3F800C9B2F9F793BF00BF167201087C1C002050
:10E40800031EB8BF2D2210B5B8BF58420C46B8BF7E
:10E4180001F8012B0A22FAF7C1FD002303702046F8
:10E4280010BD10B50446B0F90000FFF7E4FDB4F9DB
:10E438000200FFF7E0FDB4F90400BDE81040FFF763
:10E44800DABD10B504460068FFF7D5FD6068FFF730
:10E45800D2FDA068BDE81040FFF7CDBD2DE9F74F0C
:10E468000120F8F7C1FE002488B3012C2FD8194EDB
:10E478004FF04C0909FB04FA06EB0A0808F1740787
:10E48800BD7815B10134E4B2EEE790F9003090F8A8
:10E4980004E01846104B03228DE8240001212A4687
:10E4A80053F82E30F8F7C4FC834660B106F12C000F
:10E4B800504429464A4604F0D2FF01231C44C8F8B8
:10E4C8002CB0BB70E4B20120F8F772FECCE703B0C1
:10E4D800BDE8F08F7C1C0020FC53010808B52222FF
:10E4E8001148002104F0BBFF104B00221049042002
:10E4F800515C83F8F0110132052183F8F501042AF3
:10E508004FF0000083F8F41183F8F70183F8F6114F
:10E5180003F10803EAD1074B0122A3F8B6225222DD
:10E5280083F8B22208BD00BF2E1F0020401D002026
:10E53800127201087C1C002010B5F7F799FD4FF402
:10E548003024012806D11CB1F7F792FD013CF8E709
:10E55800052010BD002C08BF052010BD70B506466B
:10E56800441E14F8011F89B1094D284604F0ADFF77
:10E578000028F6D005F1080398423FBF054B401B21
:10E58800C018A31B38BF80F84C32EAE770BD00BF43
:10E59800167201087C1C002007B51C4B03F6A40268
:10E5A800C3F8A02893F854225AB1012A14D10321A0
:10E5B80083F8A618072183F8A82883F8A7180C223F
:10E5C80008E0022183F8A618032183F8A82883F815
:10E5D800A718072283F8A4280D4B0E4A1A63402077
:10E5E800F8F702FE70B10122002390F900004021E3
:10E5F8008DE80C00084A4FF4E133F8F719FC0030B5
:10E6080018BF012003B05DF804FB00BF7C1C00208C
:10E6180074000020055B0008315C0008012000211F
:10E6280000F0A4B9F0B5184A92F8A938D2F8AC7835
:10E638001546032B11D807EBC3025E1C941CF6B2D7
:10E6480009D013469288D10705D5104203D008E0B7
:10E658000131042908D13346EBE785F8A9380020B1
:10E66800F0BD93F802E00021074C0C2204F50B6C76
:10E6780002FB01F31CF803209645E9D1234484F8F2
:10E68800A968D3F8B408F0BD7C1C00200B4B10B56A
:10E6980019684FF6FB720A401A60094A92F8EA288C
:10E6A8001C46084B0AB1052200E001221A60FFF758
:10E6B8008BFB4FF43643236010BD00BF405C004025
:10E6C8007C1C00207C2A002007B5064B0093064BD3
:10E6D80001930649064A074B0748FAF775FD03B048
:10E6E8005DF804FB0C630108E1620108CC700108C5
:10E6F800C5700108006301082B72010808B503788A
:10E7080033B90C4B0C481978BDE80840FAF75CBDE2
:10E7180004F040FF02280CD8064B1870074B0C2257
:10E7280002FB0030064B02301860FAF73BFF054841
:10E73800E5E708BD7C2500204F720108E824002089
:10E74800040F00203C65010808B503783BB90B4B62
:10E758000B4893F8A817BDE80840FAF735BD04F050
:10E7680019FF022808D8054B83F8A807FAF780FE96
:10E77800FAF73CFF0348E8E708BD00BF401D00204A
:10E78800537201083C65010838B5037803BB214B77
:10E798001B6801330F2B07D81F490C2202FB0312F9
:10E7A8001C4695682DBB00E01C4601340F2C01DD8A
:10E7B800002400E005D818490C2202FB04129568D1
:10E7C800BDB99C42F1D11548BDE83840FAF7FCBC08
:10E7D80004F0E0FE0F28044605D80F4A0C2303FB7B
:10E7E80000239D682DB921460D48BDE83840FAF749
:10E7F800EBBC084B1C6000F02FFC21462A46094858
:10E80800FAF7E2FC0C235C43034B185DBDE8384083
:10E8180000F036BCC4000020BC5401086072010836
:10E82800767201088E72010873B5037813B9F7F789
:10E83800B9FF3DE01F4901AA04F00DFF002401467D
:10E848002646254699B134B1012C08D1084604F072
:10E85800A1FE064603E0084604F09CFE054615495D
:10E86800002001AA04F0F7FE01340146EAE70B2D67
:10E8780002D911480C220BE0022C10D1A6F57A73AC
:10E88800B3F57A7F07D90D484FF47A714FF4FA62DD
:10E89800F7F705FF0CE00A4B03EB45035E80084BD6
:10E8A800084803EB45032946B3F90220FAF78CFC24
:10E8B80002B070BDFF6901085C670108CA6D0108F4
:10E8C8007C250020A572010838B50D4C23688342C9
:10E8D800054606D1F8F798FA204600214C2204F0A4
:10E8E800BEFDE36CAB4209D12846F8F78DFA05481E
:10E8F80000214C22BDE8384004F0B1BD38BD00BF4E
:10E90800A81C0020F41C0020034BDA69D379591C99
:10E918001344D171187A70477C25002010B5FFF791
:10E92800F3FF84B2FFF7F0FF04EB002080B210BDC4
:10E9380010B5FFF7F3FF0446FFF7F0FF04EB0040C4
:10E9480010BD38B5054D04462146286A00F023FC61
:10E95800EB6998796040987138BD00BF7C2500202C
:10E96800014BDB699879ECE77C25002038B5044633
:10E9780024200D46FFF7E5FF4D20FFF7E2FF002CAE
:10E98800084C14BF21203E20FFF7DBFFE36900227B
:10E9980028469A71FFF7D5FFE36993F84900BDE867
:10E9A8003840CEE77C25002001460020DEE710B580
:10E9B8000446C0B2FFF7C5FF200ABDE81040C0E713
:10E9C80010B5044680B2FFF7F2FF200CBDE81040F6
:10E9D800EDE737B582888368044610060D4641BFC7
:10E9E8002B4991F8A8174FF4CC7000FB0133D105DF
:10E9F80044BF2849097802F03F0244BF01EB4101B6
:10EA080003EB8103042A12D006D8012A0DD0022A6A
:10EA180032D193F9001030E0102A0AD0202A0AD007
:10EA2800082A29D1B3F9001027E0197825E01988B8
:10EA380023E0196821E093ED000A6846FAF744FAE2
:10EA480001461548FAF7C0FB05B3D4ED037A6846CA
:10EA5800B8EEE70AFAF738FA01461048FAF7B4FBB5
:10EA680094ED040A6846B8EEC00AFAF72DFA014692
:10EA78000A48FAF7A9FB09E000210948FAF7A4FBBC
:10EA880025B10848E1682269FAF79EFB03B030BD5A
:10EA9800401D00207C250020796801087268010863
:10EAA8005D710108B4720108024B0146586A00F012
:10EAB80072BB00BF7C25002010B5441E14F8011F4E
:10EAC80021B1034B586A00F066FBF7E710BD00BFA1
:10EAD8007C25002010B503781BB90A48BDE8104012
:10EAE800EAE704F057FD0446082899BF214606487E
:10EAF80006480821FAF768FB601EC0B2BDE810405E
:10EB0800F8F71EB9BB720108027301082E730108D9
:10EB18002DE9F3412B4E2C4B96F828002B4D1C6801
:10EB28002B4B05EB80001A882A4BD0F8C0101B78B5
:10EB3800294800914FF47A71B4FBF1F1FAF744FBDC
:10EB480026484821FAF740FB254BD3F800800027D8
:10EB5800FBB205EB8302D2F8D010E9B101249C4046
:10EB680014EA080F16D0220714D01E4AD25C0B20D4
:10EB780000FB0323154A1C4802EB8303D3F8F0205B
:10EB8800FAF722FB022C05D196F8341011B1174878
:10EB9800FAF71AFB0137DBE71548FFF78DFF154B2E
:10EBA80015481A68154B9A420CBF154B154B1A8815
:10EBB800154B198892B240F2DC7302B0BDE8F041FF
:10EBC800FAF702BB7C250020442A0020BC54010827
:10EBD800D811002008010020597301089C7301080E
:10EBE800940E002004010020AC730108B4730108DE
:10EBF800FC7301088C0E0020B87301080054004013
:10EC0800900E0020920E0020880E00202DE9F04181
:10EC18000024804625460F4EA7594146384604F041
:10EC2800A1FC58B139460C48FAF7CEFA3019002140
:10EC3800FFF7CFFE0948FFF73FFF0135143440F6D0
:10EC4800CC339C42E7D11DB90548BDE8F04133E714
:10EC5800BDE8F0815C5601080F690108FC730108E2
:10EC6800B36701082DE9F04F2DED028B83B00546FF
:10EC780004F039FC064620B1012818D12B782A2B3C
:10EC880015D15C48FFF718FF00245B4D5B486159BC
:10EC9800FAF79AFA28193146FFF79BFE5848FFF70A
:10ECA8000BFF143440F6CC339C42EED19CE028464E
:10ECB8003D2104F00AFC002800F08F8003469946A5
:10ECC80013F8012D202AFAD0441C204604F062FCD7
:10ECD80080462046FAF76EF8C5EB0909B0EE408A7F
:10ECE8000026DFF834A1142202FB06F40AF5D07BD3
:10ECF80054F80B70384604F0F6FB03461A462846CB
:10ED08003946019304F0F8FB019B00285BD15FFAB8
:10ED180089F29A4257D10AEB0402D2ED6B7AF8EEE7
:10ED2800E77A0BEB0405B4EEE78AF1EE10FA48DB5C
:10ED3800D2ED6C7AF8EEE77AB4EEE78AF1EE10FAE3
:10ED48003FD8B2F8A431D2F8A82113F0200F08BF99
:10ED580008EE108A1C0641BF2A4991F8A8174FF4FB
:10ED6800CC7404FB0122D90544BF2749097803F074
:10ED78003F0344BF01EB410102EB8102042B18EE73
:10ED8800100A0BD004D8013B012B0ED810700CE0F0
:10ED9800102B05D0202B06D0082B06D1108004E0BC
:10EDA80082ED008A01E082ED008A39461748FAF7B9
:10EDB8000BFA2846002103B0BDEC028BBDE8F04FEA
:10EDC80007E6134803E00136972E8AD1114803B0AD
:10EDD800BDEC028BBDE8F04F6EE6284603B0BDECF3
:10EDE800028BBDE8F04F11E703B0BDEC028BBDE824
:10EDF800F08F00BFEA7301085C5601080F6901082B
:10EE0800FC730108401D00207C250020FF730108C9
:10EE18000A740108B3670108BC54010810B50A4810
:10EE2800FFF74AFE094B5C6A204600F0ABF918B9B7
:10EE38000A2000F0EDF8F7E700F018FBFAF7EEFA11
:10EE4800034B044ADA6010BD2A7401087C250020AF
:10EE580000ED00E00400FA0508B50548FFF72CFEB0
:10EE6800FEF708FDFAF704FBBDE80840D6E700BF47
:10EE78003674010808B50448FFF71EFEFAF7F8FAD9
:10EE8800BDE80840CAE700BF4C7401084FF0904342
:10EE9800012208B19A6170471A8570474FF0904374
:10EEA800012208B11A8570479A61704710B54478F5
:10EEB8000078002202FB02F3193B634303F6C413F4
:10EEC800534340F6C411434393FBF1F3034921F83C
:10EED80012300132072AEDD110BD00BFCC25002029
:10EEE8000430114B33F91000B0F5617F10B506DB23
:10EEF80040F6330398420246A8BF1A4601E04FF491
:10EF080061720C78192340F2833013FB0404944295
:10EF180007DA497813FB01039342B4BF00200120AC
:10EF280010BD002010BD00BF821C002010B500F1EC
:10EF3800500302788A4203D18478C278944204D379
:10EF480004309842F5D1002010BD012010BD0B4BB4
:10EF58001B6813F4805F0A4BB3F9063005D0C089EB
:10EF6800421A934207DD084400E0008A8342B4BF96
:10EF78000020012070470120704700BF382A002078
:10EF8800821C00201FB5094B1B681B030AD58DF88E
:10EF9800040001230D2001A98DED030A8DF8053029
:10EFA800FBF7FEFD05B05DF804FB00BF382A002022
:10EFB8001FB5084B1B681B0309D58DF80400029187
:10EFC80000230D2001A98DF80530FBF7E9FD05B0F8
:10EFD8005DF804FB382A002010B50A4A0A4B11686C
:10EFE8009B6800BF12689142F7D1084A14694FF430
:10EFF8007A7000FB04F2D31AB3FBF4F300FB013080
:10F0080010BD00BF442A002010E000E0CC250020FD
:10F0180038B5044654B1FFF7DFFF0546FFF7DCFFBC
:10F02800401BB0F57A7FF9D3013CF3E738BD024ABB
:10F038001368013313607047442A0020024B5B6950
:10F0480003B11847704700BFCC250020014B1B684F
:10F05800184700BF802A002010B50020FFF7F6FFF0
:10F06800054B00241C7001F03DF9044B1C76DC6153
:10F078001C845C6210BD00BF6C2A0020CC250020D7
:10F0880010B510B9BDE81040E6E700230C225A433A
:10F098000A4C1119125D824203D00133102BF5D1AD
:10F0A80010BD074B586A18B14A784078824203D29B
:10F0B800002259621A84DA6110BD00BFBC540108ED
:10F0C800CC25002010B540001428A8BF1420002328
:10F0D800074A022199540B4499181424834201F8D1
:10F0E800014CF5DBFF21D1540F20BDE81040C7E7E4
:10F0F800B42500202DE9F84307460B24013C35D000
:10F108001D4B20229A617D1C32264FF00508DFF83E
:10F118006890B9F814309BB283F02003A9F8143032
:10F128000120FFF793FF3046FFF772FFB9F814305C
:10F138009BB283F020030020A9F81430FFF786FF64
:10F148003046FFF765FFB8F1000F08D0B8F10108A5
:10F15800DDD14FF4FA70FFF75BFFFA26D7E7013DE0
:10F16800D5D14FF47A70FFF753FFC7E7034B044A32
:10F17800DA60BDE8F88300BF0004004800ED00E055
:10F188000400FA0503681B69184703689B68184759
:10F1980003685B68184703681B6818472DE9F84F30
:10F1A800B0F90230934218BF00232DED048B18BF2D
:10F1B8000370057804460E469146002D40F097806E
:10F1C80007EE902ADFED7D8AF8EEE77AB6EE009A30
:10F1D80067EEA88ADFED7A7A68EEA78AA04668EE1D
:10F1E800898A2746B0EE680AFAF780F8B0EE408AB6
:10F1F800B0EE680AFAF7DAF888EE000A40F2DC5353
:10F2080063651023A4F852301823A4F85030DFEDBA
:10F218006D6A60EE266AB7EE006AB0EE667AA0EE16
:10F22800007AD0EE006A37EE067A76EE866AC6EE87
:10F23800077A84ED046A27EE807AB0EE498A27EED1
:10F24800007A77EE075A84ED017AC4ED025A70EE1F
:10F25800005A84ED037AB8EE007AA5EE807A27EE9C
:10F26800877A67EEA67A84ED057AC4ED067ADFED33
:10F27800567A98ED047A27EE277AF0EE678AB5EE8B
:10F28800C07AF1EE10FA4CBF77EE487A77EE087A3A
:10F29800013517EE900A01F089FAD8ED017A67EE88
:10F2A800A87AC7E90E01F5EEC07AF1EE10FA4CBF64
:10F2B80077EEC87A77EE887A08F1040817EE900A94
:10F2C80001F074FA032DC7E9080107F10807CED148
:10F2D800A6F2DC531B042367E3676367C4F8803036
:10F2E800A367C4F884300123A4F802902370D4F8EB
:10F2F8005490B4F95280636A276A206FE26FD4F899
:10F3080040C0D4F88010C4F88020C9EB060606FA7D
:10F3180008F64FEAE67B734307FB0B332667A7FB28
:10F3280006671F44636C656F60674FEAE27B53436F
:10F338000CFB0B3EACFB02237344B61A67EB0307C6
:10F34800E36AA26AC4F884104FEAE07B434302FBF5
:10F358000B3EA2FB00237344B6185F41E36CA06C1C
:10F36800B4F95020A5674FEAE17B4B4300FB0B3310
:10F37800A0FB01011944636B361A206B4FEAE57B49
:10F3880005FB03F300FB0B3367EB0107A0FB05014B
:10F3980019448019794100F0D7FF08F1FF320123A1
:10F3A8009340E067C01841EBE371424600F0CCFFA0
:10F3B800BDEC048B4844BDE8F88F00BF6F12833A58
:10F3C800DB0F4940F404B53F0000804B2DE9F843BA
:10F3D8000024234B93F85860E0B2B0420CD203EB00
:10F3E8008003204A9B6A32F810101BB10B2801D801
:10F3F800DB6898470134ECE71B4B1B685B032DD592
:10F4080000242346E2B2B24228D2DFF8549009F130
:10F4180028074FEA840857F8242055689D4215D0DC
:10F428002846FEF773F9EFF31283502282F312880D
:10F4380028216A6A01FB00900132C0F880206A69BD
:10F4480042F001026A61DBB283F3118857F8083091
:10F458001B6800221A6001342B46D3E7BDE8F88305
:10F46800CC250020DC0E0020382A002008B50E4BE1
:10F478001B6813F4805F0D4B14BFD3F82421D3F815
:10F48800282193F8581092880023D8B2884204D2D1
:10F49800074820F813200133F7E7FFF797FF3220DA
:10F4A800BDE80840B4E500BF382A0020CC2500207C
:10F4B800DC0E00200A4B1A680A4B30B502F4805261
:10F4C800D3F82441D3F8285100230AB1A18800E0D9
:10F4D800A988054820F8131001330C2BF5D130BD4D
:10F4E800382A0020CC2500207E25002070B5124D3A
:10F4F8000024214605F22D10702285F82C4103F0D6
:10F50800AEFF2146D5F8A0310B4A0B4493F902000F
:10F5180080B102F22D141E680E5108199C8884804F
:10F528009B79837192F82C3107310133702982F865
:10F538002C31E7D170BD00BFCC250020094B1A68DB
:10F548000E2303FB0020437AFF2B07D0064A1278CC
:10F558009A4203D9054A32F8130000E0808800B2C5
:10F56800704700BF8812002020250020821C002040
:10F57800D0ED024A91ED016A90ED015A91ED027ABF
:10F58800D0ED005AD1ED007A66EE646AE5EE076ABE
:10F5980027EE657AC2ED006AA4EEA77A67EEC57A0F
:10F5A80082ED017AE5EE867AC2ED027A7047D0EDF7
:10F5B800017A91ED017AD1ED026A91ED006A37EE98
:10F5C800877AD0ED027A77EEA67AD0ED006A82EDDE
:10F5D800017A76EE866AC2ED027AC2ED006A704759
:10F5E80090ED017AD0ED027AD0ED006A20EE077A2C
:10F5F80060EE277A26EE800A81ED017A81ED000A15
:10F60800C1ED027A704700BF054B1968054B4A8A5D
:10F6180018B99B889B1A0B8270471868104470476A
:10F628007C1C0020C8000020074B1B681B7803F0D7
:10F638007F03212B06D100F0DF00022814BF02202F
:10F6480000207047022070477C1C0020212810B53C
:10F6580008D1114B1B681B7803F07F03212B10D0B6
:10F66800022010BD2028FBD10B4B0C4A1B681070E0
:10F678001B7803F07F03212B094B18BF00230BB91C
:10F68800EEE7084B044A126800249361548220462E
:10F698009847204610BD00BF7C1C00209A2A0020F5
:10F6A80001E1000819E100087047034B1A78202A85
:10F6B80004BF00221A7070479A2A0020014B0422C6
:10F6C8001A6070477C2A0020034B9B7A13B1034BC6
:10F6D80005221A60704700BF5C2500207C2A0020A4
:10F6E8000D4B0E491A680E4B92B213445B000D4A3B
:10F6F8001B68C3F3090310B5136013689BB2013389
:10F708005B1000229A4206D0074851F8044B20F8B3
:10F7180012400132F6E710BD505C00402062004004
:10F728001E3000207027002074270020014B002283
:10F738005A647047702700202DE9F843664B674EDE
:10F748001B68DFF8B881664A00254FF0C0099D7232
:10F7580083F80990DD723560D8F8003023F4EC4363
:10F7680023F0700343F400739BB2C8F80030D8F854
:10F77800003023F4E04323F040039BB248F28004B6
:10F7880083F010032343C8F80030336812FA83F378
:10F798005B0040271A681F6033689BB203F100536F
:10F7A80003F540535B0028461A6880221A60D8F88F
:10F7B800003023F4F8731B051B0D2343C8F80030F1
:10F7C800484B93F83410F6F7EFFAD8F80030464A69
:10F7D800464923F4804323F070039BB283F44053DB
:10F7E8002343C8F80030136823F4EC4323F0700374
:10F7F8009BB21360336811FA83F35B000320196826
:10F80800C3F8009013683A4923F4E04323F0400317
:10F818009BB283F0200323431360136823F48043CF
:10F8280023F0700323439BB21360536823F4EC4323
:10F8380023F0700343F4C0639BB25360336811FA3A
:10F8480083F35B0019684FF480711960536823F4DF
:10F85800804323F0700323439BB25360536823F41F
:10F86800E04323F040039BB283F02003234353601B
:10F87800D8F80C301F4A23F4EC4323F070039BB2F2
:10F88800C8F80C30336812FA83F35B0039461A68FB
:10F898004FF488721A60F6F787FAD8F80C3023F418
:10F8A800804323F070039BB283F440532343C8F88A
:10F8B8000C30D8F80C3023F4E04323F040031C4309
:10F8C800A4B2C8F80C402846FCF7CFFD0A4B012229
:10F8D8001A60BDE8F88300BF7C1C0020505C004023
:10F8E80004300020C8000020045C004008300020DC
:10F8F800103000201C3000207C2A0020005C0040D2
:10F90800134A144B50681B68181810B5146808D0AF
:10F9180011490822FCF795FD204610490422FCF7FE
:10F9280090FD0F4B1A68002393720E4A0121116053
:10F938000D4913604FF4E0500B6010600B480B60EA
:10F948004FF43641A0F848101160094A136010BD01
:10F95800B0F7FF1FACF7FF1FAA000020BA00002075
:10F968007C1C0020405C0040445C00407027002064
:10F978007C2A0020024B4FF480221A60704700BF97
:10F98800140401402DE9F04FAB490B7813F0010F37
:10F9980085B003F0040200F03E81002A40F048815F
:10F9A800A648076817F0806740F04281980700F181
:10F9B800328143F004030B70A14BA24C1B882380B7
:10F9C800A14BA24D1A6812F4002F984600F013813B
:10F9D8009F4B80201F70FEF725FE08B1FEF774FFCD
:10F9E800A678012E40F0078195F8CE272AB1974BCB
:10F9F80093F8CF370BB19A4203D3012385F8CE375A
:10FA08000FE01846114630B191FBF0FE00FB1E1EB8
:10FA180001467046F7E792FBF1F285F8CE2793FB93
:10FA2800F1F385F8CF3795F8D037012B82BF874B94
:10FA3800002283F8D027874B95F8D0971B6841F6AA
:10FA4800690203EBC303934284BF40F2E242B3FB73
:10FA5800F2F3814A8CBFDBB204231370B9F1000FB3
:10FA680003D0B9F1010F1FD024E08020F7F7BCFBC9
:10FA78008246F8B18021F7F791FB9AF80620774B78
:10FA8800E07053F822309AF90000B3F5613F0CBFDB
:10FA98000222002202218DE8060080214A46F7F75B
:10FAA800C7F9606040B905E06D4BDB6813B1FEF73C
:10FAB800BFF908B100239DE000211422694803F032
:10FAC800CEFC694BE36103F16C02D8336362674B88
:10FAD800D8F800101B88A4F86C3195F8923195F885
:10FAE800CE97634895F884A12262002B6B79039026
:10FAF800A3F1190CC1F3C03818BF4FF00108DCF1AD
:10FB0800000E4EEB0C0E012B95F8CF37D0F800C045
:10FB180008BF4FF0010E9945564B1B780293C1F36D
:10FB2800400B28BF4FF0000901F4006138BF4FF0C7
:10FB38000109721ED2B2531E132B37D8DFE803F027
:10FB48000C0C0C0C0C0C0C0C0A3939722939741277
:10FB580012123339734668E0029B9342B4BF002304
:10FB6800012322E09CF80030022B0BD10CEB82031E
:10FB780053ED027AF5EE407AF1EE10FA14BF012344
:10FB8800002312E00CEB02035B79003318BF01235A
:10FB98000BE021B10AF1FF304342434100E00B463C
:10FBA80003F0010341E04B463FE013B101239340CA
:10FBB8001F43142E02D80136F6B2BAE7039BC4F8E5
:10FBC8007071186819218530FFF7B0F90023C4F85F
:10FBD8007831A4F87C31A4F87E31C4F88831264BFA
:10FBE800D4F884211B68C4F88C3184F87401C4F8F3
:10FBF80080210223A370204B95F8E0211B684FF465
:10FC08007A7101FB02331D4A0520136005B0BDE877
:10FC1800F04FFFF735BA5AB9012005B0BDE8F04FEB
:10FC2800FFF750BA5B4600E04346002BBED1C2E75F
:10FC380005B0BDE8F08F00BF942A00209C0E00207C
:10FC4800F80E0020BC270020382A0020401D002084
:10FC580025250020000F002009010020FC53010881
:10FC68000C000020C4270020E42700204C110020AD
:10FC7800D80E002024260020442A0020F40D00205D
:10FC880010B5154A1378590725D523F004031370C6
:10FC9800124B1B681B0319D5114CA378A3F108025A
:10FCA800012A0BD8FF200021FAF77AFF0D4B1B68B9
:10FCB800C4F88C31FEF7ECF80A2306E0012B05D9CD
:10FCC8000A2B03D0FEF7CAF80123A3700420BDE86D
:10FCD8001040FFF7D5B910BD942A0020382A00201B
:10FCE800BC270020442A00202DE9F04F2DED088B79
:10FCF800CB4D83B0044601932B8813F0020F0AEE14
:10FD0800102AF7EE009A4CD0149BC648DE89B0F949
:10FD180000309B1B03F2F31740F2E632974203D8F8
:10FD2800002BB8BF5B4201E04FF4FA73B0F9022030
:10FD3800921B02F2F31640F2E630864203D8002AFC
:10FD4800B8BF524201E04FF4FA7294F84C0058B32D
:10FD58009342B8BF1346C3F5FA7307EE903A9FED86
:10FD6800B27AF8EEE77A6423C7EE877A93FBF0F36A
:10FD780007EE103A77EEE97AB8EEC77AB0EE699AEC
:10FD8800A7EE879AF7EE006AB5EEC09AF1EE10FA80
:10FD98000AD4B4EE669AF1EE10FAC8BFB0EE669ACD
:10FDA80004E0B0EE699A01E09FEDA09AA04E01F13F
:10FDB8000308A3464FF0000ABAF1020F18F8010F22
:10FDC8009C4F4FEA4A09F2EE04AA0ED100F10A014B
:10FDD800B7F904009FED987A00FB01F307EE903A1B
:10FDE800F8EEE77AC7EE877A51E0B8EE4A7ADFEDA7
:10FDF8008E6A37F91A1087EE267A07EE901A1AEEED
:10FE0800103AF8EEE77A5B4227EE877A07EE903AE7
:10FE1800F8EEE77AB4EEE77AF1EE10FA08D4F8EEE5
:10FE2800CA7AB4EEE77AF1EE10FAD8BFF0EE477A64
:10FE3800824F37F909302F8807EE103A019BB8EE48
:10FE4800C77A33F91A3077EEC77A07EE103AB8EE68
:10FE5800C77AFB0737EE877A87EE2A7A04D5D4ED7E
:10FE6800117A67EE277A12E0143001FB00F307EEEF
:10FE7800903ADFED716AF8EEE77AB907C7EEA67A2D
:10FE880042BFD4ED126A27EE267AE7EE097A6C496A
:10FE98006C4F31F909306C499BED08BAD1ED046A11
:10FEA8009FED6A8A07EE103AB8EEC77A684BE7EE1C
:10FEB800667A1AF80330BAF1020FF0EE678A67EE35
:10FEC8008B7A0BEE103AB8EECBBAF0EE48BA27EEC2
:10FED8008BBA8BEE08BA09D1B0EE4B0A5D48D7ED64
:10FEE800000A1E21F8F73CFFB0EE40BAD7ED000A31
:10FEF8009BED0B7A68EEA07A67EE877A96ED007A2A
:10FF0800A7EEAA7ADFED547AB4EEE77AF1EE10FAAA
:10FF1800F0EE47AA09D4DFED517AB4EE677AF1EE34
:10FF280010FAC8BFF0EE67AA01E0F0EE67AA89EE02
:10FF3800A08A4B494FEA8A07394491ED000AC6ED79
:10FF480000AAC1ED008A38EEC00A94F8501020EEDD
:10FF5800080A21B1434800EBCA00F8F701FF3C4BFF
:10FF6800DBED0E7A13F80A3060EE277A00EE103ACD
:10FF7800B8EEC00A27EE800ADFED3B7A80EE2B8AC6
:10FF8800B4EEE78AF1EE10FA09D4DFED387AB4EE70
:10FF9800678AF1EE10FAC8BFB0EE678A01E0B0EEEA
:10FFA800678A3BEE2A0A30EE080A03F067FC3049FC
:10FFB800B0F57A7FA8BF4FF47A708842B8BF084678
:10FFC8002C4921F8090029880A0507D52A49097802
:10FFD8004B0703D55FFA8AF0F8F728FDBDEECBBAD8
:10FFE80026491BEE103AFDEEEAAA7B50BDEEC88A00
:08FFF80023491AEE903A0AF1C8
:020000040801F1
:10000000010A7B50214918EE103ABAF1030F7B50D8
:100010000BF1040B06F104067FF4D2AE03B0BDEC85
:10002000088BBDE8F08F00BF980E0020821C0020D6
:100030000000FA4300000000EC1200203C190020F0
:1000400000004842F40E0020C20E0020501900208B
:10005000B01900200000C8424419002048190020AF
:1000600000007AC300007A43502900206C19002058
:10007000000096C30000964318FCFFFF841900207F
:10008000942A00208C19002098190020A41900201F
:10009000044B00221A605A60034B00221A605A6017
:1000A000704700BF18130020F812002010B50B4C49
:1000B0000123E3704FF48060022384F82030F9F7C5
:1000C00091F9074A074BD2681B685178642212FBEA
:1000D0000133636123880133238010BD482A002047
:1000E00050290020442A00200A4BDFED0B7A53F8F8
:1000F000213007EE103AB8EE477AF6EE046AE7EEE2
:10010000267A82B0FCEEE77ACDED017ABDF80400E4
:1001100002B070476029002000005C44024B03EBF2
:100120004101B1F84800704760290020024B03EB01
:100130004101B1F86C00704760290020024B03EBCD
:100140004101B1F86C007047602900200020704721
:1001500038B50446FEF744FF274A2749D2F88430D1
:10016000C2F88400C31AB3F57A6F84BF002382F803
:10017000883092F8883033B9A82C3BD181F8893087
:10018000A1F88A3006E0022B02D181F88C4001E010
:10019000242B02D8D11881F88D4092F88C10164D7E
:1001A00001330231DBB249008B4282F8883018DA21
:1001B000B5F88A30E0B283EA0020082310F4004F3B
:1001C0004FEA400018BF80F4815003F1FF3318BF9D
:1001D00080F0010013F0FF0380B2EFD1A2F88A0093
:1001E00038BD01318B4201BF002385F888300123DF
:1001F00085F8893038BD00BF6029002010B504465D
:10020000FEF7EEFE104AD2F8B43040F6AC51C31AF5
:100210008B42C4BF002382F8B83092F8B830D118AE
:1002200081F8B94023B90F2C0DD10749C1F8B400AA
:100230000133DBB2192B044982F8B8300CBF01231B
:10024000002381F8D23010BD60290020104910B57C
:10025000D1F8D43003EB4002147E2CB1022C0DD027
:100260000C4B33F8100010BD032805D1D1F8D8206D
:10027000D20401D4988A10BDD88910BD507E00EBFD
:10028000800000EB800000F2EE2080B210BD00BFC5
:1002900060290020821C002008B5FEF7A1FE074B54
:1002A000022283F8E020D3F8E420C3F8F0200122F2
:1002B000C3F8DC0083F8092108BD00BF60290020D5
:1002C00008B5FEF78DFE084B022283F8E020D3F834
:1002D000F02000F5B71000F5587002F2DC52C3F8B8
:1002E000DC00C3F8F02008BD60290020104B93F813
:1002F0000C21012A10B51C460DD008D3022A0DD1BD
:100300000C4A938A9BB283F02003938206E0094B48
:1003100020229A6102E0074B20221A85FEF760FE38
:1003200000F5F42000F59070C4F8100110BD00BF76
:10033000602900200004004808B5044B1B7803F036
:100340000503052B01D1FFF795F8FEE7742A00207D
:10035000D0400B1C1141203A03D49C461341184352
:100360006346524293401843704700BF81F00041FA
:1003700002E000BF83F0004330B54FEA41044FEA8A
:10038000430594EA050F08BF90EA020F1FBF54EA25
:10039000000C55EA020C7FEA645C7FEA655C00F0C1
:1003A000E2804FEA5454D4EB5555B8BF6D420CDD92
:1003B0002C4480EA020281EA030382EA000083EA15
:1003C000010180EA020281EA0303362D88BF30BDB5
:1003D00011F0004F4FEA01314FF4801C4CEA11310B
:1003E00002D0404261EB410113F0004F4FEA03336A
:1003F0004CEA133302D0524263EB430394EA050FF5
:1004000000F0A780A4F10104D5F1200E0DDB02FA63
:100410000EFC22FA05F2801841F1000103FA0EF2F7
:10042000801843FA05F359410EE0A5F120050EF1BD
:10043000200E012A03FA0EFC28BF4CF0020C43FAEE
:1004400005F3C01851EBE37101F0004507D54FF0FB
:10045000000EDCF1000C7EEB00006EEB0101B1F54B
:10046000801F1BD3B1F5001F0CD349085FEA300091
:100470004FEA3C0C04F101044FEA445212F5800F9C
:1004800080F09A80BCF1004F08BF5FEA500C50F139
:10049000000041EB045141EA050130BD5FEA4C0C1C
:1004A000404141EB010111F4801FA4F10104E9D1A5
:1004B00091F0000F04BF01460020B1FA81F308BF9C
:1004C0002033A3F10B03B3F120020CDA0C3208DD68
:1004D00002F1140CC2F10C0201FA0CF021FA02F143
:1004E0000CE002F11402D8BFC2F1200C01FA02F1B3
:1004F00020FA0CFCDCBF41EA0C019040E41AA2BFD8
:1005000001EB0451294330BD6FEA04041F3C1CDA9F
:100510000C340EDC04F11404C4F1200220FA04F0BF
:1005200001FA02F340EA030021FA04F345EA030169
:1005300030BDC4F10C04C4F1200220FA02F001FA2B
:1005400004F340EA0300294630BD21FA04F02946AD
:1005500030BD94F0000F83F4801306BF81F4801146
:100560000134013D4EE77FEA645C18BF7FEA655CB9
:1005700029D094EA050F08BF90EA020F05D054EA8B
:10058000000C04BF1946104630BD91EA030F1EBF90
:100590000021002030BD5FEA545C05D14000494194
:1005A00028BF41F0004130BD14F580043CBF01F587
:1005B000801130BD01F0004545F0FE4141F470016D
:1005C0004FF0000030BD7FEA645C1ABF1946104648
:1005D0007FEA655C1CBF0B46024650EA013406BF49
:1005E00052EA033591EA030F41F4002130BD00BF08
:1005F00090F0000F04BF0021704730B54FF48064C5
:1006000004F132044FF000054FF0000150E700BF45
:1006100090F0000F04BF0021704730B54FF48064A4
:1006200004F1320410F0004548BF40424FF0000191
:100630003EE700BF42004FEAE2014FEA31014FEAD4
:1006400002701FBF12F07F4393F07F4F81F0605123
:10065000704792F0000F14BF93F07F4F704730B592
:100660004FF4607401F0004521F0004120E700BF25
:1006700050EA010208BF704730B54FF000050AE0AC
:1006800050EA010208BF704730B511F0004502D5AD
:10069000404261EB41014FF4806404F132045FEAAF
:1006A000915C3FF4DCAE4FF003025FEADC0C18BF54
:1006B00003325FEADC0C18BF033202EBDC02C2F14A
:1006C000200300FA03FC20FA02F001FA03FE40EADC
:1006D0000E0021FA02F11444C1E600BF4FEA4102C4
:1006E000B2F1E04324BFB3F5001CDCF1FE5C0DD990
:1006F00001F0004C4FEAC0024CEA5070B2F1004FDA
:1007000040EB830008BF20F00100704711F0804FDC
:1007100021D113F13872BCBF01F00040704741F4A1
:1007200080114FEA5252C2F11802C2F1200C10FAA5
:100730000CF320FA02F018BF40F001004FEAC12389
:100740004FEAD32303FA0CFC40EA0C0023FA02F32D
:100750004FEA4303CCE77FEA625307D150EA013303
:100760001EBF4FF0FE4040F44000704701F00040D3
:1007700040F0FE4040F40000704700BF7BB972B902
:100780000029BEBF00204FF0004106E008BF00284E
:100790001CBF6FF000414FF0FF3000F073B882B023
:1007A000EC462DE9005000F03DF8DDF804E002B021
:1007B0000CBC704707EE900AF5EEC07AF1EE10FA25
:1007C00001D400F009B808B580F0004000F004F84A
:1007D000404261EB410108BDD0B5FFF72BFF00227D
:1007E0000E4B06460F4600F04FF800F05FFA044645
:1007F000FFF7FEFE00220A4B00F046F802460B46C9
:1008000030463946FFF7B6FD00F050FA2346002285
:1008100042EA000210461946D0BD00BF0000F03D7C
:100820000000F0412DE9F041069C154606460F46B2
:10083000984600F05BFA05FB01F300FB0838A5FBC6
:100840000023B21A434467EB0303C4E90023BDE865
:10085000F08100BF2DE9F041069C904606460F4608
:100860001D4600F091FB00FB05F5A0FB082308FBEB
:100870000155B21A2B4467EB0303C4E90023BDE81A
:10088000F08100BF704700BF70B54FF0FF0C4CF413
:10089000E06C1CEA11541DBF1CEA135594EA0C0FBE
:1008A00095EA0C0F00F0DEF82C4481EA030621EAF9
:1008B0004C5123EA4C5350EA013518BF52EA033534
:1008C00041F4801143F4801338D0A0FB02CE4FF0E6
:1008D0000005E1FB02E506F00042E0FB03E54FF016
:1008E0000006E1FB03569CF0000F18BF4EF0010E0E
:1008F000A4F1FF04B6F5007F64F5407404D25FEA0A
:100900004E0E6D4146EB060642EAC62141EA5551BC
:100910004FEAC52040EA5E504FEACE2EB4F1FD0CFE
:1009200088BFBCF5E06F1ED8BEF1004F08BF5FEA7C
:10093000500E50F1000041EB045170BD06F000462E
:1009400046EA010140EA020081EA0301B4EB5C04DB
:10095000C2BFD4EB0C0541EA045170BD41F48011D3
:100960004FF0000E013C00F3AB8014F1360FDEBFF8
:10097000002001F0004170BDC4F10004203C35DAD4
:100980000C341BDC04F11404C4F1200500FA05F357
:1009900020FA04F001FA05F240EA020001F00042F8
:1009A00021F0004110EBD37021FA04F642EB06016E
:1009B0005EEA430E08BF20EAD37070BDC4F10C0498
:1009C000C4F1200500FA04F320FA05F001FA04F25C
:1009D00040EA020001F0004110EBD37041F1000148
:1009E0005EEA430E08BF20EAD37070BDC4F1200553
:1009F00000FA05F24EEA020E20FA04F301FA05F2BB
:100A000043EA020321FA04F001F0004121FA04F262
:100A100020EA020000EBD3705EEA430E08BF20EA32
:100A2000D37070BD94F0000F0FD101F0004640006C
:100A300041EB010111F4801F08BF013CF7D041EAEE
:100A4000060195F0000F18BF704703F000465200F2
:100A500043EB030313F4801F08BF013DF7D043EAC3
:100A60000603704794EA0C0F0CEA135518BF95EA79
:100A70000C0F0CD050EA410618BF52EA4306D1D100
:100A800081EA030101F000414FF0000070BD50EA1F
:100A9000410606BF1046194652EA430619D094EAA9
:100AA0000C0F02D150EA013613D195EA0C0F05D193
:100AB00052EA03361CBF104619460AD181EA0301E7
:100AC00001F0004141F0FE4141F470014FF000009F
:100AD00070BD41F0FE4141F4780170BD70B54FF03A
:100AE000FF0C4CF4E06C1CEA11541DBF1CEA1355BA
:100AF00094EA0C0F95EA0C0F00F0A7F8A4EB05049C
:100B000081EA030E52EA03354FEA013100F0888092
:100B10004FEA03334FF0805545EA131343EA12635B
:100B20004FEA022245EA111545EA10654FEA002610
:100B30000EF000419D4208BF964244F1FD0404F5C9
:100B4000407402D25B084FEA3202B61A65EB030525
:100B50005B084FEA32024FF480104FF4002CB6EBE2
:100B6000020E75EB030E22BFB61A754640EA0C0062
:100B70005B084FEA3202B6EB020E75EB030E22BFA2
:100B8000B61A754640EA5C005B084FEA3202B6EBE3
:100B9000020E75EB030E22BFB61A754640EA9C00A2
:100BA0005B084FEA3202B6EB020E75EB030E22BF72
:100BB000B61A754640EADC0055EA060E18D04FEA30
:100BC000051545EA16754FEA06164FEAC30343EAD0
:100BD00052734FEAC2025FEA1C1CC0D111F4801F9D
:100BE0000BD141EA00014FF000004FF0004CB6E796
:100BF00011F4801F04BF01430020B4F1FD0C88BF35
:100C0000BCF5E06F3FF6AFAEB5EB030C04BFB6EB3F
:100C1000020C5FEA500C50F1000041EB045170BD32
:100C20000EF0004E4EEA113114EB5C04C2BFD4EB5F
:100C30000C0541EA045170BD41F480114FF0000EE3
:100C4000013C90E645EA060E8DE60CEA135594EA5F
:100C50000C0F08BF95EA0C0F3FF43BAF94EA0C0F62
:100C60000AD150EA01347FF434AF95EA0C0F7FF4D7
:100C700025AF104619462CE795EA0C0F06D152EA2B
:100C800003353FF4FDAE1046194622E750EA41060F
:100C900018BF52EA43067FF4C5AE50EA41047FF420
:100CA0000DAF52EA43057FF4EBAE12E74A0011D2D2
:100CB00012F5001211D20DD56FF47873B3EB6252B6
:100CC0000ED44FEAC12343F0004343EA505323FAC2
:100CD00002F070474FF00000704750EA013002D137
:100CE0004FF0FF3070474FF00000704700292DE9AA
:100CF000F043C0F2A6800026002BC0F29C808846FC
:100D000094469E46154604460F46002B3DD18A4226
:100D100059D9B2FA82F33BB1C3F120029F4020FAC5
:100D200002F29D4017439C40290C220CB7FBF1FEB8
:100D3000A8B201FB1E7742EA074700FB0EF3BB4255
:100D40000AD97F190EF1FF3280F00581BB4240F2D3
:100D50000281AEF1020E2F44FF1AA4B2B7FBF1F3E9
:100D600001FB137744EA074700FB03F0B84208D9B8
:100D70007F1903F1FF3280F0F080B84240F2ED803D
:100D8000023B43EA0E43002203E08B420FD90022CC
:100D90001346341C18BF012460424FF0000565EB78
:100DA00045015840514000196941BDE8F083B3FA4C
:100DB00083F2002A40F086808B4202D3844500F201
:100DC000DB800123E5E712B90123B3FBF2F5B5FAA5
:100DD00085F000283BD1781B4FEA154E1FFA85FCA1
:100DE0000122B0FBFEF8210C0EFB180741EA074771
:100DF0000CFB08F3BB4207D97F1908F1FF3102D27F
:100E0000BB4200F2BD808846FF1AA4B2B7FBFEF3D6
:100E10000EFB137744EA07470CFB03FCBC4507D9DC
:100E20007F1903F1FF3102D2BC4500F2A7800B46C7
:100E300043EA0843ADE752426FEA060663EB430319
:100E40005DE7404261EB41014FF0FF3654E7C0F1EE
:100E5000200224FA02F107FA00F385404FEA154E0A
:100E6000D7401943B7FBFEF20B0C0EFB12771FFAAB
:100E700085FC43EA07430CFB02F79F4204FA00F4A7
:100E800007D95B1902F1FF3074D29F4272D9023A3E
:100E90002B44DF1B89B2B7FBFEF80EFB187341EA47
:100EA00003430CFB08F79F4208D95B1908F1FF3197
:100EB0005CD29F425AD9A8F102082B44D81B48EAB9
:100EC00002428EE7C2F120032CFA03F10EFA02FE71
:100ED00020FA03F741EA0E0E08FA02F028FA03F1AD
:100EE0004FEA1E453843B1FBF5F8030C05FB18111A
:100EF0001FFA8EF743EA014107FB08F38B420CFA15
:100F000002FC09D911EB0E0108F1FF3930D28B42F6
:100F10002ED9A8F102087144C91A80B2B1FBF5F3C9
:100F200005FB131140EA014107FB03F78F4208D983
:100F300011EB0E0103F1FF3016D28F4214D9023BA0
:100F4000714443EA0843C91BA3FB0C89494509D3F3
:100F500005D000221DE79646FEE6134611E79440B1
:100F60004445F6D2013BF4E70346EAE78846A5E7A5
:100F7000C846D1E702468CE713460AE7023B57E72B
:100F8000A8F102082F443FE72DE9F041002B44D19E
:100F90008A42154604464FD9B2FA82F70E464FB13F
:100FA000C7F12003B94020FA03F602FA07F50E4311
:100FB00000FA07F44FEA154E230CB6FBFEF0AFB271
:100FC0000EFB106143EA014307FB00F1994209D986
:100FD0005B1900F1FF3280F0EC80994240F2E98029
:100FE00002382B445A1AA4B2B2FBFEF30EFB1322B2
:100FF00044EA024207FB03F7974208D9521903F16A
:10100000FF3180F0D880974240F2D580023B43EA1E
:10101000004000263146BDE8F0818B4247D8B3FA44
:1010200083F6002E48D18B4202D3824200F2CD805B
:1010300001203146BDE8F08112B90125B5FBF2F57A
:10104000B5FA85F8B8F1000F77D14A1B4FEA154E73
:10105000AFB20126B2FBFEF0230C0EFB102143EAD7
:10106000014107FB00F38B4207D9491900F1FF3218
:1010700002D28B4200F2BA801046C91AA4B2B1FB68
:10108000FEF30EFB131144EA014407FB03F7A742EA
:1010900008D9641903F1FF3280F08F80A74240F233
:1010A0008C80023B43EA00403146BDE8F0810026D7
:1010B00030463146BDE8F081C6F1200422FA04F53D
:1010C000B3402B4320FA04FC01FA06F721FA04F599
:1010D0004FEA134E4CEA0707B5FBFEF8390C0EFB3E
:1010E00018551FFA83FC41EA05450CFB08F1A9429B
:1010F00002FA06F204D9ED1808F1FF3467D3A046CE
:101100006D1ABFB2B5FBFEF40EFB145547EA05415C
:101110000CFB04FC8C4504D9C91804F1FF355CD3E1
:101120002C4644EA0844CCEB0101A4FB022399427B
:1011300048D344D0204600266CE7C8F1200401FAC9
:1011400008F305FA08F520FA04F7E1404FEA154ED6
:101150001F43B1FBFEF63A0C0EFB16111FFA85FC7D
:1011600042EA01430CFB06F29A4200FA08F407D95E
:101170005B1906F1FF3137D29A4235D9023E2B4432
:101180009B1ABFB2B3FBFEF00EFB103347EA0343DA
:101190000CFB00F1994207D95B1900F1FF3221D213
:1011A00099421FD902382B445A1A40EA064667462C
:1011B00050E7104616E70B4629E7134672E7B040A2
:1011C0009042B7D2601E002624E7304622E7A942AB
:1011D00095D9A8F102081D4492E78C45A0D9023C9C
:1011E00019449EE71046DFE70E46C9E70238294456
:1011F00043E700BF4FF0FF3C06E000BF4FF0010C9B
:1012000002E000BF4FF0010C4DF804CD4FEA410C55
:101210007FEA6C5C4FEA430C18BF7FEA6C5C1BD022
:1012200001B050EA410C0CBF52EA430C91EA030FA3
:1012300002BF90EA020F0020704710F1000F91EA00
:10124000030F58BF994208BF90422CBFD8176FEACE
:10125000E37040F0010070474FEA410C7FEA6C5C9C
:1012600002D150EA013C07D14FEA430C7FEA6C5CA3
:10127000D6D152EA033CD3D05DF8040B704700BFCF
:101280008446104662468C461946634600E000BF1D
:1012900001B5FFF7B7FF002848BF10F1000F01BDEF
:1012A0004DF808EDFFF7F4FF0CBF012000205DF8BA
:1012B00008FB00BF4DF808EDFFF7EAFF34BF01203F
:1012C00000205DF808FB00BF4DF808EDFFF7E0FFD8
:1012D00094BF012000205DF808FB00BF4DF808ED29
:1012E000FFF7CEFF94BF012000205DF808FB00BF90
:1012F0004DF808EDFFF7C4FF34BF012000205DF872
:1013000008FB00BF11481249026800608A4218D0E9
:10131000002103E00F4B5B58435004310E480F4B44
:1013200042189A42F6D30E4A02E0002342F8043BE8
:101330000C4B9A42F9D3FCF74BFD00F019F87047BB
:10134000FEE70948D0F800D040680047FC9F002025
:10135000EFBEADDE287F01080000002078010020EC
:1013600078010020A02A002000D8FF1FFEE700001F
:101370002DE9804895B0EEF707FFB34CB34F2378C3
:10138000396843B1B24B1B68CB1A002BA1BFB14ADD
:10139000002323701370DFF810B3DBF8000042F273
:1013A000010303400BB9AA4A1371030740F193816B
:1013B000A94B1B681B7A062B00F27C81DFE813F037
:1013C000070007003400D40010013C013C01A34B8E
:1013D0001A78002A00F06E8100221A70A04B93F850
:1013E00000E0A04B1B6893F800C09F4B93F800806F
:1013F00002229E4EB35C43FA0EF303F00F036345E3
:1014000002F101090CD20B2B9FBFB55C16F80960E5
:1014100005EA080506EB05259CBF954E46F82350C6
:101420000232102AE5D10CE1924B1A78002A00F022
:10143000418100221A70904B904A93F802C093F8B1
:1014400003E05D780CF0070645EA06250EF03F063E
:10145000760146EADC0615601D7956605E7993F8E0
:1014600006C0AD0045EA9E1506F0010E45EA8E2540
:10147000956093F807E00CF00F05ED0145EA56057D
:101480000EF07F06D56036011D7A46EA1C1693F8E9
:1014900009C016616D000CF0030645EADE1545EA49
:1014A000462593F80AE05561DD7A0EF01F06B60175
:1014B000ED0046EA9C0645EA5E1593F80DC093F8E8
:1014C0000EE0D5611D7B96610CF0070645EA062506
:1014D0000EF03F06760146EADC061562DD7B5662B9
:1014E0001E7C93F811C0AD0045EA9E1506F0010E72
:1014F00045EA8E25956293F812E00CF00F05ED0198
:1015000045EA56050EF07F06360146EA1C16D562FE
:10151000DD7C166393F814C06D0045EADE150CF00F
:10152000030693F815E045EA462555630EF01F06BD
:101530009D7DDB7DB60146EA9C06ED0045EA5E1521
:101540009663DE07D5634CBF40F21475AD25156474
:101550009D074CBF40F21475AD2513F0080F55647C
:1015600014BF03230123A6E0454A1378002B00F0A3
:10157000A18000231370434ADFF830E11678424D12
:101580000EEB460CB5F800809CF803909CF80450D4
:1015900045EA0925A84540F08D809EF80150012DAF
:1015A00004D0812D40F08780032300E02B46102ECD
:1015B00084BF10251570354D92F800E00022D6B298
:1015C000764505F1020576D215F802CC15F8016CC6
:1015D00046EA0C26DFF8D8C02CF812600132EEE79C
:1015E0002B4B1A78002A65D000221A70294B1A78E2
:1015F000A82A1E465ED1DA7C002A5BD106EB4205A2
:101600009FED257A95F803E02B7903EB0E2307EE87
:10161000903AF8EEE77A214BC7EE877A9FED207A71
:1016200077EEC77AFCEEE77A17EE905A43F822502D
:101630000132082AE2D104E01A4B1A78D2B3002210
:101640001A70012337E000BF6C0D0020782A0020BB
:10165000780100206D0D0020342A0020DD100020CC
:10166000222500201C25002023250020CD1000204D
:1016700048100020322A0020192A0020602900206A
:10168000E9290020EC290020EA290020F029002087
:10169000FE100020E9100020CDCCCC4078100020B6
:1016A0000080BB4344100020382A0020ED29002090
:1016B000981000200023DA070DD59B4A01251571EB
:1016C0009A4DC3F340032B7083F00103237001F59F
:1016D000C333A0331360460411D5954A13780BB178
:1016E00000251570904A13714BB1012323708F4B65
:1016F00000241C7001F5433303F5A0731360C50784
:101700000FD5894B5C799A79A2420AD0894A9C719B
:1017100001251570884A0025157001F5C332A032E5
:101720001A60840409D50023844A32F81320002A61
:1017300041F02A8601330C2BF6D17B4C237923B957
:101740007F4B1B68CB1A002B0DDBA368C91A11F164
:10175000500F02D4744B1B7B2BB1F0F7D1FA01234D
:10176000637323730DE023695A1C22611BB9800344
:1017700001D5F6F700FE2369002BC2BF6A4B002299
:101780001A61FDF72DFC6F4B38600DADDB68284604
:1017900098479DF8343033B96B4BA2681B689B1A8D
:1017A000642B00F10487DFF8C8813B68D8F800207B
:1017B000664E1344A36000232373654B3068198879
:1017C000643001B10221FAF781F9FDF709FCD8ED87
:1017D000000ADFED607A63695F4A3860F8EE600AFC
:1017E000C31A60EEA70A5D4FC2ED000A5C4A606151
:1017F0009BB23B80AE4602F1080810685168F4467F
:10180000ACE8030008324245E646F6D110689288FB
:10181000CCF80000ACF80420BDF8409051480021FD
:101820000022844696463CF8028F35F802A02CF838
:10183000028C02320C2A18FB0AEEF4D1DFF834C114
:101840003CF81120828112FB09EE4FF480729EFB5E
:10185000F2FE2CF811E00131032900F10E00DFD176
:1018600007EE903ADFF8C080B4F8425008F1440027
:10187000B8EE670A0121F7F777FABCEEC00A637B7E
:101880008DED050ABDF81400B5FBF0F0451CADB2B6
:10189000A4F84C5033B3B8F84E30059300232249D6
:1018A000314ABDF814A032F8138001F1580C01F14F
:1018B00050093CF813E039F813202CF81380CEEBD4
:1018C000080E12FB0AF20FFA85FA92FBFAF2724442
:1018D00029F813200133042BE1D100234B73A1F825
:1018E0004E0004E0B8F84E30013BA8F84E30B4F892
:1018F0004E000D4A03B2002B4FF000033CDDB2F95D
:101900004C501A4931F81320083112FB00F231F81B
:10191000131092FBF5F28A1A134921F813200133B0
:10192000042BEED12AE000BF780100200300002044
:101930007E0E00206D0D002004000020CC29002028
:10194000440D0020B0190020782A0020D80E002075
:10195000980E0020BD37863550190020880E0020D3
:101960004442010890010020821C0020C801002090
:10197000000F0020C20E0020A2F84E30F1F732FA1C
:10198000BC4BBD4D1B68DFF8408313F4801F00F093
:101990009380B5F8009009F400691FFA89F9B9F14C
:1019A000000F76D1B54B1B78590772D54FF4006004
:1019B000F7F718FDD8F8003023661978B04A0229E5
:1019C00006BF012182F8641082F86490B3F85C20AD
:1019D00094F864904FF47A7353433A8893FBF2F38C
:1019E000A84A5B4292F800C0226E9BB2A4F866300F
:1019F00002F12007002092F857E092F85410BEF14F
:101A0000000F01D0714504D8BCF1030F05D802289E
:101A100003D14FF0000E82F857E0DFF8B0E2B9F1E1
:101A2000000F19D007EE901A97ED007AF2EE046AD3
:101A3000F8EEE77A27EE267AB4EEE77AF1EE10FABE
:101A400044BFC7EEA67AC7ED007AD7ED007AFDEE67
:101A5000E77A17EE901A05E092F801A08A4538BFA0
:101A60005170517889012EF81010854901F16E0EE0
:101A70004FF0000A2EF810A001F1740E01322EF87A
:101A800010300130032807F10407B4D1012381F895
:101A90007A302B881A051AD4784B1B7803F004038C
:101AA00003F0FF079BB994F87A3083B1F7F734FF5E
:101AB000734B83F87A700AE02B881B0507D56F4BB0
:101AC0001B785F0703D54FF40060F7F77BFC6E4B84
:101AD000DFF8FC911B786D4FABB16D4BB3F906206D
:101AE000B9F898319A420EDC99F80530012B01D0F3
:101AF000192B02D199F8E6212AB90E2B03D0082B15
:101B00001CBF0023BB80D8F8003093F82481B8F1C3
:101B1000000F46D02B88980743D09FED5E8ADFEDFB
:101B20005E7A88EE088AB4EEE78AF1EE10FA34D9CC
:101B3000B7EE000A30EE480A01F04CFF9FED577AED
:101B4000DFED577AE8EE077A9FED567AA8EE277A0E
:101B5000DFED557AE8EE077A20EE270AD4ED1F7AFA
:101B600020EE270A01F08EFEB0F5617FA8BF4FF48A
:101B7000617007EE900AB8EEE70ADFED4C7A80EE6E
:101B8000270AF7F7B7FB07EE908AF8EEE77A27EE19
:101B9000800A01F077FE80B200E00020FB88184444
:101BA000F880434B3068B9F86C210093414B1D68B5
:101BB000414B196800F16403A847324B3F491E7836
:101BC000032E15D9D4F880305D88B5F5FA7F0FD291
:101BD000B7F90400B1F904E00028B8BF40426A42F6
:101BE000131A9E4503DB2B187345A8BF73468B80E1
:101BF000FD88B1F800E04F88D4F880C0B1F90480C6
